:020000020000FC
:0E0000000C940E0B0C9400000C9400000C9459
:10000E0000000C9400000C94020C0C94300C0C9418
:10001E005E0C0C948C0C0C949E0C0C94A50C0C94F5
:10002E0000000C9400000C9400000C9400000C9442
:10003E0000000C9400000C94240F0C9400000C94FF
:10004E0000000C9400000C94300F0C9400000C94E3
:10005E0000000C9400000C94AA120C9400000C9456
:10006E0000000C9400000C9400000C9400000C9402
:10007E0000000C94480E0C9400000C9400000C949C
:10008E0000000C9448140C9400000C9400000C9486
:10009E0000000C9400000C9400000C94810E0C9443
:1000AE0000000C9400000C9400000C9400000C94C2
:1000BE0000000C9400000C9400000C9400000C94B2
:1000CE0035160C9400000C9400000C94A9170C9497
:1000DE0000000C9400001027E80364000A000100E1
:1000EE0000100001100001004D6F6E746167004D2D
:1000FE006F6E646179004469656E73746167005454
:10010E00756573646179004D697474776F63680007
:10011E005765646E657364617900446F6E6E6572C7
:10012E007374616700546875727364617900467206
:10013E006569746167004672696461790053616D27
:10014E007374616700536174757264617900536FE3
:10015E006E6E7461670053756E64617900002042A3
:10016E00726964676520626F61726420666F756E76
:10017E0064002072756E6E696E6720626F617264C4
:10018E0020686172647761726520746573742E2EB7
:10019E002E2E00444332632E30342E3035623032F0
:1001AE002E30332E323032330044433220535776C2
:1001BE0065723A2000444332635F6F6374323032AB
:1001CE0032004443322048577665723A2000504F31
:1001DE0032655F6E6F763230323200504F322048C9
:1001EE00577665723A200052616D204572726F72B9
:1001FE000052616D204F4B00202044433220746921
:10020E006D653A2000202044433220646174653AC3
:10021E0020005254432F545749206572726F72005A
:10022E002020696E742E20656570726F6D20657268
:10023E00726F72002020696E742E20656570726F69
:10024E006D204F4B004443322055494420696E20A7
:10025E006865783A20004443322055494420696E3F
:10026E00206465633A2000766F6C74616765206563
:10027E0072726F720020496E70757420766F6C7496
:10028E00616765205B6D565D3A200054656D706543
:10029E00726174757265206572726F72002054659A
:1002AE006D7065726174757265205BB0435D3A2046
:1002BE000020206469676974616C20746573742012
:1002CE006572726F723A20002020646967697461EA
:1002DE006C2074657374204F4B005254432D436C45
:1002EE006F636B206572726F72005254432D5457B8
:1002FE0049206572726F72005254432069732077E1
:10030E006F726B696E67006F766572616C6C2073CD
:10031E00756363657373006F766572616C6C2066CE
:10032E0061696C757265006578742E2065657072F2
:10033E006F6D206572726F72006578742E20656520
:10034E0070726F6D203332206B42204F4B006578F8
:10035E00742E20656570726F6D203634206B4220CE
:10036E004F4B006578742E20656570726F6D203965
:10037E00366B42204F4B203F3F3F006578742E2056
:10038E00656570726F6D20313230206B42204F4B9D
:10039E000000676F74206D6462204E414B006D64E7
:1003AE00622072657370206572726F720072657072
:1003BE006561742073746F70006D6462206F666681
:1003CE00006D6462206F6E006D64622073746172E2
:1003DE007420706F6C6C696E67006D64622073744C
:1003EE006F7020706F6C6C696E67006D6462207246
:1003FE00657065617400656D70206F666600454DB1
:10040E005020636F756E7472793A2000454D5020FE
:10041E007363616C653A2000454D502064656369D5
:10042E006D616C733A2000656D7020706179207378
:10043E00746172742000656D702070617920737420
:10044E006F702000656D7020676F742068436F6950
:10045E006E2000656D7020676F7420636F696E206B
:10046E0000656D7020726420657272002D64796E65
:10047E005072302D002D64796E5072312D002D6426
:10048E00796E5072322D002D64796E5072332D00BC
:10049E002D64796E5072342D002D64796E50723544
:1004AE002D002D64796E5072362D002D64796E50AC
:1004BE0072372D002D2D2D2041544220476D62485C
:1004CE00202D2D2D002D2D2D205053412031323534
:1004DE0036202D2D2D002D2D205465737420507235
:1004EE00696E74202D2D004C4F474F3A0051523AF1
:1004FE00002041544220476D6248202D2D2D205062
:10050E00534131323536202D2D2D205072696E74A7
:10051E0065722074657374202D2D2D200A20415490
:10052E00422D5072696E74657220697320776F72F6
:10053E006B696E6720636F72726563746C79200AE3
:10054E002020205468697320697320616E20415405
:10055E0042205152636F64652D74657374203A297D
:10056E00202000426172436F646520322F353A00BD
:10057E00313233343536373839303132333435362B
:10058E0037383930002D2D2D2D2D2D2D2D2D2D2D96
:10059E002D2D2D2D2D2D2D2D2D2D2D0020202020DE
:1005AE00207468697320697320612074696E7920E4
:1005BE0074657874006E6F726D616C2074657874FA
:1005CE000074686973206973206120686967682008
:1005DE0074657874002020426F6C642054657874C2
:1005EE002000756E6465726C696E65642074657842
:1005FE00740020696E76657273207465787400706D
:10060E0072696E7465722074656D706C61746520AC
:10061E00002D2D2D20656E64206F662066696C6539
:10062E00202D2D2D00444F57206E6F74207365744E
:10063E000074686973206973206120322F356261FE
:10064E0072636F646500205468697320697320615A
:10065E006E204154422044656D6F205152636F6489
:10066E00652020003C20536C6176652052657370C6
:10067E006F6E736500444332635F6F637432303262
:10068E003200504F32655F6E6F7632303232004438
:10069E004332632E30342E30356230322E30332ECC
:1006AE003230323300007468697320697320616ED2
:1006BE0020415442206163636573732063617264E9
:1006CE00000044436D616B655265736574002D00C7
:1006DE00776F6B656E206279206D646200776F6B49
:1006EE00656E20627920636F696E00776F6B656E41
:1006FE00206279207074750074726967676572691B
:10070E006E67206865617274626561742E2E2E00AC
:10071E00414C41524D00706F77657220646F776E59
:10072E00006C696768742077616B650066756C6C28
:10073E002077616B65007374617274696E672062F5
:10074E006F6F746C6F616465722E2E2E000074656F
:10075E0073742063616E63656C6C656400737461A1
:10076E007274696E6720436F696E436865636B656B
:10077E007220746573742E2E2E0077696C6C206255
:10078E00652073746F707065642061667465722085
:10079E0032307320776974686F757420636F696E79
:1007AE0000496E7365727420636F696E7320706C8E
:1007BE00656173653A00656D7020696E2069646CC1
:1007CE006520737461746500656D702073746F704D
:1007DE0000656D702077616974696E6720666F724F
:1007EE0020636F696E7300207E3E2076616C7565A6
:1007FE003D00636F696E207465737420656E6400CE
:10080E0072756E6E696E6720737461727475702086
:10081E0074657374732E2E2E0052616D204F4B0033
:10082E0052616D206572726F7220666F756E640014
:10083E00426F617264206877204F4B00426F617285
:10084E0064206877206572726F7220005274632084
:10085E006572726F722000527463206F6B0055695F
:10086E0064206572726F722000556964206F6B0090
:10087E00557070657220646F6F72206973206F708F
:10088E00656E005661756C7420646F6F72206973AB
:10089E00206F70656E004261747465727920646FAA
:1008AE006F72206973206F70656E00446F6F727384
:1008BE00206F6B0054656D70657261747572652082
:1008CE006572726F72200054656D70657261747519
:1008DE007265206F6B00566F6C7461676520657270
:1008EE00726F722000566F6C74616765206F6B00BB
:1008FE00496E746565206572726F722000496E7460
:10090E006565206F6B004578746565206572726F42
:10091E007220004578746565206F6B00436F696EB9
:10092E0020657363726F77206572726F7220004359
:10093E006F696E20657363726F77206F6B005072F4
:10094E00696E746572206572726F722000202020AD
:10095E006E6F207061706572002020206E6F7420A3
:10096E007265616479002020206E6F20726573704D
:10097E006F6E736500202020696E7465726E616CF7
:10098E00206572726F720020202068656164206F8E
:10099E0070656E005072696E746572206F6B002008
:1009AE0020206C6F77207061706572004E6F20632F
:1009BE006F696E207361666500436F696E207361A7
:1009CE006665206F6B004E6F2062696C6C20626FE3
:1009DE00780042696C6C20626F78206F6B004D64FA
:1009EE0062206572726F72004D6462206F6B004DF3
:1009FE006966526561646572206F6B004D6966525F
:100A0E006561646572206572726F7220004368655D
:100A1E00636B696E67206D6F64656D2C20706C73EF
:100A2E0020776169742E2E2E00436F696E206368E5
:100A3E0065636B6572206F6B00436F696E20636830
:100A4E006B206572726F722000466F756E64204562
:100A5E0052524F522873290053797374656D206F6B
:100A6E006B00444332632E30342E30356230322EDA
:100A7E0030332E32303233004443322053577665B2
:100A8E00723A2000444332635F6F63743230323205
:100A9E00004443322048577665723A2000504F3258
:100AAE00655F6E6F763230323200504F32204857CB
:100ABE007665723A20004D6F64656D206F6B007223
:100ACE00656769737465726564005369676E616CFE
:100ADE0020004D6F64656D206572726F7220007715
:100AEE00726F6E6720747970650053494D206E6F7A
:100AFE00742072656164790074657374696E672021
:100B0E007072696E7465722E2E2E000041542B4346
:100B1E0053510041542B435245473F0041542B4300
:100B2E004C54533D3F002B4353513A20002B43521C
:100B3E0045473A2000415400524459004F4B004162
:100B4E005445300041542B434C54533D31004154D5
:100B5E00490053494D37303030470041542B4353F1
:100B6E00494D3D3F000006046F04DF045705D705CD
:100B7E005E06EC0682072008C5087109250AE10AFF
:100B8E00A40B6E0C400D170EE90EA80F4610B810F0
:100B9E00301106046F04DF045705D7055E06EC0618
:100BAE0082072008C5087109250AE10AA40B6E0CFC
:100BBE00400D170EE90EA80F4610B81030110001A7
:100BCE0002030405060708090A0B0C0D0E0F001090
:100BDE0000006410B71DC8206E3BAC30D926904182
:100BEE00DC76F4516B6B5861B24D3C71055020832D
:100BFE00B8ED44930FF0E8A3D6D68CB361CBB0C258
:100C0E00649BD4D2D38678E20AA01CF2BDBD417497
:100C1E006250736131323536507475355F2100374D
:100C2E0078A730203F3F660041544256414C55450F
:100C3E004341524456303032000066696C6520697B
:100C4E007320746F6F206269672C206D6178203578
:100C5E00303062797465002D2D2D2D2D2D2D2D2DDD
:100C6E002D2D2D2D2D2D2D2D2D2D2D2D2D2D2D2DA6
:100C7E002D2D2D2D2D2D2D2D2D2D2D2D2D2D2D2D96
:100C8E002D2D2D2D2D2D2D2D2D002D2D2D2D2D2DB3
:100C9E002D2D2D202044657669636520436F6E747B
:100CAE00726F6C6C65722048656C70205363726550
:100CBE00656E202D2D2D2D2D2D2D2D2D007C2D2DC8
:100CCE002D2D2D2D2D2D2D2D2D2D2D2D2D2D2D2D46
:100CDE002D2D2D2D2D2D2D2D2D2D2D2D2D2D2D2D36
:100CEE002D2D2D2D2D2D2D2D2D2D2D2D2D2D2D0053
:100CFE007C007C202020275027203D2044697370E3
:100D0E006C6179204D616368696E652053657474FA
:100D1E00696E6773007C202020275327203D2044D6
:100D2E006973706C617920446576696365205374CC
:100D3E00617465007C202020274427203D204469D3
:100D4E0073706C61792044796E616D6963205661B0
:100D5E006C756573007C202020275727203D20448A
:100D6E006973706C61792057616B6520536F757272
:100D7E006365007C2020202754787827203D20446E
:100D8E006973706C6179205469636B6574206E723F
:100D9E00207878203D2030312E2E3332007C2020DA
:100DAE0020277427203D2052756E20636F6D706C66
:100DBE006574652073797374656D20636865636B04
:100DCE00202831377329007C202020277027203DD2
:100DDE00205072696E7420546573747469636B6508
:100DEE0074007C202020276327203D2052756E2022
:100DFE00636F696E2074657374007C2020202764F5
:100E0E00787827203D205072696E74205469636B88
:100E1E006574206E72207878203D2030312E2E336E
:100E2E0032007C202020276B636363636327203DA1
:100E3E0020656E6361736820616D6F756E74202816
:100E4E00356469676974732920696E2063656E74F1
:100E5E00007C20202073656E64206A736F6E2D6691
:100E6E00696C652077697468202253454E4420468C
:100E7E00494C452D427574746F6E004D61636869FF
:100E8E006E652053657474696E67733A00437573AB
:100E9E00746F6D65724E723A20004D616368696EB3
:100EAE00654E723A202000426F726F7567683A2065
:100EBE00202020005A6F6E653A202020202020200E
:100ECE0000416C6961734E723A20202020004D79EA
:100EDE00506C6163653A20004D61737465722049F0
:100EEE006E746572666163653A0043757272656E03
:100EFE00742042617564726174653A20002020206E
:100F0E0020303D393630302020313D31346B3420A5
:100F1E0020323D31396B322020333D33386B342053
:100F2E0020343D35372C362020353D3131356B326E
:100F3E002020363D3233306B3400437263206368B9
:100F4E0065636B3A20005061726974793A00202013
:100F5E00202020202F2F207061726974793A203062
:100F6E003D6E6F2020313D6576656E2020323D6FDF
:100F7E0064640044617461626974733A20002020D5
:100F8E00202020202F2F20646174612062697473E9
:100F9E003A20303D356269742020313D36626974E5
:100FAE00202020323D37626974202020333D386284
:100FBE006974202020343D396269740053746F7057
:100FCE00626974733A20002020202020202F2F20C9
:100FDE00303D3173746F7062697420202020313D72
:100FEE003273746F706269747300446576696365F9
:100FFE00733A005072696E7465722020203A200098
:10100E00436F696E43686B2020203A20004D69665D
:10101E00617265202020203A20004D61696E735365
:10102E007570706C793A20004D6F64656D202020CC
:10103E0020203A2000437265646974436172643AF9
:10104E002000457363726F77202020203A200052D3
:10105E00656A4D6F746F7220203A20005368757464
:10106E007465722020203A200042696C6C2020208A
:10107E002020203A20005661756C744C6F636B20F3
:10108E003A20004175746F416C61726D203A2000F8
:10109E004175746F4F70656E20203A200053746155
:1010AE007465206F6620616C6C204465766963659B
:1010BE00732028313D4F4B20203178783D77617277
:1010CE006E696E6720203278783D6572726F722974
:1010DE000052616D3A2000496E7445653A20004514
:1010EE00787445653A20005274633A200042726467
:1010FE002048573A200050726E3A20004D6F6465BA
:10110E006D3A20005369676E616C3A200052656734
:10111E006973743A20004D64624275733A2000433D
:10112E006F696E43686B3A2000457363726F773A4E
:10113E0020004D6966526561643A20004343746530
:10114E00726D3A200052656A6563743A20005661EA
:10115E00756C743A200042696C6C626F783A2000AC
:10116E00566F6C743A200054656D703A20005077BB
:10117E00724F6E5473743A2000446F6F72537461E1
:10118E0074653A2000446F6F725761734F70656ECD
:10119E003A20004368616E6765723A2000436F69BA
:1011AE006E536C6F743A200042696C6C3A20004C9E
:1011BE006173742052657365742062793A20004120
:1011CE006C6C20436865636B65643A2000416C610A
:1011DE00726D3A2000444332632E30342E30356225
:1011EE0030322E30332E32303233004443322053DD
:1011FE00577665723A2000444332635F6F637432F0
:10120E00303232004443322048577665723A20001D
:10121E00504F32655F6E6F763230323200504F3241
:10122E002048577665723A2000616C6C2064796EA6
:10123E00616D69632076616C7565733A006B6570DC
:10124E0074206177616B652062793A2000006572C7
:10125E00726F7220696E20636F6E666967206669B1
:10126E006C6500636F6E6669672075706461746586
:10127E002073756363657373006572726F72206994
:10128E006E2073657269616C2066696C65007365AA
:10129E007269616C20757064617465207375636327
:1012AE00657373006572726F7220696E2064657665
:1012BE006963652066696C6500646576696365209F
:1012CE00757064617465207375636365737300650F
:1012DE0072726F7220696E20636173682066696C2A
:1012EE006500636173682075706461746520737541
:1012FE006363657373006572726F7220696E20701E
:10130E0072696E7478782066696C65007072696EA9
:10131E007478782075706461746520737563636585
:10132E007373006572726F7220696E2074696D65D9
:10133E002066696C650074696D65207570646174F2
:10134E006520737563636573730077726F6E6720C4
:10135E0066696C65007469746C65003F3F3F444379
:10136E0032435F636F6E666967003F3F3F444332AF
:10137E00435F73657269616C003F3F3F4443324384
:10138E005F646576696365003F3F3F444332435F68
:10139E00636173682020003F3F3F444332435F70D8
:1013AE007269003F3F3F444332435F74696D65008D
:1013BE00637573744E756D006D6163684E756D0067
:1013CE00626F726F756768007A6F6E6500616C6927
:1013DE006173006C6F636174696F6E006372634357
:1013EE00686B00626175645261746500646174615A
:1013FE00007061726974790073746F700070726935
:10140E006E74657200636F696E43686B006D69661A
:10141E00526400736F6C6172507772006D6F646509
:10142E006D00637265646974436172640065736311
:10143E00726F770052656A4D6F746F7200736875C4
:10144E00747465720062696C6C5264007661756CBE
:10145E00744C6F636B006175746F416C61726D00DB
:10146E006175746F4F70656E007265736572766527
:10147E00006C6F63616C436F696E4163636570747A
:10148E00004E616D65206F6620437572006C6F6350
:10149E00616C20746178207261746500666F72658C
:1014AE0069676E436F696E56616C75650043757240
:1014BE0072656E63794E616D6500666F7265696700
:1014CE006E2074617800546F6B656E4368616E6E4A
:1014DE00656C0042696C6C7328372E2E30290073B0
:1014EE00757263686172676500646973636F756EA8
:1014FE007400657863686752617465006375727213
:10150E002E7965617200637572722E6D6F6E7468DE
:10151E0000637572722E646F6D00637572722E6841
:10152E006F757200637572722E6D696E00637572DF
:10153E00722E73656300637572722E646F7700701E
:10154E00726F6A656374007465787400697373757D
:10155E006564007374796C0066656564007661720B
:10156E00690067726166000063617368207374615D
:10157E007274207061796D656E740063617368209A
:10158E0073746F70006361736820726561647900B3
:10159E0063617368206C61737420636F696E0020E1
:1015AE006361736820676F7420636F696E3A200001
:1015BE0063617368207374617274436F6C6C20770F
:1015CE006974682000636173682073657475702098
:1015DE000073746F70207061796D656E7420617424
:1015EE0020000A00000000000000000000000000C3
:1015FE0000000000000000000000000000000000DD
:10160E00000000000100391CF01500000000F894E5
:10161E00EE27EFBBF1E0F5BFE5BFE0937400E0937A
:10162E0075008DE0A2E0BB27ED938A95E9F780E087
:10163E0090E2A0E0B2E0ED930197E9F7E2E1F6E186
:10164E00D0E0DBBF87919791009781F0A791B7917A
:10165E0007901790C791D791BF01DBB7F001CBBFB1
:10166E0007900D920197E1F7FB01EBCFE0E0EEBBA7
:10167E00EFEFEDBFE1E2EEBFC0E0DAE00C94A56E55
:10168E000E94AEB91A2F2B2F3C81343010F40C94DB
:10169E00510B30E03295307F330F330F307C309367
:1016AE007C00E7E9E0937A00012FAEE7B0E0EC9121
:1016BE00E02BEC93EFEF0E27E0B3E023E0BB122F0D
:1016CE002227012FADE7B0E0EC91E02BEC93EFEF8A
:1016DE000E27A7E0B1E0EC91E023EC930E94B5B9A0
:1016EE0025960895E0E0E0937A0008950A930A2F74
:1016FE00003110F40C94860BE0E009910895083047
:10170E0010F40C94910BE0917B00E860E0937B0069
:10171E00077005C0E0917B00E77FE0937B00083007
:10172E0010F00C94A90BE0917C00E87FE0937C0014
:10173E00ACE7B0E0EC91E02BEC93E0917A00E06442
:10174E00E0937A00E1E0099108950E94AFB900E0BC
:10175E0010E0E0917A00E0712E2F81E791E0019781
:10176E00F1F7203011F00C94C60BF80131968F0171
:10177E00E436A0E0FA0710F00C94C60B01C001C0CD
:10178E00E8CFE0917A00E061E0937A000091780072
:10179E0010917900F8010E94B6B923960895E0E001
:1017AE00EDBBE093680008950A930A2F003011F004
:1017BE000C94EA0BE0916A00E2600E942EA5EE7F87
:1017CE00E0936A00EC9A013011F00C94F40BE09166
:1017DE006A00E360E0936A00EC9A023011F00C9418
:1017EE00FE0BE0916A00EC7FE0936A00EC9A09919F
:1017FE000895EC9808950E9433A50E94B4720E9439
:10180E0045A518950A930A2F003011F00C94180C68
:10181E00E0916A00E8600E942EA5EB7FE0936A00DB
:10182E00ED9A013011F00C94220CE0916A00EC60FC
:10183E00E0936A00ED9A023011F00C942C0CE091BA
:10184E006A00E37FE0936A00ED9A09910895ED989E
:10185E0008950E9433A50E94C8720E9445A518954E
:10186E000A930A2F003011F00C94460CE0916A0096
:10187E00E0620E942EA5EF7EE0936A00EE9A0130A0
:10188E0011F00C94500CE0916A00E063E0936A0052
:10189E00EE9A023011F00C945A0CE0916A00EF7C33
:1018AE00E0936A00EE9A09910895EE9808950E94C9
:1018BE0033A50E94DB720E9445A518950A930A2F44
:1018CE00003011F00C94740CE0916A00E0680E94F4
:1018DE002EA5EF7BE0936A00EF9A013011F00C9485
:1018EE007E0CE0916A00E06CE0936A00EF9A0230A1
:1018FE0011F00C94880CE0916A00EF73E0936A008B
:10190E00EF9A09910895EF9808950E9433A50E94C9
:10191E00EE720E9445A518950E9457A50E9457A5E4
:10192E000E9457A5A8E6B0E0EC91EC9308950E94B2
:10193E0033A50E9445730E9445A518950E9433A5B4
:10194E000E9448730E9445A518950D9400F00895C5
:10195E000E945DA5F99B01C0FDCF22BD11BDF89A75
:10196E0000B50E9462A508950E9467A5F99B01C06B
:10197E00FDCF09851A852F81388540E0F901A42F06
:10198E00B0E0AE17BF0710F00C94D80C0E946CA5F7
:10199E00AD81BE81EE27A40FBE1FE0B5EC934F5F65
:1019AE00EDCF0E94B4B92B9608950E94ADB92A2F9F
:1019BE003D814E81F99B01C0FDCF1FB742BD31BDA8
:1019CE00F89A00B5201711F40C94F20C20BDE4E047
:1019DE00EFBBE2E0EFBB17FF01C078940E94B4B9F1
:1019EE00279608950E9473A5F99B01C0FDCF0C8523
:1019FE001D852A853B85EFB7EE8340E0F901A42FC4
:101A0E00B0E0AE17BF0710F00C94260DA885B9856F
:101A1E00EE27A40FBE1F5C910E946CA5E0B5EF836C
:101A2E00AF815A1711F40C94240D50BDE4E0EFBBB6
:101A3E00E2E0EFBBF99B01C0FDCF4F5FDFCFEE8140
:101A4E00E07811F40C942C0D78940E94B3B92E9674
:101A5E0008950A932B9823982A98229A2998219AC6
:101A6E00289A209A02E0E02FE03011F00C94440DF9
:101A7E00E1E0EDBDE0E5ECBD35C0E13011F00C94D8
:101A8E004D0DE0E0EDBDE0E5ECBD2CC0E23011F017
:101A9E000C94560DE1E0EDBDE1E5ECBD23C0E33065
:101AAE0011F00C945F0DE0E0EDBDE1E5ECBD1AC068
:101ABE00E43011F00C94680DE1E0EDBDE2E5ECBD13
:101ACE0011C0E53011F00C94710DE0E0EDBDE2E5D2
:101ADE00ECBD08C0E63011F00C94790DE0E0EDBDE0
:101AEE00E3E5ECBD09910895E0E0ECBD0895E0E07A
:101AFE00E4BDE5BDE0936E00E093B000E093B1006D
:101B0E00E0937000E093B600E3BDE0938000E093B5
:101B1E009000E093A000E0932001E0938100E09319
:101B2E009100E093A100E0932101E0938200E09305
:101B3E009200E093A200E0932201E0936F00E09305
:101B4E007100E0937200E093730008951A930A9364
:101B5E001CE0E3B70E2FAE2FE5E0EA23AE2FE5E053
:101B6E000E944BBAE03011F40C94CE0DE12FE150EF
:101B7E001E2FEF5FAE2FEAE00E9455BAE03011F44F
:101B8E000C94CA0DF3CFE0E0099119910895E0E0AD
:101B9E00E4BDE1E0E5BDE0E0E7BDE6EBF0E0DF014E
:101BAE00E0E0EC93E6BDE6B5AE2FE7E30E9450BA57
:101BBE00E03011F40C94E40DF6CFE0E009911991A8
:101BCE0008950E94AEB99D017894E0E0F0E08F0197
:101BDE000E94AD0DF80131968F013197F801FF93F8
:101BEE00EF93F901AF91BF910E9460BAE03011F40A
:101BFE000C94020EEDCFE7E0F0E08F018F010E9412
:101C0E00B5B9249608950E94ACB9AD01FA019F01B1
:101C1E00E0E0F0E08F01E4E6F0E0DF010E94E80D85
:101C2E00F80131968F013197F801FF93EF93F90187
:101C3E00AF91BF910E9460BAE03011F40C94280E5F
:101C4E00EACFE8E0F0E08F018F010E94B3B926964B
:101C5E000895E0E0E0939000E09392000E9479A551
:101C6E00E0917100E260E0937100E2E0E093910098
:101C7E00E8E4E0939900E0E0E0939800EFEFE8BB32
:101C8E0008950E9433A50E9479A5A0E0BAE00E94B3
:101C9E007FA50E944073A4E0BAE00E947FA5A091A8
:101CAE00040AB091050AA436E0E0BE0710F40C94C5
:101CBE006B0EE0E0E093040AE093050AA2E0BAE0BE
:101CCE000E947FA50E943F73EFEFE8BB0E9445A5DF
:101CDE001895A0919100A03011F40C947D0EA09156
:101CEE007100A03011F40C947D0E02C0E0E0089556
:101CFE00E1E0089518950A930A2F083210F40C9417
:101D0E008B0EE1E009910895E02F0E9485A5EA0F60
:101D1E00FB1FA091000AB091010AA083B183E0E0FD
:101D2E00099108950E94ACB95A2F583210F40C94B0
:101D3E00A40E0E948BA526960895452F2091000A89
:101D4E003091010AE42F0E9485A50E9490A510F4FF
:101D5E000C94BC0EE42F0E9485A50E9497A5DF016E
:101D6E00F901EA1BFB0B8F0107C0E42F0E9485A52A
:101D7E000E9497A50E949CA5F8010E94B3B92696D1
:101D8E0008950A930A2F0F3010F40C94D10EE1E04F
:101D9E0009910895E02F0E94A6A5EA0FFB1FA091BE
:101DAE00020AB091030AA083B183E02FF0E0EC5851
:101DBE00F54FA1E0A08309910895AA930E94ADB9B1
:101DCE004D814F3010F40C94F20EE0E0F0E00E94E2
:101DDE00B4B926960895E42FF0E0EC58F54FE08163
:101DEE00E03011F00C94010FE0E0F0E00E94B4B985
:101DFE00269608952091020A3091030AE42F0E943C
:101E0E00A6A50E9490A510F40C94180FE42F0E9422
:101E1E00A6A50E9497A5DF01F901EA1BFB0B8F0116
:101E2E0007C0E42F0E94A6A50E9497A50E949CA51C
:101E3E00F8010E94B4B9269608950E9433A5E0E0F9
:101E4E00E0938500E09384000E9443730E9445A5B1
:101E5E0018950E9433A5E0E0E6BD0E9444730E94EF
:101E6E0045A518952C970A930E94ACA50E94B1A582
:101E7E000E94B6A50E94B6A5EAB1E360EAB9EBB13D
:101E8E00E360EBB9E0916400EF77E0936400E4E087
:101E9E00E093BC00E985FA856B857C850E94BFA521
:101EAE000E94C4A50E94C9A50E94CEA50E94D1A5DC
:101EBE00E051F040604070400E94D6A50E9441BAA9
:101ECE000E94BFA500E00E94C9A5A030E1E0BE07B8
:101EDE00E0E08E07E0E09E0710F40C94800F0E9465
:101EEE00C9A5E4E0F0E060E070E00E94CEA50F5FCF
:101EFE00EACFED81E093B8000093B90008812D96EA
:101F0E000895E0E0E093BC00E0916400E068E093A7
:101F1E006400EAB1EC7FEAB9EBB1E360EBB9089586
:101F2E000E94D9A50F5F1F4F81E38A95F1F7E091CB
:101F3E00BC00E07811F00C94AB0F0436E0E01E0705
:101F4E0014F00C94AB0F01C001C0ECCF0436E0E0EE
:101F5E001E0714F40C94B70FE1E00991199108953E
:101F6E00E0E00991199108950E94DEA5022F409399
:101F7E00BB00303011F40C94C80FE4EAE093BC00BF
:101F8E0003C0E4E8E093BC000E94970F1E2F1130AF
:101F9E0010F40C94D70FEAE00E94B4B92796089576
:101FAE00E091B900E87F0E1711F40C94E60FE4E906
:101FBE00E093BC00E1E00E94B4B927960895E0E0FA
:101FCE000E94B4B9279608950E94AFB90E94880F57
:101FDE00509A51985998AAE0B0E00E9415BDE9B107
:101FEE00E1700E2FE9B1E2701E2F103011F00C943B
:101FFE001C1020E058988AE08A95F1F7589A8AE0EA
:10200E008A95F1F7E9B1E2701E2F2F5F103011F0B3
:10201E000C941610203210F00C94161001C001C052
:10202E00E9CFA2E0B0E00E9415BD103011F40C947F
:10203E0022100E94390FA2E0B0E00E9415BD0E944E
:10204E00B6B9239608950E9473A50E94E4A511F0D7
:10205E000C9434100770000F202B0E94EFA511F482
:10206E000C943C100E94FAA508950E94FFA511F051
:10207E000C944610E2E00E94B3B92F9608953130C9
:10208E0011F00C944D100E9408A60895503011F4D2
:10209E000C9459100E940DA611F40C9459100E9424
:1020AE0016A608950E941BA611F40C9461100E94AE
:1020BE0016A60895E0E0EE83EF830E9424A6AE17E5
:1020CE00BF0710F00C947F100E9429A6AE0FBF1F01
:1020DE00EC91EA93E0E0EA93A8E20E942EA611F4B6
:1020EE000C947C100E9433A608950E9438A6E5CF6A
:1020FE000E943EA608950E9446A60E944DA60E94EA
:10210E002A100E2F013010F40C948F100E94EB0F3A
:10211E00013010F40C9499101F5F153010F00C94D0
:10212E00991001C001C0E9CF7894013010F40C94DD
:10213E00A010E02F0E94B3B92B9608950E9473A5AC
:10214E000E94E4A511F00C94AF100770000F202B25
:10215E000E94EFA511F40C94B7100E94FAA50895F1
:10216E000E94FFA511F00C94C110E2E00E94B3B9D9
:10217E002F960895313011F00C94C8100E9408A6C5
:10218E000895503011F40C94D4100E940DA611F441
:10219E000C94D4100E9416A608950E941BA611F44A
:1021AE000C94DC100E9416A608950E9457A6A0E17A
:1021BE000E942EA611F40C94E7100E94FAA5089521
:1021CE0021602A93E0E0EA93A0E40E942EA611F487
:1021DE000C94F4100E9408A608954150E0E0EE839E
:1021EE00EF830E9424A6EA17FB0710F40C944F11FC
:1021FE000E9424A6EA17FB0711F00C940A11E4E8DA
:10220E00E093BC0003C0E4ECE093BC000E94970F87
:10221E00E03011F40C9416110E9433A60895E0914B
:10222E00B900E87FE03511F00C9425110E9424A628
:10223E00AE17BF0710F00C94251101C008C00E9404
:10224E0029A6AE0FBF1FE091BB00EC931EC0E0911C
:10225E00B900E87FE83511F00C943D110E9424A6D8
:10226E00EA17FB0711F00C943D1101C008C00E9443
:10227E0029A6AE0FBF1FE091BB00EC9306C0E4E9A8
:10228E00E093BC000E9433A608950E9438A6A9CF01
:10229E000E943EA608950E9446A60E944DA60E9448
:1022AE00A5100E2F013010F40C945F110E94EB0F4D
:1022BE00013010F40C9469111F5F153010F00C945E
:1022CE00691101C001C0E9CF7894013010F40C946B
:1022DE007B1110E0E8851E1710F00C947B110E9404
:1022EE005CA6EC931F5FF6CFE02F0E94B3B92B963E
:1022FE000895A091EF0AA23010F40C948B11AE3F0A
:10230E0010F00C948B1101C005C0E091EF0AEF5F45
:10231E00E093EF0AA091590BA23010F40C949C118B
:10232E00AE3F10F00C949C1101C005C0E091590B0A
:10233E00EF5FE093590BA091530DA23010F40C9463
:10234E00AD11AE3F10F00C94AD1101C005C0E0917F
:10235E00530DEF5FE093530DA091BD0DA23010F41D
:10236E000C94BE11AE3F10F00C94BE1101C005C00E
:10237E00E091BD0DEF5FE093BD0D08950A930A2F16
:10238E00E02FE13011F00C94CF11EFE30991089595
:10239E00E23011F00C94D611EFE209910895E3307A
:1023AE0011F00C94DD11E7E109910895E43011F07C
:1023BE000C94E411EFE009910895E53011F00C94BE
:1023CE00EB11E7E009910895E63011F00C94F2114B
:1023DE00E3E009910895EFE5099108950E9461A641
:1023EE00E093C000E0E0E093C100E093C200E09310
:1023FE00C500E4E6F0E0E093ED0AF093EE0AA0915A
:10240E00ED0AB091EE0A139710F00C941412E3E05B
:10241E00F0E0E093ED0AF093EE0AA32F0E94C511AF
:10242E00E093C400E22FE13011F00C942412E091FD
:10243E00C200E260E093C20022C0E23011F00C94C0
:10244E002E12E091C200E460E093C20018C0E330A7
:10245E0011F00C943812E091C200E660E093C200D5
:10246E000EC0E43011F00C944612E091C200E6600A
:10247E00E093C200E091C100E460E093C100E12F5F
:10248E00E13011F00C945012E091C200E860E0933C
:10249E00C200E02FE13011F00C945B12E091C2000B
:1024AE00E062E093C20009C0E23011F00C946412B5
:1024BE00E091C200E063E093C200E42FE13011F03E
:1024CE000C946F12E091C100E861E093C10009C065
:1024DE00E23011F00C947812E091C100E869E093BB
:1024EE00C1000E94B4B929960895E0E0E093C100BE
:1024FE0008950A930A2FE091C000E07211F00C9437
:10250E008912F9CF0093C600099108950E94D9A5AA
:10251E000E946AA60E171F0710F00C949D12A6E8D3
:10252E00BAE00E946FA60F5F1F4FF2CFE0E0E0937C
:10253E00EA0AE093EB0AE093EC0AE1E0E093EF0A9B
:10254E000991199108950E9474A60E94AEB9A091A6
:10255E00EF0AA13010F40C94B712E2E0E093EF0A08
:10256E00E091C100E47011F40C94F1120E946AA67D
:10257E0032970E947BA610F00C94DF12E091C100FE
:10258E00E27011F40C94D3120E9482A63197EA578E
:10259E00F54FA1E0A08307C00E9482A63197EA57AB
:1025AE00F54FA0E0A0830E9482A60E9485A602C0DD
:1025BE000091C600E091EA0AE2501E2FF0E0EA57C1
:1025CE00F54F0E948DA6EA57F54FE081F0E02E2BD5
:1025DE003F2B0EC00E946AA60E947BA610F00C94A0
:1025EE00FD120E9482A60E9485A602C00091C6001E
:1025FE00E091C000EC710E2F013010F40C940E130C
:10260E00A091EC0AA03011F00C940E1301C002C080
:10261E000093EC0A0E94B5B924960E9495A61895CF
:10262E000E949CA608950E94ACB9AD01A091EA0A41
:10263E00B091EB0A4A175B0710F00C942813FA01BD
:10264E0002C00E949CA69F0100E010E00217130733
:10265E0010F00C943B130E94A1A6A6E8BAE00E94CB
:10266E00A8A60F5F1F4FF2CF0E94AEA6A436E0E0E1
:10267E00BE0710F00C9447130E949CA60E94B3A6AE
:10268E000E94B3B9289608950E94BAA60E94C1A6C8
:10269E0010F40C945513A22F0E948012003DE7E017
:1026AE001E0710F00C946013213010F40C9460137C
:1026BE0001C001C0EBCF78940E94B4B9259608955D
:1026CE000E94C9A600E010E00217130710F00C9448
:1026DE007913F801E40FF51FA0810E9480120F5F9D
:1026EE001F4FF2CF0E94B3B9289608950E9461A69B
:1026FE00E093C800E091C900EC79E093C900E09145
:10270E00C900E861E093C900E091CA00EE73E0935E
:10271E00CA00E0E0E093CD00E4E6F0E0E093570B72
:10272E00F093580BA091570BB091580B139710F0D4
:10273E000C94A713E3E0F0E0E093570BF093580BE3
:10274E00A32F0E94C511E093CC00E22FE13011F0CF
:10275E000C94B713E091CA00E2600E94D1A622C089
:10276E00E23011F00C94C113E091CA00E4600E94B3
:10277E00D1A618C0E33011F00C94CB13E091CA002F
:10278E00E6600E94D1A60EC0E43011F00C94D9136D
:10279E00E091CA00E660E093CA00E091C900E460EF
:1027AE00E093C900E12FE13011F00C94E313E091B6
:1027BE00CA00E860E093CA00E02FE13011F00C94FB
:1027CE00EE13E091CA00E062E093CA000FC0E2305F
:1027DE0011F00C94F813E091CA00E063E093CA0084
:1027EE0005C0E091CA00EF7CE093CA00E42FE1300F
:1027FE0011F00C940814E091C900EF77E093C90032
:10280E0009C0E23011F00C941114E091C900E06897
:10281E00E093C90089E18A95F1F70E94B4B929962F
:10282E000895E0E0E093C90008950A930A2FE0911D
:10283E00C800E07211F00C942514F9CF0093CE006D
:10284E00099108950E94D9A50E94D9A60E171F07B7
:10285E0010F00C943914A0EFBAE00E946FA60F5F2F
:10286E001F4FF2CFE0E0E093540BE093550BE09353
:10287E00560BE093BE0DE1E0E093590B09911991CF
:10288E0008950E9474A60A93A091590BA13010F4DA
:10289E000C945714E1E0E093BE0DE2E0E093590B87
:1028AE00E091C900E47011F40C9484140E94D9A62E
:1028BE0032970E94AEA6AE17BF0710F00C9481148B
:1028CE00E091C900E27011F40C9475140E94DEA61A
:1028DE003197E051F54FA1E0A08307C00E94DEA61C
:1028EE003197E051F54FA0E0A0830E94DEA60E9432
:1028FE00E1A602C00091CE0010C00E94D9A60E948F
:10290E00AEA6AE17BF0710F00C9492140E94DEA66E
:10291E000E94E1A602C00091CE00E091C800EC71C9
:10292E000E2F013010F40C94A314A091560BA0306E
:10293E0011F00C94A31401C002C00093560B099120
:10294E000E9495A61895E091560BE03011F00C946C
:10295E00B3140E94E9A60895E091560BE07111F4AC
:10296E000C94BC14EFEFFFEF0895E091560BE87056
:10297E0011F40C94C514EEEFFFEF0895E091560B91
:10298E00E47011F40C94CE14EDEFFFEF089508955A
:10299E000E94ACB9AD010E94AEA64A175B0710F0BB
:1029AE000C94DB14FA0102C00E94E9A69F0100E01C
:1029BE0010E00217130710F00C94EE140E94A1A65B
:1029CE00A0EFBAE00E94A8A60F5F1F4FF2CF0E94A1
:1029DE00AEA6A436E0E0BE0710F00C94FA140E94E6
:1029EE00E9A60E94B3A60E94B3B928960895A091B5
:1029FE00590BA53010F40C940915E0E0E093590B37
:102A0E00E1E00895E0E0089508950E94EEA600E04A
:102A1E0010E02F81388540E050E00E945026E030D3
:102A2E0011F00C9421154436E0E05E0710F00C9482
:102A3E00211501C007C0A1E0B0E00E9415BD4F5F97
:102A4E005F4FEBCFF8010F5F1F4FA985BA85AE0F11
:102A5E00BF1FEC91EE83AE810E941C140217130768
:102A6E0010F00C943B15D7CF0E94B3B92B96089556
:102A7E000E9444BB0E94ADB900E010E020E030E0BF
:102A8E000E945026E03011F00C9454152436E0E0EC
:102A9E003E0710F00C94541501C007C0A1E0B0E041
:102AAE000E9415BD2F5F3F4FEBCFF8010F5F1F4FF9
:102ABE000E94C9A50E94F4A66BBF4691413010F446
:102ACE000C946C15A42F0E941C14003DE7E01E0709
:102ADE0010F00C947715413010F40C94771501C05A
:102AEE0001C0CCCF78940E94B4B9299608950E9463
:102AFE0061A6E093D000E0E0E093D100E093D20035
:102B0E00E093D500E4EFF1E0E093510DF093520D18
:102B1E00A091510DB091520D139710F00C949D157C
:102B2E00E3E0F0E0E093510DF093520DA32F0E94DD
:102B3E00C511E093D400E22FE13011F00C94AD15E5
:102B4E00E091D200E260E093D20022C0E23011F0B8
:102B5E000C94B715E091D200E460E093D20018C057
:102B6E00E33011F00C94C115E091D200E660E093D1
:102B7E00D2000EC0E43011F00C94CF15E091D200CB
:102B8E00E660E093D200E091D100E460E093D100E2
:102B9E00E12FE13011F00C94D915E091D200E860EC
:102BAE00E093D200E02FE13011F00C94E415E091A7
:102BBE00D200E062E093D20009C0E23011F00C9432
:102BCE00ED15E091D200E063E093D200E42FE13006
:102BDE0011F00C94F815E091D100E861E093D1006A
:102BEE0009C0E23011F00C940116E091D100E869B1
:102BFE00E093D1000E94B4B929960895E0E0E093E5
:102C0E00D10008950A930A2FE091D000E07211F0DE
:102C1E000C941216F9CF0093D600099108950E94D4
:102C2E00D9A5E091510DF091520D0E171F0710F01E
:102C3E000C942816AAE5BBE00E946FA60F5F1F4FEB
:102C4E00F0CFE0E0E0934E0DE0934F0DE093500D8A
:102C5E00E1E0E093530D0991199108950E9474A635
:102C6E000A93A091530DA13010F40C944116E2E09A
:102C7E00E093530DE091510DF091520D0E94F9A683
:102C8E00AE17BF0710F00C945816AEE4BDE00E94CC
:102C9E007FA53197E65AF44FDF01E091D600EC9311
:102CAE0002C00091D600E091D000EC710E2FE091A1
:102CBE00500DE03011F00C9466160093500D0991F2
:102CCE000E9495A618950E94FEA608950E94ACB982
:102CDE00AD010E94F9A64A175B0710F00C94791605
:102CEE00FA0102C00E94FEA69F0100E010E002174A
:102CFE00130710F00C948C160E94A1A6AAE5BBE057
:102D0E000E94A8A60F5F1F4FF2CF0E94F9A6A43F04
:102D1E00E1E0BE0710F00C9498160E94FEA60E94E9
:102D2E00B3A60E94B3B928960895A091530DA4306E
:102D3E0010F40C94A716E0E0E093530DE1E0089533
:102D4E00E0E0089508950E94BAA60E94C1A610F46C
:102D5E000C94B416A22F0E940916003DE7E01E0740
:102D6E0010F00C94BF16213010F40C94BF1601C055
:102D7E0001C0EBCF0E94B4B9259608950E9467A5B5
:102D8E0000E010E02D813E81F8010F5F1F4F0E9481
:102D9E0003A74C91A42F0E9409160217130710F0D7
:102DAE000C94DA16F1CF0E94B4B9299608950E94B8
:102DBE0061A6E0933001E0E0E0933101E09332014F
:102DCE00E0933501E4E6F0E0E093BB0DF093BC0D2B
:102DDE00A091BB0DB091BC0D139710F00C94FD1685
:102DEE00E3E0F0E0E093BB0DF093BC0DA32F0E9447
:102DFE00C511E0933401E22FE13011F00C940D1760
:102E0E00E0913201E260E093320122C0E23011F033
:102E1E000C941717E0913201E460E093320118C070
:102E2E00E33011F00C942117E0913201E660E0934B
:102E3E0032010EC0E43011F00C942F17E0913201E4
:102E4E00E660E0933201E0913101E460E0933101FC
:102E5E00E12FE13011F00C943917E0913201E86066
:102E6E00E0933201E02FE13011F00C944417E09121
:102E7E003201E062E093320109C0E23011F00C94AD
:102E8E004D17E0913201E063E0933201E42FE1301F
:102E9E0011F00C945817E0913101E861E093310183
:102EAE0009C0E23011F00C946117E0913101E8692C
:102EBE00E093310181E38A95F1F70E94B4B9299626
:102ECE000895E0E0E093310108950E94D9A50E9493
:102EDE0008A70E171F0710F00C947C17A4E5BDE091
:102EEE000E946FA60F5F1F4FF2CFE0E0E093B80D88
:102EFE00E093B90DE093BA0DE1E0E093BD0D0991B9
:102F0E00199108950A930A2F003011F40C94951715
:102F1E00E0913101E160E093310105C0E0913101B2
:102F2E00EE7FE0933101099108950A930A2FE09103
:102F3E003001E07211F00C94A517F9CF0093360111
:102F4E00099108950E9433A50E94AEB9A091BD0DBE
:102F5E00A13010F40C94B617E2E0E093BD0DE091B1
:102F6E003101E47011F40C94F3170E9408A7329704
:102F7E000E940DA710F00C94DE17E0913101E27063
:102F8E0011F40C94D2170E9414A73197EC5AF24FF9
:102F9E00A1E0A08307C00E9414A73197EC5AF24F0C
:102FAE00A0E0A0830E9414A70E9417A702C0009160
:102FBE003601E091B80DE2501E2FF0E0EC5AF24FC0
:102FCE000E948DA6EC5AF24FE081F0E02E2B3F2BA3
:102FDE00D9010E942D381BC00E9408A70E940DA780
:102FEE0010F00C9400180E941FA710F00C940018FB
:102FFE0001C005C00E9414A70E9417A702C000912D
:10300E0036010E941FA710F40C940E1800E0E091F8
:10301E003001EC710E2FE091BA0DE03011F00C94EE
:10302E001A180093BA0D0E94B5B924960E9445A5B0
:10303E001895BA93AA932997E0E0ED83EE830E9448
:10304E00ACB90B8D1C8D00FF02C0E1E0EC8704369D
:10305E00E0E01E0710F00C943F18E1E0EB87E4E689
:10306E00F0E0E01BF10BAF01F695E7959F0108C06C
:10307E00E0E0EB8704561040F801F695E7959F01C6
:10308E002436E0E03E0710F40C946818E3E0EA877B
:10309E00D901E4E6F0E00E94ACBAAF014987D9014C
:1030AE000E9424A7ED87FE87AD85BE850E9429A7C5
:1030BE00AD85BE85EAE0F0E00E94F0BAAF014F8325
:1030CE001DC02A30E0E03E0710F40C947F18E2E0B9
:1030DE00EA87E0E0E987D9010E9429A7D901EAE051
:1030EE00F0E00E94F0BAED87FE87ED85EF8306C013
:1030FE00E1E0EA87E0E0E987E8872F83E985E05D94
:10310E00E9870E9430A7A985A03311F00C94971877
:10311E00E0E2E987A885A03311F00C949718E887B0
:10312E00EC85E03011F40C949F18E5E3EE8302C0B9
:10313E00E0E3EE83EA85A98DBA8DEC93E985AF893C
:10314E00B88DEC93E885AD89BE89EC93EF81AB89A0
:10315E00BC89EC93EB85A989BA89EC93EE81AF8596
:10316E00B889EC930E94B3B96D960895BA93AA9359
:10317E0060970E94ACB9EB8DE987E98DE887EA8DFF
:10318E00EF83E88DEE83EC8DFD8DFA93EA93EDB728
:10319E00FEB7FA93EA932F93EDB7FEB7FA93EA933D
:1031AE003F93EDB7FEB7FA93EA934F93EDB7FEB7A1
:1031BE00FA93EA935F93FE017596FA93EA93DE0112
:1031CE0056960E9420185F914F913F912F9100E0EB
:1031DE000A3010F00C94F9180E9437A7E0E0EC9337
:1031EE000F5FF6CF00E0E985E03011F40C9405197D
:1031FE00EB85E03011F40C94051901C006C00E9455
:10320E003EA7AE0FBF1FEDE2EC93E885E03011F460
:10321E000C9421190E943EA7EA0FFB1F30830E94D7
:10322E003EA7EA0FFB1F40830E943EA7EA0FFB1F3B
:10323E00508317C0233010F40C942A190E943EA715
:10324E00EA0FFB1F3083223010F40C9433190E94C6
:10325E003EA7EA0FFB1F40830E943EA7EA0FFB1F0B
:10326E005083EF81E03011F40C9451190E943EA767
:10327E000E9444A7EA85E03011F40C944D190E9487
:10328E003EA7AE0FBF1FE5E3EC9304C00E943EA71E
:10329E000E9449A7EE81E03011F40C9462190E944D
:1032AE003EA7AE0FBF1FE8EFEC930E943EA7AE0FF6
:1032BE00BF1FE3E4EC9300E00E9437A71C91E02FC0
:1032CE00AE89BF89F0E0EA0FFB1F10830F5F0A3053
:1032DE0010F00C947719113010F40C94771901C07A
:1032EE0001C0EACF0E94B3B96E9608950E94C9A696
:1032FE000217130714F00C949E190E944EA7F801A2
:10330E00E40FF51FE081EA1711F40C949719F801F8
:10331E00E40FF51FA081AF3311F40C94971901C07F
:10332E0003C00E9455A708950F5F1F4FE1CFE1E044
:10333E000E94B3B92A9608950E945AA70030E0EF72
:10334E001E0710F00C94BB19F801E20FF31FE08179
:10335E00E03011F00C94B819F8010E94B5B924961A
:10336E0008950F5F1F4FEACFE0E0F0E00E94B5B97D
:10337E0024960895BA93AA93EF97EF97EF972F9706
:10338E000E94ACB9DE01AC52BF4F0D90BC91A02D86
:10339E000E94A3199F01DE01AE52BF4F0D90BC914A
:1033AE00A02D0E94A319AF012436E0E03E0714F0D1
:1033BE000C94F119FE01EC52FF4F0190F081E02DBB
:1033CE00FA93EA93FE01E459FF4FFA93EA93D90177
:1033DE000E94961A4436E0E05E0714F00C94021A2E
:1033EE00FE01EE52FF4F0190F081E02D0E9460A78A
:1033FE00DA010E94961A00E010E0E0E00E9467A752
:10340E00DE01A659BF4FA00FB11FAC91EE81EA1796
:10341E0011F00C944E1AE1E00E9467A7D801A40F98
:10342E00B51F2A173B0714F00C94201A0E946CA7A4
:10343E000895E0E0DE01A053BF4FED93EC930E94A0
:10344E0074A7A417B50714F00C944E1AF8010E9435
:10345E0074A7EA0FFB1FDE01A659BF4FAE0FBF1FA9
:10346E001C90FE01E053FF4F0190F081E02D0E9471
:10347E007BA7EC91E11511F40C94481AE0E00E9440
:10348E0067A7DE01A053BF4F0E947FA5D8CFFE01D4
:10349E00E153FF4FE081E03011F40C94671AE02FF6
:1034AE00DE01A053BF4FAC91EA0FDE01A253BF4F16
:1034BE00EC930E94B3B9EF96EF96EF966996089546
:1034CE00F80131968F01E217F30714F00C94701A7D
:1034DE0094CF0E946CA708950E9444BB0E94D9A568
:1034EE000030E0EF1E0710F00C94901AF8010E94C5
:1034FE0080A70E94F4A66BBFE691E03011F00C9409
:10350E008D1AF80119810881269608950F5F1F4FB5
:10351E00E7CFE0E0F0E019810881269608950E9439
:10352E00C9A6022E032A11F00C94AB1A0E944EA7C4
:10353E00A13010F40C94A81A0E9485A70F5F1F4F9C
:10354E00F5CF0E9492A70EC000E010E002171307FD
:10355E0010F00C94B71A0E9485A70F5F1F4FF6CF7D
:10356E000E9492A70E94B3B92A9608950E94C9A6F6
:10357E00022E032A11F00C94D21A0E9498A7E13061
:10358E0010F40C94CF1A0E94A0A70E94A5A7F5CF05
:10359E000E9492A710C000E010E00217130710F06F
:1035AE000C94E01A0E94A0A7D001EC930F5F1F4F5E
:1035BE00F4CF0E9492A70E94B3B92A9608950E9452
:1035CE00C9A6022E032A11F00C94FB1A0E944EA7D4
:1035DE00A13010F40C94F81A0E94AAA70F5F1F4F87
:1035EE00F5CF0E94B8A70EC000E010E00217130737
:1035FE0010F00C94071B0E94AAA70F5F1F4FF6CF67
:10360E000E94B8A70E94B3B92A9608950E9473A586
:10361E00488559852C853D8500E010E0021713077B
:10362E0010F00C942C1BFA01E00FF11FEE83FF83B8
:10363E00AA85BB85EA0FFB1F0F01F801AE85BF857A
:10364E000E94BFA70F5F1F4FE9CF0E94B3B96096CC
:10365E0008950E9473A50E851F852A853B85488592
:10366E005985E0E0EE83EF83AE81BF81A417B507E5
:10367E0010F00C94561BEE81FF81E20FF31FAC8508
:10368E00BD85EA0FFB1F0F01EE81FF81E00FF11FD9
:10369E00A889B9890E94BFA70E9438A6E5CF0E94CB
:1036AE00B3B9629608950E94C9A6002402160306B5
:1036BE0010F00C94641B215030400E94C5A76BBFC4
:1036CE00A691A13010F40C94731B0034E0E01E0799
:1036DE0010F00C94731B01C00BC0F901E00FF11F29
:1036EE00E40FF51F0F010E94C5A70E94CBA7E5CFDF
:1036FE000E94B3B92C9608950E94CEA700E010E068
:10370E0000E010E00217130710F00C94951BF8015F
:10371E000E94D3A740830F5F1F4FF4CF0E94B4B90E
:10372E00289608950E945AA70E94D8A76BBFA6910B
:10373E00A13010F40C94A81B0E94DEA70E94CBA708
:10374E00F3CFF801E20FF31FA0E0A0830E94B5B9FA
:10375E00289608950E945AA70E94D8A76BBFA691DB
:10376E00A13010F40C94C01B0E94DEA70E94CBA7C0
:10377E00F3CF0E94B5B928960895BA93AA932797C6
:10378E000E94ADB930E040E000E0073010F00C943C
:10379E00DA1BAC85BD850E94E3A70E94EAA7E0E094
:1037AE00EC930F5FF2CF1E852F8500E0012E022ACB
:1037BE0011F00C94E61B0E94EFA70E9449A722234A
:1037CE0012F00C94F81B0E94EFA7AE0FBF1FEDE294
:1037DE00EC93E12FF22FAFEFBFEF0E9494BA1E2FA2
:1037EE002F2F00240116020614F00C94161CE32F42
:1037FE00F42F3F5F4F4F0E94F5A7BF01A12FB22FAD
:10380E00EAE0F0E00E94F3BADB01EC93A12FB22FB5
:10381E00EAE0F0E00E94BFBA1E2F2F2FE2CF002465
:10382E000316040614F00C942B1C0E94EFA7EA0F4B
:10383E00FB1F0F01E32FF42F31973E2F4F2F0E94C6
:10384E00EAA70E94FAA7EBCF0E94B4B9609608953A
:10385E000E94FFA70C3010F00C943F1CA32FB42F26
:10386E000E94E3A70E9408A8E0E0EC930F5FF2CF5E
:10387E000E940DA811F00C94481C0E9419A8A0E3F8
:10388E00A083A885AA2312F00C945B1C0E9419A891
:10389E00ADE2A0830E94D1A5AFEFBFEF8FEF9FEFF8
:1038AE000E9499BA0E94BFA50E94C9A50E9489BB19
:1038BE0014F00C94741C0E941FA8FF93EF930E94A7
:1038CE0028A80E9405BBAF91BF91EC930E9428A837
:1038DE000E94E8BA0E94BFA5E7CF00240116020697
:1038EE0014F00C94811C0E9419A80E942FA80E940B
:1038FE00FAA7F3CF0E94B4B9699608950E94FFA764
:10390E000C3010F00C94951CA32FB42F0E94E3A73B
:10391E000E9408A8E0E0EC930F5FF2CF0E940DA882
:10392E0011F00C949E1C0E9419A8A0E3A0830E9483
:10393E00C9A50E9489BB10F00C94B51C0E941FA84B
:10394E00FF93EF930E9428A80E9401BBAF91BF91F5
:10395E00EC930E9428A80E94CEA5E9CF0024011660
:10396E00020614F00C94C21C0E9419A80E942FA8E3
:10397E000E94FAA7F3CF0E94B4B969960895AA934C
:10398E00A5970E94ACB9E9A9FAA96BA97CA90E94D6
:10399E0036A8ECA5E88B1DA51B3010F40C94D81C92
:1039AE001AE0E889E03011F00C94DE1C10E0A889D2
:1039BE00A03210F40C94E81CA03810F00C94E81C03
:1039CE0002C0EEE2E88B0EA50D3010F40C94F01C44
:1039DE000CE0E0E0EE87EF87AE85BF851D9714F013
:1039EE000C94061D0E943BA80E9449A7EE85FF85F8
:1039FE00DE015E960E9449A70E9440A8EDCF0E946C
:103A0E0046A8DE0155960E94851CDE0151960E9445
:103A1E00A319EA87FB87AA85BB851B9714F40C9420
:103A2E001C1DEAE0F0E0EA87FB87EA85FB8530970C
:103A3E0011F00C94281DE0E3E98BE1E0F0E0EA8759
:103A4E00FB8750E0113010F40C94B61DEA85FB850F
:103A5E00A12FB0E0AE17BF0714F40C94831DE0E362
:103A6E00EE8FE889EF8FE2E0F0E0EE87FF875E5F92
:103A7E00AA85E12FEA1B2E2F520F213010F40C9441
:103A8E00511D0E9440A83197DE015E960E9449A703
:103A9E002150F3CFE0E0EC87ED87AE85BF851C9714
:103AAE0014F00C946B1D0E9440A831970E944DA8F3
:103ABE000F01EC85FD853196EC87FD873197DE0190
:103ACE0051960E94BFA7E9CFE0E0EE87EF87AE8563
:103ADE00BF851C9714F00C94821D0E943BA8EA0F20
:103AEE00FB1F0F01EE85FF85DE015E960E94BFA7CC
:103AFE000E9440A8ECCF2BC0EA85E11B2E2FEBE0F5
:103B0E00F0E0EE87FF87E22FAE85BF85F0E0EA1783
:103B1E00FB0714F00C94A51D0E943BA8EA0FFB1F97
:103B2E000F01EE85FF853197DE0151960E94BFA7EA
:103B3E00EE85FF853197EE87FF87E5CFE22FF0E028
:103B4E00DE015196EA0FFB1FA889A0835F5FE52F68
:103B5E00AA85BB85F0E0EA0FFB1FEA87FB87EBA582
:103B6E00E03011F40C94BD1D40E301C040E2EA8543
:103B7E00FB85A02FB0E0EA17FB0714F00C94FD1D97
:103B8E00AA85E02FEA1B3E2FEBE0F0E0EE87FF87E1
:103B9E000E943BA8EA0FFB1FBF010E9452A80E9481
:103BAE0049BBEA1BFB0BDE0151960E9457A8EE851E
:103BBE00FF853197EE87FF870E9452A8AE17BF0789
:103BCE0014F40C94EB1DE4CFE0E0EE87EF870E9437
:103BDE0052A8AE17BF0714F00C94FD1D0E943BA80F
:103BEE00EA0FFB1F40830E9440A8F1CFE0E0EE8772
:103BFE00EF87AE85BF851C9714F00C94141EEE85CE
:103C0E00FF85AFA5B8A9EA0FFB1F0F010E943BA8C5
:103C1E000E94BFA70E9440A8ECCF0E94B3B9E596C0
:103C2E0008950E94EEA63D854C855B85383110F4D3
:103C3E000C94221E30E04C3310F40C94271E40E0FE
:103C4E005C3310F40C942C1E50E0E985EE8310E0EA
:103C5E0020E01C30E0E02E0714F00C943F1EE12F04
:103C6E00F22F0E9403A7E0E0EC931F5F2F4FF1CFDE
:103C7E000A85003011F40C946C1E303011F40C9443
:103C8E004D1E3C3011F40C944D1E08C0AF81B8850A
:103C9E00E1E3EC931196E2E3EC9316C03C3010F0A6
:103CAE000C945C1E0E945DA80FC0A32FAC500E9406
:103CBE006FA8AF81B885EC93A32FAC500E9474A867
:103CCE00AF81B8851196EC9302C00E945DA8AF81BA
:103CDE00B8851296EAE3EC93A42F0E946FA8AF81E9
:103CEE00B8851396EC93A42F0E9474A8AF81B88563
:103CFE001496EC9315E020E0EE81E03011F40C9474
:103D0E009E1E0E9479A80E9403A7EAE3EC930E94EC
:103D1E0079A80E947EA80E946FA8DB01EC930E94F6
:103D2E0079A80E947EA80E9474A8DB01EC93003053
:103D3E0011F40C94BF1E0E9479A80E9403A7E0E222
:103D4E00EC933C3010F00C94B31E0E9479A80E94A4
:103D5E0003A7E1E4EC9306C00E9479A80E9403A792
:103D6E00E0E5EC930E9479A80E9403A7EDE4EC93A2
:103D7E00E1E00E94B3B92E960895BA93AA932697BE
:103D8E000E94ACB9E989EF70E05DE987E989E07FCF
:103D9E00E295EF70E05DEA870B891A8928891D305C
:103DAE0010F00C94DF1E103011F40C94DF1E01C0C5
:103DBE0011E0003210F00C94E91E003011F40C9456
:103DCE00E91E01C001E0233310F00C94F31E2B30DA
:103DDE0010F40C94F31E01C021E0EE85E03011F0DA
:103DEE000C94FC1EEEE2EE830FC0AE85A13011F0F6
:103DFE000C94041FEFE2EE8307C0AE85A03210F4E0
:103E0E000C940B1FEE85EE83A02FEAE00E949EBA63
:103E1E003E2FA02FEAE00E94EDBA4E2FA12FEAE02E
:103E2E000E949EBA5E2FA12FEAE00E94EDBAEB87A8
:103E3E000E9485A8E8870E948AA8EF83305D405DC6
:103E4E00505DEB85E05DEB870E9430A7EF85E0309B
:103E5E0011F00C943D1F0E948FA8EC85FD855383B5
:103E6E00EB850E949BA80E94A0A84DC0E13011F0E6
:103E7E000C944A1F0E94BAA8EC85FD8533834483B7
:103E8E000E94A0A840C0E23011F00C945B1F0E946B
:103E9E00C8A8EC85FD855583EB850E94DDA830878B
:103EAE00EC85FD8541872FC0E33011F00C94681F1F
:103EBE000E948FA80E94E9A80E94F0A80E94F7A86D
:103ECE0022C0E43011F00C94771F0E94BAA80E9411
:103EDE00E9A80E94F0A83087EC85FD85418713C0C4
:103EEE00E53011F00C948A1F0E94C8A8EC85FD8560
:103EFE0035834683EE81AC85BD851796EC93EC85B4
:103F0E00FD850E94F7A8AC85BD851A96E0E0EC937E
:103F1E000E94B3B9649608950E9473A5A885B985C9
:103F2E000E94A3190E94FEA8A030E1E0BE0710F483
:103F3E000C94A51FEFEFF0E0EE83FF830E9403A920
:103F4E000E94731A5E2F00E010E00E9408A910F084
:103F5E000C94F81F0E944EA70E940DA96BBFE6910C
:103F6E00EA1711F00C94F51FE52FF0E0E00FF11FAA
:103F7E00DF01EE81FF81EA17FB0710F00C94CC1FD6
:103F8E00E0E00E94B3B92E96089520E030E040E0C4
:103F9E00451710F00C94E91FE42FF0E0E00FF11F2D
:103FAE00A885B985AE0FBF1F0C90E42F0E9403A900
:103FBE000E9412A9E01511F40C94E71F21E030E0E5
:103FCE004F5FE6CF022E032A11F00C94F51FE02F5F
:103FDE00E40F5E2F0E94B3B92E9608950F5F1F4F08
:103FEE00B4CFE0E00E94B3B92E9608950E94AFB907
:103FFE002A2F022F02950F700F70AAE00A9F002D34
:10400E00E22FEF701E2F010F0E9462A508950E94ED
:10401E00AEB93A2F032FA02FEAE00E949EBA1E2FB0
:10402E001295107FA02FEAE00E94EDBA2E2F120FEC
:10403E00E12F0E94B5B9249608950A930A2F0033F2
:10404E0010F40C942F200A3310F00C942F2001C082
:10405E0003C0E1E009910895E0E009910895099106
:10406E0008950A930A2F0E942420E03011F40C9434
:10407E004420E02FE05309910895E0E0099108955E
:10408E00099108950E94ACB94A2F5E81F52FE0E0A8
:10409E008F010070E42FF0E0F0709F01022B132BC4
:1040AE00F8010E94B3B92796089528970E94AEB9D9
:1040BE000A2F1C852D853E85E32F0E941AA90E948A
:1040CE0022A90E9427A90E942CA9E22F0E941AA9B8
:1040DE000E9430A9E12F0E941AA90E9430A9E02F58
:1040EE000E941AA9EC83FD836E837F830E9427A909
:1040FE000E94D2B90E9422A9E885F9856A857B853E
:10410E000E94B5B92F9608950E94AEB92A2F3C8110
:10411E00E22FE0531E2FE32FE0530E2FAAE00A9F4B
:10412E00002D010FE02F0E94B5B925960895BA9380
:10413E00AA932B970E94ACB9A989BA890E94A31998
:10414E001E2FE989FA890E943DA9A6E0B0E00E94DF
:10415E00961A10E0E0E0E88B0E9444A9A03310F418
:10416E000C94C0200E9444A9AA3310F00C94C020D5
:10417E0002C0E1E0E88BE889E03011F00C94C82031
:10418E001F5F153010F00C94D220A889A03011F0CA
:10419E000C94D22001C001C0DFCF163010F00C9469
:1041AE00DD20103011F40C94DD2004C00E948BA58C
:1041BE0063960895153011F00C94F920E989FA8967
:1041CE00E481E88BA989BA8913965C91A989BA8989
:1041DE0012964C91A989BA8911963C91A989BA89EE
:1041EE002C9147C0143011F00C940E21E989FA89F4
:1041FE00E381E88BA989BA8912965C91A989BA895B
:10420E0011964C91A989BA893C9120E332C01330A2
:10421E0011F00C942021E989FA89E281E88BA989B1
:10422E00BA8911965C91A989BA894C9130E320E341
:10423E0020C0123011F00C942F21E989FA89E18106
:10424E00E88BA989BA895C9140E330E320E311C081
:10425E00113011F00C943C21A989BA89EC91E88BAC
:10426E0050E340E330E320E304C00E948BA5639645
:10427E000895E22FE0530E2F0A3010F40C944821CB
:10428E0000E00E944BA9A0E1B7E20E9450A9EE8384
:10429E00FF83E32FE0530E2F0A3010F40C945821B5
:1042AE0000E00E944BA9A8EEB3E00E9450A90E9424
:1042BE00D3A7EE83FF83E42FE0530E2F0A3010F4C2
:1042CE000C946A2100E00E9455A9E4E60E945CA9C4
:1042DE00EE83FF83E52FE0530E2F0A3010F40C947B
:1042EE00792100E00E9455A9EAE00E945CA9EE83C4
:1042FE00FF83E889E0530E2F0A3010F40C948821C6
:10430E0000E00E944BA90E94D3A7EE83FF830E9478
:10431E00B3B963960895BA93AA932A970E94ACB93B
:10432E005A890B891C8930E0E52FE1502E2F283059
:10433E0010F40C94A32127E0422FE22F2150F0E03D
:10434E000E947BA7E02FEF70EC93F8010E9438BA21
:10435E008F013F5F341710F00C94B621EECFE22F91
:10436E000E9461A900834F5FE42FF0E00E947BA7BB
:10437E00E0E0EC9330E00E9467A9AC91AA3010F413
:10438E000C94CE210E9467A9EC91E95FEC93E32F88
:10439E00A889B9890E946AA90E9467A90E94FAA7F2
:1043AE003F5F341710F00C94DD21E5CFA889B98951
:1043BE00EE27A30FBE1FEC930E94B3B96596089526
:1043CE000E946FA90217130710F00C94F021F80148
:1043DE0001C0F9010E94B5B9269608950E9475A9EB
:1043EE00123011F00C940B22E02FE37011F40C94A8
:1043FE000522ECE11981088123960895EDE11981DA
:10440E0008812396089527C0113011F40C942822A8
:10441E00133011F40C942822153011F40C94282228
:10442E00173011F40C942822183011F40C94282211
:10443E001A3011F40C9428221C3011F40C942822FA
:10444E0005C0EFE11981088123960895EEE11981E7
:10445E000881239608951981088123960895AA93B9
:10446E0021970E947AA9498528853F81203011F431
:10447E000C9452222D3010F00C945222303011F444
:10448E000C945222303210F00C945222443610F01A
:10449E000C94522204C00E948BA52A96089551E0D6
:1044AE00223010F40C9466225A93A42F0E94F52108
:1044BE00EE83F0E00E0F1F1F21505F5FF1CFE32F51
:1044CE000E947FA90E94B3B92A9608950A930A2FD3
:1044DE00E02FE37011F00C947722E1E0099108953A
:1044EE00E0E009910895AA931A930A930A81102F76
:1044FE00E02FEC5F1E1710F00C949122E12FE37069
:10450E0011F00C948F22E12F1981088123960895C2
:10451E001F5FEECF1981088123960895AA931A93EF
:10452E000A930A81043010F00C94A222E0E0198163
:10453E00088123960895E02FE37011F00C94AC22BD
:10454E00E02F19810881239608950450102FE02F33
:10455E00EC5F1E1710F00C94C022E12FE37011F0E7
:10456E000C94BE22E12F19810881239608951F5FB6
:10457E00EECF1981088123960895AA931A930A9370
:10458E001B81EB81E1500E2FA8E10A9F002DEA81DD
:10459E000E0FE02F19810881249608950E94DEA542
:1045AE004A93A32F0E94C4220E2F11270E9484A982
:1045BE000E94B4B9279608950E94AEB92A2F3C8165
:1045CE00E32FE1500E2F11270E948CA90E94B5B93E
:1045DE00259608950E94DEA54A93A32F0E94E322FA
:1045EE008F010E9484A90E94B4B9279608950E9453
:1045FE00ACB92A2F3E814F8158855A934A93A32FE7
:10460E000E9436228F01015010400E948CA90E94F8
:10461E00B3B92996089524970E94ADB90A2F19852A
:10462E002A853B854C854A933A932A93A12F0E9463
:10463E00FE22662777270E94D6A5319760407040EC
:10464E000E94D6A50E9494A90E94BFA50E949BA974
:10465E000E94D6A50E94B4B92D960895AA930E94E1
:10466E00AEB92D813E810D811E81EC81E03011F4B9
:10467E000C944823012F1127E02F0E94B5B92796DD
:10468E000895E02F0E94B5B9279608950E94B5B9F6
:10469E0027960895AA9324970E94D1A50E94A4A9B3
:1046AE00EC81E03011F00C945F23E8812996089597
:1046BE000E94A7A9A13011F00C946823E8812996D5
:1046CE0008950E94A7A9A23011F00C947123E881DD
:1046DE00299608950E9435BBE8E00E9418BA0E9400
:1046EE00A4A9E881299608950E94ADB92A2F3D818B
:1046FE004E8111E000E0021710F00C949223A32FCC
:10470E00B42F0E94B0A9E03011F00C94902313E660
:10471E0002C00F5FF0CF113011F00C949B23E12FEC
:10472E000E94B4B92796089510E000E0021710F029
:10473E000C94AF23A32FB42FEE27A00FBE1FAC9166
:10474E00A13010F40C94AD2313E602C00F5FEECF30
:10475E00E12F0E94B4B9279608950E94AFB91A2F7F
:10476E002B81A22F0E942420E03011F00C94C42340
:10477E00EFEF0E94B6B924960895A12F0E9424202F
:10478E00E03011F40C94D723A22F0E9438200E2F64
:10479E00AAE00A9F002DA12F0E9438200E0F04C000
:1047AE00A22F0E9438200E2FE02F0E94B6B9249619
:1047BE000895AA930E94ADB93D81AE81BF810E943A
:1047CE00A3192E2FE31B1E2F112311F00C94F4238B
:1047DE00E1E00E94B4B92896089500E0011710F0A8
:1047EE000C940F24E32FE00F4E2F421710F00C9471
:1047FE000D24E02FAE81BF810E946AA9AE81BF81D8
:10480E00EE27A40FBE1FEC91D001EC930F5FE6CF05
:10481E00012F021710F00C941D24AE81BF81EE27DC
:10482E00A00FBE1FE0E2EC930F5FF3CFE0E00E941B
:10483E00B4B92896089524970E94B5A92AE010E0ED
:10484E001A3010F00C943924A32FB42FEE27A10F99
:10485E00BE1F0E94BAA911F00C943724212F02C05A
:10486E001F5FEECF213010F40C9442242B3010F049
:10487E000C94422404C00E94BFA92996089510E00A
:10488E00E0E0ED83EE83EF83E8870E94D1A5AAE0F6
:10489E00B0E080E090E00E946EBA0E94BFA5E12FCA
:1048AE001F5FF0E0E30FF41FA0810E9438200E2F4F
:1048BE000E949BA90E94BFA5121710F00C946824A9
:1048CE00E4CF0E94D1A50E94B4B9299608950E9402
:1048DE00AEB98D012C813D811A930A930E94C6A90F
:1048EE00E32FE13011F00C949224213011F00C944E
:1048FE008724E6EFF0E060E070E00E94CCA90AC0E9
:10490E00223011F00C949124EDEFF0E060E070E0B5
:10491E000E94CCA99BC0E23011F00C94AC24213043
:10492E0011F00C94A124E4E0F1E060E070E00E944C
:10493E00CCA90AC0223011F00C94AB24EDE0F1E0CA
:10494E0060E070E00E94CCA981C0E33011F00C94BD
:10495E00C624213011F00C94BB24E5E1F1E060E0B7
:10496E0070E00E94CCA90AC0223011F00C94C5242C
:10497E00EEE1F1E060E070E00E94CCA967C0E430A7
:10498E0011F00C94E024213011F00C94D524E8E2BF
:10499E00F1E060E070E00E94CCA90AC0223011F074
:1049AE000C94DF24E3E3F1E060E070E00E94CCA918
:1049BE004DC0E53011F00C94FA24213011F00C9416
:1049CE00EF24ECE3F1E060E070E00E94CCA90AC0B5
:1049DE00223011F00C94F924E4E4F1E060E070E090
:1049EE000E94CCA933C0E63011F00C94142521306E
:1049FE0011F00C940925EBE4F1E060E070E00E9408
:104A0E00CCA90AC0223011F00C941325E3E5F1E095
:104A1E0060E070E00E94CCA919C0E73011F00C9450
:104A2E002D25213011F00C942325ECE5F1E060E00A
:104A3E0070E00E94CCA90AC0223011F00C942D25F2
:104A4E00E4E6F1E060E070E00E94CCA90E94B5B906
:104A5E0026960895759A749A769A779AE09104013B
:104A6E00E068E09304015D9A559A5D985F9A579AB3
:104A7E005F980895E0E00895E0E0E1B9E2B9E4B9A5
:104A8E00E5B9E7B9E8B9EAB9EBB9EDB9EEB9E0BB0A
:104A9E00E1BBE3BBE4BBE0930101E0930201E4E17F
:104AAE00E0930401E0930501E0E0E0930701E09359
:104ABE000801E0930A01E0930B0108950A930A2F6F
:104ACE0000FF03C05D9A559A01C05D980991089543
:104ADE000A930A2F00FF03C05F9A579A01C05F988E
:104AEE00099108950A930A2F6B9A003011F40C94D1
:104AFE008225739A01C0739809910895639B02C031
:104B0E00E1E00895E0E008950E94D1A9E860E09305
:104B1E000101003011F40C949A25E0910201E86035
:104B2E00E093020105C0E0910201E77FE0930201EC
:104B3E00099108956F980E94D6A9679B02C0E0E084
:104B4E000895E1E008951A930A9300E010E0649945
:104B5E0001C011E0A39B01C010E0A49B01C010E0B6
:104B6E00103011F40C94BC250061659901C00062EF
:104B7E00669901C00064679901C00068E02F099131
:104B8E00199108950A930A2F9A9A003011F40C94F1
:104B9E00D225A29A01C0A298099108950A930A2FCC
:104BAE00003011F40C94DF25A0E00E94C92503C04B
:104BBE00A1E00E94C925099108959A9B03C0A29B6A
:104BCE0001C001C002C0E1E00895E0E008956E98D2
:104BDE000E94D6A9669B02C0E0E00895E1E0089528
:104BEE000E94D1A9E061E0930101003011F40C9410
:104BFE000626E0910201E061E093020105C0E0911A
:104C0E000201EF7EE093020109910895E091000107
:104C1E00E07111F40C941526E1E00895E0E008959A
:104C2E000E94DAA9E064E0930A01003011F40C94BA
:104C3E002626E0910B01E064E0930B0105C0E091A4
:104C4E000B01EF7BE0930B0109910895E0910901AF
:104C5E00E07411F40C943526E1E00895E0E0089537
:104C6E000A930A2F0E941814539A003011F40C94D0
:104C7E0042265B9A01C05B98099108950E94181410
:104C8E0052980E94D6A94A9B02C0E1E00895E0E046
:104C9E0008950E94AB2CE03011F00C945826E0E001
:104CAE00089523980E94D6A91B9B02C0E0E00895A8
:104CBE00E1E0089523980E94D6A91B9B02C0E1E073
:104CCE000895E0E008950A930A2F249A003011F413
:104CDE000C9473262C9A01C02C98099108950A936E
:104CEE000A2F229A003011F40C947F262A9A01C0C2
:104CFE002A98099108950E94DAA9E062E0930A01C8
:104D0E00003011F40C949126E0910B01E062E093D7
:104D1E000B0105C0E0910B01EF7DE0930B010991B2
:104D2E000895E0910901E07211F40C94A026E1E0DF
:104D3E000895E0E008950A930A2F0E940516E09167
:104D4E000101E260E0930101003011F40C94B526EC
:104D5E00E0910201E260E093020105C0E0910201E0
:104D6E00ED7FE0930201099108950E940516E091EE
:104D7E000101EE7F0E94DFA9E0910001E17011F4C4
:104D8E000C94CB26E1E00895E0E008950E94D1A9AD
:104D9E00E064E0930101003011F40C94DC26E09104
:104DAE000201E064E093020105C0E0910201EF7B95
:104DBE00E093020109910895E0910101EF7D0E94B7
:104DCE00DFA9E0910001E07211F40C94F026E0E00E
:104DDE000895E1E0089538980E94D6A9309B02C04C
:104DEE00E0E00895E1E008950A930A2F399A003021
:104DFE0011F40C940427419A01C041980991089529
:104E0E00419B02C0E1E00895E0E008953A980E94C7
:104E1E00D6A9329B02C0E1E00895E0E00895E0914A
:104E2E000101EF770E94DFA9E0910001E07811F413
:104E3E000C942327E1E00895E0E008950E941627E0
:104E4E0008950A930A2F0E946817E0910401E26008
:104E5E00E0930401003011F40C943B27E09105011E
:104E6E00E260E093050105C0E0910501ED7FE0935E
:104E7E000501099108950E946817E0910401EE7FE3
:104E8E00E09304010E94D6A9E0910301E17011F4B0
:104E9E000C945327E1E00895E0E008950A930A2F59
:104EAE00279A003011F40C945E272F9A01C02F9888
:104EBE00099108952F9B03C0279B01C001C002C01A
:104ECE00E1E00895E0E008950A930A2F9C9A0030DD
:104EDE0011F40C947427A49A01C0A4980991089512
:104EEE00A49B02C0E0E00895E1E008956C980E9452
:104EFE00D6A9649B02C0E0E00895E1E008950A930C
:104F0E000A2F9B9A003011F40C948F27A39A01C09C
:104F1E00A398099108956D98759A0E94D6A9659BDC
:104F2E0002C0E0E00895E1E008950A930A2F269A60
:104F3E00003011F40C94A5272E9A01C02E980991D9
:104F4E0008952E9B03C0269B01C001C002C0E1E064
:104F5E000895E0E008950A930A2F259A003011F47F
:104F6E000C94BB272D9A01C02D98099108951D9B75
:104F7E0002C0E1E00895E0E008950A930A2F569AE0
:104F8E00003011F00C94CD275E9805C0013011F061
:104F9E000C94D2275E9A099108954E9B02C0E1E0CF
:104FAE000895E0E008950E94DAA9E068E0930A010E
:104FBE00003011F00C94E927E0910B01EF77E093AC
:104FCE000B0109C0013011F00C94F227E0910B0196
:104FDE00E068E0930B0109910895E0910901E078F2
:104FEE0011F40C94FC27E1E00895E0E00895549844
:104FFE000E94D6A94C9B02C0E1E00895E0E008951E
:10500E000A930A2F3B9A003011F40C941028439AFD
:10501E0001C04398099108953C980E94D6A9349BEB
:10502E0002C0E1E00895E0E008950A930A2F0030EF
:10503E0011F00C9425283D9845980DC0013011F0C3
:10504E000C942C283D9A459806C0023011F00C9411
:10505E0032283D98459A099108953D98459A0E94A7
:10506E00D6A9359B02C0E0E00895E1E008950A93C9
:10507E000A2F003011F00C9447283E9846980DC028
:10508E00013011F00C944E283E9A469806C002301C
:10509E0011F00C9454283E98469A099108950A935B
:1050AE000A2F3E9A003011F40C945F28469A01C0E4
:1050BE004698099108953E98469A0E94D6A9369B25
:1050CE0002C0E0E00895E1E008950A930A2F00304F
:1050DE0011F00C9475289898A0980DC0013011F01D
:1050EE000C947C28989AA09806C0023011F00C946B
:1050FE0082289898A09A099108950A930A2F989A4F
:10510E00003011F40C948D28A09A01C0A09809913A
:10511E0008959898A09A0E94D6A9909B02C0E0E0AC
:10512E000895E1E008950A930A2F003011F00C94CF
:10513E00A3289998A1980DC0013011F00C94AA28BB
:10514E00999AA19806C0023011F00C94B028999843
:10515E00A19A099108950A930A2F999A0E94D6A9A5
:10516E00003011F40C94BD28A19A01C0A1980991A8
:10517E0008959998A19A919B02C0E0E00895E1E00C
:10518E0008950A930A2F003011F00C94D1280B9831
:10519E0013980DC0013011F00C94D8280B9A139867
:1051AE0006C0023011F00C94DE280B98139A099168
:1051BE0008950A930A2F0B9A003011F40C94E928E3
:1051CE00139A01C01398099108950B98139A0E948F
:1051DE00D6A9039B02C0E0E00895E1E008950A938A
:1051EE000A2F003011F00C94FF28099811980DC069
:1051FE00013011F00C940629099A119806C002305C
:10520E0011F00C940C290998119A099108950A939A
:10521E000A2F099A003011F40C941729119A01C023
:10522E001198099108950998119A0E94D6A9019B87
:10523E0002C0E0E00895E1E008950E94DAA9E2607C
:10524E00E0930A01003011F40C943329E0910B0124
:10525E00E260E0930B0105C0E0910B01ED7FE0935E
:10526E000B0109910895E0910901E27011F40C947B
:10527E004229E1E00895E0E008950E94DAA9E46091
:10528E00E0930A01013011F00C945329E0910B01C7
:10529E00E460E0930B0105C0E0910B01EB7FE0931E
:1052AE000B0109910895E0910901E47011F40C9439
:1052BE006229E1E00895E0E008953D98459A3D9811
:1052CE00459AE0E008950A930A2F3D98459AE09199
:1052DE000A01E061E0930A01003011F40C947D297B
:1052EE00E0910B01E061E0930B0105C0E0910B0131
:1052FE00EF7EE0930B01099108950E94DAA9E06117
:10530E00E0930A01003011F40C949329E0910B0103
:10531E00E061E0930B0105C0E0910B01EF7EE0939D
:10532E000B01099108950E94DAA9E860E0930A0141
:10533E00003011F40C94A929E0910B01E860E09380
:10534E000B0105C0E0910B01E77FE0930B01099182
:10535E000895E0910901E87011F40C94B829E1E088
:10536E000895E0E0089508950E94DAA9E160E093BF
:10537E000A01013011F00C94CA29E0910B01E16091
:10538E00E0930B0105C0E0910B01EE7FE0930B0162
:10539E0009910895E0910901E17011F40C94D92955
:1053AE00E1E00895E0E008950A930A2F829A839A25
:1053BE00013011F00C94E6298A9A8B9809C00230BC
:1053CE0011F00C94ED298A988B9A02C08A988B98CA
:1053DE00099108950A930A2FA1E00E94332CA02F61
:1053EE000E94DB29099108950A9300E07B9B01C07E
:1053FE0001607A9B01C00260E02F099108950A9323
:10540E000A2F829A003011F40C940F2A8A9A01C046
:10541E008A980991089583988B9A0E94D6A97B9BAE
:10542E0002C0E1E00895E0E008950E94E2A9E09153
:10543E000701E260E0930701013011F00C94302A6D
:10544E00E0910801E1600E94EAA9ED7FE093080176
:10545E0015C0023011F00C943D2AE0910801EE7F48
:10546E000E94EAA9E260E093080108C0E0910801F9
:10547E00EE7F0E94EAA9ED7FE0930801099108955D
:10548E000A9300E0E0910601E27011F40C94502AA8
:10549E000160E0910601E17011F40C94572A02604C
:1054AE00E02F099108950E94E2A9003011F40C94A6
:1054BE00662AE0910801E160E093080105C0E091E1
:1054CE000801EE7FE093080109910895E09107012C
:1054DE00ED7F0E94EFA9E260E0930801E0910601E2
:1054EE00E27011F40C947D2AE1E00895E0E0089555
:1054FE000E94F4A9E064E0930701003011F40C94CB
:10550E008E2AE0910801E064E093080105C0E09165
:10551E000801EF7BE093080109910895E0910801DD
:10552E00E07411F40C949D2AE1E00895E0E00895F2
:10553E00E0910701EF770E94EFA9E0680E94F9A9B8
:10554E00E0910601E07811F40C94AF2AE1E00895A1
:10555E00E0E00895E0910701EB7F0E94EFA90E9421
:10556E00FCA911F40C94BD2AE0E00895E1E0089541
:10557E00E0910701EB7F0E94EFA90E94FCA911F4B4
:10558E000C94CB2AE1E00895E0E00895E091070144
:10559E00E77F0E94EFA9E8600E94F9A9E091060159
:1055AE00E87011F40C94DD2AE1E00895E0E008952E
:1055BE000E94F4A9E860E0930701003011F40C9406
:1055CE00EE2AE0910801E860E093080105C0E09141
:1055DE000801E77FE093080109910895E091070122
:1055EE00EF7E0E94EFA9E0610E94F9A9E091060109
:1055FE00E07111F40C94052BE0E00895E1E00895BC
:10560E000E94F4A9E061E0930701003011F40C94BC
:10561E00162BE0910801E061E093080105C0E091CE
:10562E000801EF7EE093080109910895E0910701CA
:10563E00EF7D0E94EFA9E0620E94F9A9E0910601B8
:10564E00E07211F40C942D2BE1E00895E0E0089542
:10565E000A930C98149A0E94D6A900B104FF03C0B5
:10566E00E1E009910895E0E0099108950A930C98FC
:10567E00149A0E94D6A900B104FF03C0E1E009917B
:10568E000895E0E0099108950A930D98159A0E94E5
:10569E00D6A900B105FF03C0E1E009910895E0E04D
:1056AE00099108950A930A2F0D9A003011F40C9463
:1056BE00622B159A01C01598099108950A932098A6
:1056CE00289A0E94D6A903B100FF03C0E0E0099119
:1056DE000895E1E0099108950A930A2F209A003067
:1056EE0011F40C947C2B289A01C0289809910895E6
:1056FE002198299A0E94D6A9199B02C0E0E008952C
:10570E00E1E008950A930A2F219A003011F40C94C7
:10571E00922B299A01C02998099108950F98179AEA
:10572E000E94D6A9079B02C0E0E00895E1E008952B
:10573E000E9407AAE068E0930401013011F00C9476
:10574E00AE2BE0910501E068E093050105C0E09104
:10575E000501EF77E093050109910895E0910301AA
:10576E00E07811F40C94BD2BE1E00895E0E008958B
:10577E000E9407AAE064E0930401003011F40C9437
:10578E00CE2BE0910501E064E093050105C0E091A8
:10579E000501EF7BE093050109910895E091030166
:1057AE00E07411F40C94DD2BE1E00895E0E008952F
:1057BE000E9407AAE062E0930401003011F40C94F9
:1057CE00EE2BE0910501E062E093050105C0E0914A
:1057DE000501EF7DE093050109910895E091040123
:1057EE00EF7DE0930401E0910501E062E093050195
:1057FE00E0910301E07211F40C94072CE1E008959E
:10580E00E0E00895E0910301E07211F40C94112C84
:10581E00E1E00895E0E008950E9407AAE061E093B8
:10582E000401003011F40C94222CE0910501E0618A
:10583E00E093050105C0E0910501EF7EE0930501BF
:10584E0009910895E0910501E07111F40C94312C49
:10585E00E1E00895E0E008950E9407AAE860E09371
:10586E000401003011F40C94422CE0910501E86023
:10587E00E093050105C0E0910501E77FE093050186
:10588E0009910895E0910301E87011F40C94512CE4
:10589E00E1E00895E0E008950E9407AAE460E09335
:1058AE000401003011F40C94622CE0910501E460C7
:1058BE00E093050105C0E0910501EB7FE093050142
:1058CE0009910895E0910401EB7FE09304010E9499
:1058DE00D6A9E0910301E47011F40C94782CE1E068
:1058EE000895E0E008950A930A2F003011F40C9405
:1058FE00822C479A01C047983F9A09910895479B79
:10590E0002C0E1E00895E0E008953F9847980E94B4
:10591E000CAA379B02C0E1E00895E0E008956A9872
:10592E000E94D6A9629B02C0E1E00895E0E00895CE
:10593E000E94E32608950A930A2F0E947A2C099159
:10594E0008950E94692C08959D980E94D6A9959B52
:10595E0002C0E1E00895E0E00895E0910101EB7FDF
:10596E000E94DFA9E0910001E47011F40C94C12CA7
:10597E00E1E00895E0E008950A98129A0E94D6A9EF
:10598E00029B02C0E1E00895E0E008950A930A2F19
:10599E00089A003011F40C94D92CA1E00E94332CFB
:1059AE00109A01C01098099108950898109A0E94B3
:1059BE00D6A9009B02C0E1E00895E0E00895A1E0C1
:1059CE000E94332C08950A930E94AB2C0E2F0030A8
:1059DE0011F00C94F52CE3E6099108950E98169AA1
:1059EE000E94D6A9069B03C0E0E009910895E1E06C
:1059FE00099108950E98169A0E94D6A9069B02C088
:105A0E00E0E00895E1E008950E9410AA08950E9432
:105A1E0044BBA1971A930A930E9410AA0E9416AA39
:105A2E00ABA1BCA18DA19EA10E941CAA10F40C9446
:105A3E00212D10E200E0011710F00C94362D0E947B
:105A4E0021AAEA0FFB1F0F01E02FABA1BCA18DA174
:105A5E009EA10E9412A9D001EC930F5FECCF0E9481
:105A6E0026AA0E944B1319810881A7960895EF97D5
:105A7E0023970E94AEB99D010E9410AA0E9416AAF9
:105A8E000E9431AA0E941CAA10F40C944F2D10E211
:105A9E0000E0011710F00C94622D0E943AAAFF93B9
:105AAE00EF93E02F0E9431AA0E9412A9AF91BF91ED
:105ABE00EC930F5FEECF0E9441AAD9010E94A31969
:105ACE001E2F113410F40C946D2D10E400E001170C
:105ADE0010F00C947C2D0E943AAA0F01D9010E945D
:105AEE00B0A9D001EC930F5FF2CF0E9441AA0E94A1
:105AFE00B5B9EF962B9608950E94AFB911E020E04C
:105B0E002A3010F00C94A12DA0E00E94C925AFE020
:105B1E000E944DAA11F40C94952D10E0A1E00E9464
:105B2E00C925A3E00E944DAA11F00C949F2D10E000
:105B3E002F5FE6CFE12F0E94B6B923960895EF9717
:105B4E00A597E2E0EA93E0E00E9455AA0E94F511C3
:105B5E00A1E00E94F7250E945CAAACE6B1E080E0CD
:105B6E0090E00E940E2DA0E8B1E080E090E00E944F
:105B7E000E2D0E9460AAE1EAF1E060E070E00E9462
:105B8E006CAA0E94991BE7EBF1E060E070E00E94C6
:105B9E006CAA0E943E2D0E9460AAE3ECF1E060E048
:105BAE0070E00E946CAA0E94991BE0EDF1E060E0AB
:105BBE0070E00E946CAA0E943E2D0E9460AAECED3D
:105BCE00F1E060E070E00E946CAA0E94991BE9EE81
:105BDE00F1E060E070E00E946CAA0E943E2D0E94EF
:105BEE000B2DEF96A5960895AA93EF972F970E94E7
:105BFE0071AA40E00E9476AAE03011F40C940E2EA9
:105C0E00A5EFB1E080E090E00E947BAA06C0AFEF66
:105C1E00B1E080E090E00E940E2D0E9480AA5230EA
:105C2E0010F40C94252E0E945CAA0E9487AAA3E071
:105C3E000E949C4F0E945CAA0E9480AA503011F0D4
:105C4E000C94642EFE01EB5BFF4FE081EA930E9401
:105C5E0095AAEA93FE01EA5BFF4FE081EA930E9468
:105C6E0057A6DE01D4960E94181EE6E0F2E060E030
:105C7E0070E00E949AAAFE01E85BFF4FE081EA9372
:105C8E00FE01E85BFF4FE081EA93E0E2EA93FE015A
:105C9E00E75BFF4FE081EA930E9457A6DE01D5969F
:105CAE000E94C41EE3E1F2E060E070E00E949AAA56
:105CBE000E9495AAE093720E06C0A0E2B2E080E0C8
:105CCE0090E00E947BAAA2E00E94EE4F0E94A0AA42
:105CDE000E946A350E94A6AADE01AF5BBF4FAC914F
:105CEE00A13010F40C94822EAEE2B2E080E090E08F
:105CFE000E947BAA06C0A2E4B2E080E090E00E947F
:105D0E000E2DA1E00E946F25A0E00E946525FE01E8
:105D1E007D960E94ABAA0E946B505E2F503011F4FC
:105D2E000C949C2E4F5FE1E0EE83E0E0EDA7E3E5FF
:105D3E00F2E060E070E00E943FBBDE0191960E94AF
:105D4E003E2DE0E0EB8FE4E6F2E060E070E00E94D2
:105D5E003FBBDE011B960E943E2DA1E00E94C7357F
:105D6E000E94A6AA0E94B0AAE03011F00C94C12E97
:105D7E00E1E0EE83A1E00E946525AAE00E94820E7A
:105D8E00A0E00E942F52AAE00E94990E8F010436C5
:105D9E00E0E01E0710F00C94D52EF2CF0E94E551D4
:105DAE000E9421539F010E9421539F010E94215363
:105DBE009F012A5F30402031E7E23E0710F40C9439
:105DCE00EF2E2138EEE33E0710F00C94EF2E07C0B5
:105DDE00A5E7B2E080E090E00E947BAA0DC03A9366
:105DEE002A93DE01AC5BBF4F0E94C41BE3E8F2E0D6
:105DFE0060E070E00E94B5AA0E9411539F012A50E4
:105E0E0030402832E0E03E0710F40C94152F253078
:105E1E00E1E03E0710F00C94152F07C0A9E9B2E09F
:105E2E0080E090E00E947BAA14C03A932A93E1E0AE
:105E3E00EA93EA93E6E0EA93E0E0EA93DE01A85BF8
:105E4E00BF4F0E94BD18EBEAF2E060E070E00E94E6
:105E5E00B5AAA1E00E946F250E94CD2F0E94A6AA8E
:105E6E00DE01AF5BBF4FAC91A13010F40C94522FFA
:105E7E000E94B0AAF0E0FA93EA93DE01AC5BBF4F4A
:105E8E000E94C41BEFEBF2E060E070E00E94B5AA46
:105E9E00E1E0EE8306C0A6EDB2E080E090E00E9465
:105EAE000E2DA1E00E94C80EA1E00E94E40E8F010B
:105EBE00E091720E0E94A6AA0E9480AA503011F0A4
:105ECE000C946D2F0E9495AA0E94A6AA0230E0E0C3
:105EDE001E0710F00C94802F503011F00C94802F70
:105EEE000E94B0AAA091720EEA1711F00C94802FA6
:105EFE0001C001C0D9CF0230E0E01E0710F40C94AF
:105F0E008F2FA8EEB2E080E090E00E947BAA19C02D
:105F1E00503011F40C949A2FA8EFB2E080E090E08C
:105F2E000E947BAA0EC00E94B0AAA091720EEA1720
:105F3E0011F40C94A82FA6E0B3E080E090E00E944C
:105F4E000E2DEE81E03011F00C94B42FA5E1B3E0EC
:105F5E0080E090E00E940E2D06C0A5E2B3E080E046
:105F6E0090E00E940E2DEE810E94B3B9EF966696D8
:105F7E0008950A930A2F003011F00C94C92F0E9435
:105F8E00A0AA02C00E94BCAA099108950E94AFB9AE
:105F9E000E94A125E093730EA1E00E94C80E0E94FC
:105FAE00BCAA0E94962CE03011F00C94E12F0E94B6
:105FBE00C2AA08950E94AB2CE03011F00C94EA2F87
:105FCE000E94C7AA08950E94B42CE03011F00C94E0
:105FDE00F52FE3E00E94B6B923960895A0E00E9443
:105FEE00CCAA11F40C940030E4E00E94B6B92396CA
:105FFE000895A1E00E94CCAA11F00C940B30E5E0BC
:10600E000E94B6B923960895A1E00E94F725A0E05C
:10601E000E943726A0E00E9417260E940A350E9491
:10602E00D4AA11F40C942030EBE00E94B6B923965A
:10603E0008950E94DEAA11F00C942A30ECE00E9422
:10604E00B6B923960895A1E00E9417260E94D4AAFD
:10605E0011F40C943730EDE00E94B6B923960895F2
:10606E000E94DEAA11F00C944130EEE00E94B6B907
:10607E00239608950E9405160E94E8AAA0E00E94A9
:10608E00EEAAA0E00E94F5AA11F40C945330EFE0B2
:10609E000E94B6B923960895A1E00E94F5AA11F0C8
:1060AE000C945E30E0E10E94B6B923960895A0E00C
:1060BE000E948226A1E00E94EEAA0E94BC260E2F0C
:1060CE00003011F40C947030E1E10E94B6B92396C1
:1060DE000895A1E00E94F5AA11F00C947B30E2E144
:1060EE000E94B6B9239608950E94FEAA0E9403ABA1
:1060FE0011F00C948730E3E10E94B6B9239608950F
:10610E00A0E00E9403AB11F40C949230E3E10E94E4
:10611E00B6B923960895A2E00E943E280E94F52B60
:10612E00A1E00E94CD260E945CAA0E946817A0E002
:10613E000E945527A1E00E9407280E940CAB0E94E6
:10614E0013AB11F40C94B030E4E10E94B6B923966F
:10615E0008950E9418AB0E9413AB11F00C94BC3042
:10616E00E5E10E94B6B9239608950E9462280E2F8B
:10617E00003011F00C94C830E6E10E94B6B92396B7
:10618E000895A0E00E94CD26A0E00E9407280E945C
:10619E005CAA0E941DAB0E9413AB11F00C94DC3074
:1061AE00E7E10E94B6B9239608950E9462280E2F49
:1061BE00003011F40C94E830E8E10E94B6B9239651
:1061CE000895A0E00E94FB26A4E1B0E00E940A0E12
:1061DE000E9422AB11F40C94F930E9E10E94B6B999
:1061EE0023960895A1E00E94FB260E940A350E9484
:1061FE0022AB11F00C940831EAE10E94B6B9239655
:10620E000895A0E00E94FB260E9427AB0E94F22672
:10621E000E2F003011F00C941931EBE10E94B6B93B
:10622E0023960895A1E00E94FB260E945CAA0E947C
:10623E00F2260E2F003011F40C942A31ECE10E945C
:10624E00B6B923960895A0E00E94FB260E948C2CDE
:10625E000E942BABA1E00E9407280E942BAB0E944C
:10626E0013280E2F003011F00C944231EDE10E94F4
:10627E00B6B923960895A0E00E9407280E940A3519
:10628E000E9427AB0E9413280E2F003011F40C949D
:10629E005531EEE10E94B6B9239608950E94FEAAEA
:1062AE000E94132CA0E00E946B270E94F52B0E94E7
:1062BE002FABA1E00E9436AB11F40C946B31EFE1E1
:1062CE000E94B6B923960895A0E00E9436AB11F055
:1062DE000C947631E0E20E94B6B9239608950E949E
:1062EE0018AB0E943BAB11F00C948231E1E20E949C
:1062FE00B6B9239608950E941DAB0E943BAB11F4D4
:10630E000C948E31E2E20E94B6B923960895A0E075
:10631E000E9486270E940A350E943BAB11F40C9412
:10632E009D31E3E20E94B6B9239608950E942FABE9
:10633E000E945CAAA0E00E9440AB11F40C94AC3118
:10634E00E4E20E94B6B923960895A1E00E9440AB04
:10635E0011F00C94B731E5E20E94B6B92396089578
:10636E000E9449ABA0E00E946B270E9427AB0E94BF
:10637E008C2C0E2F003011F00C94CA31E6E20E94E4
:10638E00B6B923960895A1E00E946B270E9450ABE8
:10639E000E948C2C0E2F003011F40C94DB31E7E2AE
:1063AE000E94B6B923960895A0E00E946B27A1E043
:1063BE000E948627A0E00E945527A0E00E94072891
:1063CE00A2E00E946C280E9427AB0E9418AB0E948C
:1063DE003BAB11F00C94F831E8E20E94B6B923966B
:1063EE0008950E941DAB0E943BAB11F40C94043235
:1063FE00E9E20E94B6B9239608950E9490280E2FC6
:10640E00003011F40C941032EAE20E94B6B92396D1
:10641E0008950E9449AB0E9427AB0E9418AB0E94C0
:10642E003BAB11F00C942032EBE20E94B6B92396EE
:10643E0008950E941DAB0E943BAB11F40C942C32BC
:10644E00ECE20E94B6B9239608950E9490280E2F72
:10645E00003011F00C943832EDE20E94B6B923965A
:10646E000895A0E00E9407280E9427ABA0E00E949A
:10647E009A280E94C0280E2F0E9453AB0E94842996
:10648E00A1E00E94BB290E9450AB0E9461AB11F0AB
:10649E000C945632EEE20E94B6B923960895A0E00F
:1064AE000E94BB290E9450AB0E9461AB11F40C9468
:1064BE006532EFE20E94B6B923960895A1E00E94DC
:1064CE0024290E9450AB0E9461AB11F00C947432DF
:1064DE00E0E30E94B6B923960895A0E00E94242915
:1064EE000E9450AB0E9461AB11F40C948332E1E335
:1064FE000E94B6B923960895A1E00E9444290E94F5
:10650E0050AB0E9461AB11F00C949232E2E30E9408
:10651E00B6B923960895A0E00E9444290E9450AB7C
:10652E000E9461AB11F40C94A132E3E30E94B6B960
:10653E0023960895A1E00E949A290E9450AB0E94D2
:10654E0061AB11F00C94B032E4E30E94B6B923961D
:10655E000895A0E00E949A290E9450AB0E9461AB60
:10656E0011F40C94BF32E5E30E94B6B92396089558
:10657E00A1E00E9484290E940CAA0E940A350E9462
:10658E0061AB11F00C94D032E6E30E94B6B92396BB
:10659E000895A0E00E9484290E940CAA0E9461AB7B
:1065AE0011F40C94DF32E7E30E94B6B923960895F6
:1065BE00A0E00E941C28A1E00E94C4270E942BABE1
:1065CE000E9434280E2F003011F40C94F332E8E3BD
:1065DE000E94B6B923960895A0E00E94C4270E9497
:1065EE002BAB0E9434280E2F003011F00C94043384
:1065FE00E9E30E94B6B923960895A1E00E94DA2736
:10660E000E9427AB0E94FE270E2F003011F00C9433
:10661E001533EAE30E94B6B9239608950E941DAB86
:10662E000E9413AB11F00C942133EBE30E94B6B928
:10663E00239608950E9418AB0E9413AB11F40C948C
:10664E002D33ECE30E94B6B923960895A0E00E9484
:10665E00DA270E945CAA0E940A350E94FE270E2F9E
:10666E00003011F40C944033EDE30E94B6B923963A
:10667E0008950E941DAB0E9413AB11F00C944C3385
:10668E00EEE30E94B6B9239608950E9418AB0E94BD
:10669E0013AB11F00C945833EFE30E94B6B9239666
:1066AE000895A1E00E9466AB11F00C946333E0E410
:1066BE000E94B6B923960895A0E00E9466AB11F42D
:1066CE000C946E33E1E40E94B6B923960895A1E0CE
:1066DE000E946FAB11F00C947933E2E40E94B6B9CC
:1066EE0023960895A0E00E946FAB11F40C948433AE
:1066FE00E3E40E94B6B923960895A1E00E9478AB18
:10670E0011F40C948F33E4E40E94B6B923960895E5
:10671E00A0E00E9478AB11F00C949A33E5E40E944D
:10672E00B6B923960895A1E00E9481AB11F00C94A6
:10673E00A533E6E40E94B6B923960895A0E00E9420
:10674E0081AB11F40C94B033E7E40E94B6B92396F2
:10675E000895A1E00E948AAB11F00C94BB33E8E4DB
:10676E000E94B6B923960895A0E00E948AAB11F458
:10677E000C94C633E9E40E94B6B923960895A1E0BD
:10678E000E9493AB11F00C94D133EAE40E94B6B997
:10679E0023960895A0E00E9493AB11F40C94DC3381
:1067AE00EBE40E94B6B923960895A1E00E949CAB3B
:1067BE0011F00C94E733ECE40E94B6B923960895D9
:1067CE00A0E00E949CAB11F40C94F233EDE40E9415
:1067DE00B6B923960895A1E00E94A5AB11F00C94D2
:1067EE00FD33EEE40E94B6B923960895A0E00E9410
:1067FE00A5AB11F40C940834EFE40E94B6B92396BD
:10680E000895A1E00E94AEAB11F40C941334E0E5B0
:10681E000E94B6B923960895A0E00E94AEAB11F087
:10682E000C941E34E1E50E94B6B923960895A1E0BA
:10683E000E94B7AB11F40C942934E2E50E94B6B96C
:10684E0023960895A0E00E94B7AB11F00C94343457
:10685E00E3E50E94B6B9239608950E94F52B0E9497
:10686E000CAB0E94F52B0E2F003011F40C94443417
:10687E00E4E50E94B6B9239608950E9418AB0E94D3
:10688E00F52B0E2F003011F00C945234E5E50E94DA
:10689E00B6B923960895A1E00E94C0AB11F00C94F6
:1068AE005D34E6E50E94B6B923960895A0E00E94F5
:1068BE00C0AB11F40C946834E7E50E94B6B9239688
:1068CE000895A0E00E946B270E94C9AB11F40C94AE
:1068DE007534E8E50E94B6B9239608950E94C9ABB7
:1068EE0011F40C947F34E9E50E94B6B9239608950D
:1068FE00A1E00E94F725A1E00E94D3AB11F00C9409
:10690E008D34EAE50E94B6B923960895A0E00E9460
:10691E00D3AB11F40C949834EBE50E94B6B92396E0
:10692E000895A0E00E94B227A1E00E949C270E9439
:10693E005CAA0E94DCAB11F00C94AA34ECE50E9428
:10694E00B6B923960895A0E00E949C270E945CAAE7
:10695E000E94DCAB11F40C94B934EDE50E94B6B98B
:10696E0023960895A0E00E949C27A1E00E94B227E2
:10697E000E945CAA0E94DCAB11F00C94CB34EEE5C5
:10698E000E94B6B923960895A0E00E94B2270E94F5
:10699E005CAA0E94DCAB11F40C94DA34EFE50E9491
:1069AE00B6B923960895A1E00E94E40E1E2F2F2F54
:1069BE000E94A1250E2F1230E0E02E0710F00C944D
:1069CE00EF34A091730E0A1711F00C94EF3401C03E
:1069DE0001C0E9CF0E94A1250E2FA091730E0A17B8
:1069EE0011F00C9401351031E0E02E0710F00C94EC
:1069FE00013501C005C0E0E60E94B6B923960895A0
:106A0E000E94E1AB08950E94E6AB0895EF97EF97D1
:106A1E00EF9765970E94ADB94A2F00E0242F3327D8
:106A2E00D901E6E00E94F0B99F0110E0103410F099
:106A3E000C9428350E94EAABE12FED5FEC931F5FBB
:106A4E00F5CF0E94F2ABDE01AB56BF4F0E94BB0CDE
:106A5E000E94F2ABDE01A15BBF4F0E94F90C0E94B7
:106A6E000CAA0E94F9ABE0E0EA93A6E40E94FEAB0A
:106A7E00E0E4F0E00E94ABAA0E94BB0C10E01034E0
:106A8E0010F00C9459350E94EAAB0C90E12FF0E017
:106A9E000E94EAA7EC91E01511F40C94573501E031
:106AAE001F5FEDCF0E94F2ABDE01AB56BF4F0E94CF
:106ABE00F90C0E940CAAE02F0E94B4B9EF96EF9643
:106ACE00EF966A9608951A930A931FE3A12F0E94D8
:106ADE000D350E2F003011F40C947935E1E009914B
:106AEE0019910895E0E009911991089528970E944F
:106AFE00ADB94A2F10E0413011F00C94873516EAEB
:106B0E00423011F00C948C351EEA2CEF3FEE0E94B1
:106B1E0004ACE1E2F3E465E070E00E94D6A50E94C9
:106B2E000FAC11F00C94A7350E9404AC0E9421AC5E
:106B3E0011F00C94A735E2E00E94B4B92D96089599
:106B4E002CEF3FE70E9404ACE4E3F2E160E070E07A
:106B5E000E94D6A50E940FAC11F00C94C2350E9473
:106B6E0004AC0E9421AC11F00C94C235E1E00E94FD
:106B7E00B4B92D960895E0E00E94B4B92D9608950B
:106B8E00AA930E94AFB92B81A0E00E948B25A1E0B1
:106B9E000E947D350E2F003011F00C94DF35A5E3E9
:106BAE00B3E080E090E00E940E2D0E942AAC089582
:106BBE00013011F00C94F235203011F40C94ED35B7
:106BCE00A7E4B3E080E090E00E940E2DE1E00E9489
:106BDE00B6B924960895A2E00E947D351E2F10307E
:106BEE0011F00C940936203011F40C940436ACE5F7
:106BFE00B3E080E090E00E940E2DE2E00E94B6B974
:106C0E0024960895113011F00C941A36203011F498
:106C1E000C941736A1E7B3E080E090E00E940E2DB1
:106C2E000E942AAC0895123011F00C942D362030AB
:106C3E0011F40C942836A9E8B3E080E090E00E94AD
:106C4E000E2DE3E00E94B6B9249608950E942AAC58
:106C5E000895A0E00E949C170895AFEF0E949C1724
:106C6E0008950A9300E0013010F00C946136ABE207
:106C7E000A9FF001EC53F14F0E942FACEB53F14FF2
:106C8E000E942FACEA53F14F0E942FACE953F14F03
:106C9E000E942FACE853F14F0E942FACE753F14FF7
:106CAE000E942FACE653F14F0E942FAC0E9435ACE0
:106CBE000F5FD9CFE1E0E03011F40C946B36E03089
:106CCE0011F40C946B3601C006C0E1E0E093C40EE3
:106CDE00EBE7E093C50EE0E0E03011F40C947C3667
:106CEE00E03011F40C947C3601C006C0E1E0E09374
:106CFE00EF0EEBE0E093F00EE0E0E03011F40C94D8
:106D0E008D36E03011F40C948D3601C006C0E1E0F2
:106D1E00E0931A0FE3E3E0931B0FE0E0E093C10E64
:106D2E00E093C30EE093C20E00E0063210F00C9416
:106D3E00A636E02F0F5F0E943AAC0F5FF6CFE0E071
:106D4E00E093C00E099108950E94AFB9E091C20E72
:106D5E00E03011F00C94B6360E9446AC08950E94B5
:106D6E008838E03011F00C94BF360E9446AC08957E
:106D7E00E091C30EE03011F00C94E436E0E0E093C5
:106D8E009C0FE0939B0F0E942D390E2F003011F4B3
:106D9E000C94E4360E946B39A091C10E0E94F23918
:106DAE001E2F103011F00C94E036E1E0E093C30E8C
:106DBE0004C020E00E94E1AB0895A091C30EA13063
:106DCE0011F00C9432370E94B83A0E2F013011F0A8
:106DDE000C9400370E944FAC0E9458AC0E945DACE0
:106DEE000E9463AC0E9468ACE553F14FA1E0A08312
:106DFE001FC0023011F00C940E37E2E0E093C30E88
:106E0E00A0EAB3E080E090E00E94649311C00330EA
:106E1E0011F00C941637E3E0E093C30E09C0E2E0E4
:106E2E00E093C30EACEAB3E080E090E00E9464937E
:106E3E00033011F40C94313720E0263210F00C940C
:106E4E002E37E22F2F5F0E943AAC2F5FF6CFE0E095
:106E5E00E093C00E84C0A091C30EA23011F00C942A
:106E6E007137E0919C0FEF5FE0939C0FA0919C0F08
:106E7E00A33010F40C945D370E945DACE553F14FD6
:106E8E00A2E0A0830E945DAC0E9463AC0E9468AC3D
:106E9E00E853F14FA0E0A083E0E0E093C30EABEB2C
:106EAE00B3E080E090E00E94649313C0A091C10E05
:106EBE000E94643A1E2F103011F00C946C37E1E0F2
:106ECE00E093C30E0E94C2AA089520E00E94E1AB97
:106EDE00089545C0A091C30EA33011F00C94B6379F
:106EEE00E0919B0FEF5FE0939B0FA0919B0FA33060
:106EFE0010F40C9490370E945DACE553F14FA3E073
:106F0E00A0830E945DAC0E9458AC0E944FAC0E94C0
:106F1E006DAC0E9480390E2F003011F40C949B370B
:106F2E00E1E0E093C30E0DC0A091C10E0E94C639E0
:106F3E000E945DACE553F14FA4E0A083E0E0E09346
:106F4E00C30E20E0263210F00C94B337E22F2F5FE1
:106F5E000E943AAC2F5FF6CFE0E0E093C00E0E94A5
:106F6E00C2AA0895A1E00E942827AEE6B0E00E94D2
:106F7E000A0EA0E00E94282708950A930E94B42CBE
:106F8E000E2F003011F40C94D337E091C20EE03086
:106F9E0011F40C94D33701C003C0E1E009910895B8
:106FAE00E0E009910895A0E00E948627A0E00E94EB
:106FBE006B270E946817E0E0E093C20EA7ECB3E0E7
:106FCE0080E090E00E9464930895A0E00E9455270F
:106FDE000E94FEAA0E94132CA1E00E946B27E2E001
:106FEE00EA93E0E0EA93E4E00E9472AC0E94DE16BF
:106FFE000E946C17E1E0E093C20EAFECB3E080E0CC
:10700E0090E00E946493E1E008950A930A2F013004
:10701E0011F00C941638A1E00E946B2715C00230B7
:10702E0011F00C942838A1E00E946B270E940CAA44
:10703E00A0E00E946B270E940CAAA1E00E946B2781
:10704E0003C0A0E00E946B27099108950E945DA5E0
:10705E00A091C00EA63210F00C944038E091C00EF4
:10706E00EF5FE093C00E0E9477ACEA0FFB1F108318
:10707E0021831030E1E02E0714F40C944D38A091CA
:10708E00C00EA13011F00C944D3801C003C0009118
:10709E00C00E0F5F0E94B6B9239608950E9475A97F
:1070AE00113010F00C948438003011F40C946D38BB
:1070BE00ABE21A9FF001EA53F14FA1E0A083A6EDD7
:1070CE00B3E080E090E00E94649317C0ABE21A9F99
:1070DE00F001EA53F14F0E947EAC0E946DAC0E940B
:1070EE0084AC0E947EAC0E9458AC0E948AACA8EE82
:1070FE00B3E080E090E00E946493198108812396AA
:10710E0008950A9300E0013010F00C949B38ABE226
:10711E000A9FF0010E948EAC11F40C949938E1E0B4
:10712E00099108950F5FEFCFE0E0099108950E9455
:10713E0075A9113010F00C94AE38ABE21A9FF00125
:10714E00E953F14F00830E9484ACA0E0A083198123
:10715E000881239608950E94ADB98D012D813E813F
:10716E004F811A930A93ABE24A9FF001E453F14F19
:10717E00FA93EA93A22FBB270E94961A413010F081
:10718E000C94D438ABE24A9FF001E953F14F3083AF
:10719E004A9FF001E753F14F20830E94B4B928961D
:1071AE0008951A930A931A2F113010F00C94F03898
:1071BE0000E0033210F00C94F038ABE21A9FF001AD
:1071CE00E453F14FDF01EE27A00FBE1FEC930F5FCC
:1071DE00F0CF0E9484AC0E947EAC0E9458AC0E94FC
:1071EE008AAC0991199108951A930A931A2FABE25A
:1071FE001A9FF001E553F14F00810E948AACE02FF7
:10720E000991199108950A930A2FABE20A9FF00192
:10721E00E653F14FE081099108950E94AFB98D01B7
:10722E002B81ABE22A9FF001E453F14FFA93EA93DC
:10723E001A930A932A9FF001E653F14FA081B0E012
:10724E000E94961A0E94B6B9249608950E94AEB96D
:10725E002FE030E0A9E00E94990E8F01021713076C
:10726E0010F00C943F39E0E00E94B5B924960895D1
:10727E00A9E00E94820E20E030E0E091C10EEF5FA7
:10728E00E093C10EA091C10EA13010F40C945239AE
:10729E00E0E0E093C10E0E945DAC0E948EAC11F452
:1072AE000C945E39E1E00E94B5B924960895F90177
:1072BE0031969F01329710F00C946639DECFE0E0E4
:1072CE000E94B5B9249608950E94D9A50632E0E031
:1072DE001E0714F00C947B39F8010E9493AC0E94A7
:1072EE009AAC0F5F1F4FF2CF0E946C170991199144
:1072FE00089522970E94ACB9A091C00EA13010F44F
:10730E000C949039E091C00EE150F0E0EE83FF83D3
:10731E0003C0E0E0EE83EF8300E010E020E030E019
:10732E00EE81FF812E173F0710F00C94A639F9015C
:10733E000E9493AC0E949FAC2F5F3F4FF1CF107015
:10734E00EE81FF810E9493AC4D915C91507040177D
:10735E00510711F40C94BD39E0E0E093740EE09304
:10736E00750EE1E00E94B3B928960895EE81FF8173
:10737E000E9493AC0E949AAC0E94A4AC08950E9405
:10738E00AFB92A2F1091C00E113010F40C94D039D1
:10739E00115000E0011710F00C94E839ABE22A9F6F
:1073AE00F001E453F14FDF01E02F0E946AA9E02FB4
:1073BE00A4E7BEE0F0E0EE0FFF1F0E94BFA70F5F35
:1073CE00E9CFABE22A9FF001E653F14F10830E9402
:1073DE00B6B9239608950E94A9AC11F00C94FC390D
:1073EE00E1E00E94B3B9AD9608950E94B7AC0E9439
:1073FE008EAC11F00C94083AE2E00E94B3B9AD964F
:10740E0008950E94B7ACE953F14F1081113010F47A
:10741E000C941B3A0E94B7ACE853F14F10830E94B4
:10742E00B7AC0E946DAC0CC00E94B7ACE853F14FE4
:10743E00BF010E94B7ACEB53F14FE081DB01EC933F
:10744E000E94BCACBF010E94B7AC0E94BFACE75318
:10745E00F14F2081103011F00C94363A20E0243296
:10746E0010F40C943B3A23E20E8140E050E0E22F00
:10747E000E94C5AC14F00C944D3A0E94B7AC0E9419
:10748E00CAAC1083010F4F5F5F4FF1CF0E94BCACAF
:10749E0000830E9467A90E94D0ACE32F0E94C5AC66
:1074AE0014F00C945F3A0E94E0AC4F5F5F4FF5CF43
:1074BE00E0E00E94B3B9AD9608950E94A9AC11F018
:1074CE000C946E3AE1E00E94B3B9AD9608950E9415
:1074DE00B7AC0E948EAC11F00C947A3AE2E00E94A6
:1074EE00B3B9AD960895A9EFB3E080E090E00E94A5
:1074FE0064930E94BCACBF010E94B7AC0E94BFACAB
:10750E00E753F14F2081243210F40C948F3A23E28A
:10751E000E8140E050E0E22F0E94C5AC14F00C94B6
:10752E00A13A0E94B7AC0E94CAAC1083010F4F5F04
:10753E005F4FF1CF0E94BCAC00830E9467A90E94EE
:10754E00D0ACE32F0E94C5AC14F00C94B33A0E9459
:10755E00E0AC4F5F5F4FF5CFE0E00E94B3B9AD9660
:10756E00089525970E94E7ACE0E0EC830E947AA98B
:10757E00EAEFF0E0EE83FF830E94E6ABA091C00E2F
:10758E00A13010F40C94F33AE885EA1710F00C943D
:10759E00D93AEE81FF81EC59FF4FEE83FF83E091E4
:1075AE00C00EE88720E030E0E091C00ED901F0E097
:1075BE00AE17BF0710F00C94F33AF9010E9493AC8A
:1075CE000E942CBBF17011F40C94F03AE22FEF5F95
:1075DE00EA872F5F3F4FE8CF0F5F1F4F0E9408A92A
:1075EE0010F00C94063BA091C00EA83210F00C9433
:1075FE00063BAA85A03011F00C94063B01C001C0D9
:10760E00BBCFA091740EB091750EA030E1E0BE0715
:10761E0011F00C94193BA091C00EA13011F00C94F6
:10762E00193B01C005C0E1E00E94B3B92B96089545
:10763E00AA85A03011F40C94303B0E9408A910F0DA
:10764E000C94303BA091C00EA03011F40C94303B42
:10765E0005C0E2E00E94B3B92B9608954091C00E8A
:10766E00552750704150504020E030E02417350728
:10767E0010F00C944C3BF9010E9493ACEC91A9854F
:10768E00EA0FE9872F5F3F4FF1CFE091C00E0E94C6
:10769E0077AC0E9497A5F070A985B0E0EA17FB07BA
:1076AE0011F40C94613B0E943436E2E00E94B3B9AF
:1076BE002B9608950E943036E3E00E94B3B92B96C4
:1076CE0008950E94B3B92B9608950A9300E00830EE
:1076DE0010F00C94833BA3E00A9FF001E356F04FA9
:1076EE000E94EBACE256F04F0E94EBACE156F04F2D
:1076FE00A0E0A0830F5FEBCFE0E0E093B50FE09347
:10770E00B70FE3E6E093B60FE0E0E093B90FE09336
:10771E00B80F09910895E3E6E093B60F0E94F1AC1D
:10772E00A4E0B4E080E090E00E9464930895AA97EC
:10773E000E94ACB9A091B60FA33611F00C94AC3BDD
:10774E00E0E00E94B3B9E0960895E091B60FE03004
:10775E0011F00C94C73B0E94C437E03011F40C9426
:10776E00C03B0E94F6AC10F40C94BF3B0E94FEACE2
:10777E0002C00E9404ADE0E00E94B3B9E096089505
:10778E00A091B60FA13011F00C94D23B0E940AAD1D
:10779E000E94FEACCCC1A091B60FA23011F00C9499
:1077AE00E83B0E94F6AC10F40C94E73BE0E0EA9361
:1077BE00A8E70E949E38A5E10E94820E0E94FEACB0
:1077CE00B6C1A091B60FA33011F00C94263C0E94C6
:1077DE0013AD013011F40C94F93B043011F40C94F8
:1077EE00F93B04C00E94FEAC0E9404ADA5E10E94CC
:1077FE00990EAF014536E0E05E0710F40C941C3C88
:10780E000E9418ADA63010F40C94193C0E94F1ACF5
:10781E00E0E0E093B80FE9ECE093C50FE0E0E09311
:10782E00B60F03C0E1E0E093B60F0E94C437E0301C
:10783E0011F00C94253CE0E0E093B60F78C1A091D6
:10784E00B60FA43011F00C94393CA5E10E94990EAC
:10785E00AF014333E0E05E0710F40C94383C0E9415
:10786E00FEAC65C1A091B60FA53011F00C94423C50
:10787E000E9420AD5CC1A091B60FA63011F00C9401
:10788E00D93C0E9413AD043011F00C94CF3C0E94F1
:10789E0026AD153010F00C946D3C0E9418ADA53637
:1078AE0010F40C94663C0E94F1ACE0E0E093B80F4B
:1078BE00EAECE093C50FE0E0E093B60F06C0A5E159
:1078CE000E94820EE4E0E093B60F62C00E942BADE0
:1078DE00E4E0F0E0FF93EF93E985EA93AB850E9435
:1078EE004920AF91BF910E9468BBEB85A0E0B0E04C
:1078FE000E9470BBA1E0B0E0EC850E9470BBA2E0DC
:10790E00B0E0ED850E9470BB20E0203110F00C94A9
:10791E009E3CA8E0B0E0E22F0E946AA9E22FE25F4F
:10792E00F0E0DE0118960E9431AD2F5FEECFA8E198
:10793E00B0E0E1E00E9470BB0E94FEACA5E10E94A7
:10794E00820EE1E0E093C50FA4E0B0E00E9438ADF6
:10795E00ECE0F4E060E070E00E943FBBAA85BB85DE
:10796E000E943DADA0E0B0E00E9454BB3E2FEAE184
:10797E00F4E060E070E00E9441ADA1E0B0E00E9452
:10798E0054BB3E2FE6E2F4E060E070E00E9441ADB1
:10799E000E94C437E03011F00C94D83CE0E0E09344
:1079AE00B60FC5C0A091B60FA73011F00C94E23CF3
:1079BE000E9420ADBCC0A091B60FA83011F00C945F
:1079CE00203DE091B80FE03011F40C94FB3CE091B7
:1079DE00B90FE03011F00C94FB3CA091B50FA33021
:1079EE0010F00C94FB3C01C003C0E9E0E093B60F2D
:1079FE00E091B80FE03011F40C94123DE091B90F04
:107A0E00E03011F40C94123DA091B50FA33010F09C
:107A1E000C94123D01C003C0EAE0E093B60F0E9441
:107A2E00C437E03011F00C941F3DE0E0E093B60F48
:107A3E007EC0A091B60FA93011F00C94613DE0917B
:107A4E00B80FE03011F00C942F3DE8E0E093B60F44
:107A5E00E091B90FE03011F40C94383DEAE0E09378
:107A6E00B60F0E94C437E03011F00C94413DE0E0B7
:107A7E00E093B60FA091B50FA83010F40C944A3DC8
:107A8E00E8E0E093B60F0E9413AD043011F00C94B1
:107A9E00603D0E9426AD113010F40C94603D0E94A2
:107AAE002BAD1A93DE0119960E94A63FE6E0E093F5
:107ABE00B60F3DC0A091B60FAA3011F00C949E3DAA
:107ACE00E091B80FE03011F00C94703DE6E0E093D9
:107ADE00B60FE091B90FE03011F00C94793DE7E06C
:107AEE00E093B60F0E94C437E03011F00C94823D43
:107AFE00E0E0E093B60FA091B50FA83010F40C940F
:107B0E008B3DE6E0E093B60F0E9413AD043011F00A
:107B1E000C949E3D0E9426AD113010F40C949E3DA7
:107B2E000E942BAD1A93DE0119960E94A63FE1E04A
:107B3E000E94B3B9E09608950E94ACB9AD01AAE1D6
:107B4E00B0E0EF81F8850E9468BBACE1B0E0EE8159
:107B5E000E9470BB00E010E00031E0E01E0710F064
:107B6E000C94CE3DF801DA010E9449AD2D913C9165
:107B7E00AEE1B0E0F801EE0FFF1FAE0FBF1FF9012F
:107B8E000E9468BB21E030E00F5F1F4FE5CFA8E1F8
:107B9E00B0E00E944EAD0895A4970E94AFB920E0C8
:107BAE00223110F00C94E53DE22FF0E0DE01139649
:107BBE000E9449AD0E949AAC2F5FF2CFE5E0F0E053
:107BCE00E98FFA8FEAE0F0E0E98FFA8FE4E1F0E076
:107BDE00EB8FFC8FE2E3F0E0ED8FFE8FE4E6F0E05A
:107BEE00EF8FF8A3E8ECF0E0E9A3FAA30FEF1FEF95
:107BFE001A930A930E9456AD0E94A33DE0E00E94A4
:107C0E00B6B9A79608950E94C437E03011F00C94CF
:107C1E00153EE0E0E093B60FE1E00895E0E0089550
:107C2E00E091B60F08950A930A2FA091B60FA336CE
:107C3E0011F00C94253EE0E0E093B60FA091B60F44
:107C4E00A63010F00C942E3EE0E00991089500301D
:107C5E0011F00C94393E0E94F1ACE0E0E093B80FC5
:107C6E00099108950E940AADE1E0099108952697C1
:107C7E001A930A93A091B60FA33611F00C944A3EB4
:107C8E00E0E0E093B60FA091B60FA63010F00C9482
:107C9E00553EE1E01981088128960895E091B80FCC
:107CAE00E03011F00C94603EE2E0198108812896D4
:107CBE000895AAE1B0E00E9450BB8F01002E012A68
:107CCE0011F00C94723EE0E0E093B90FE3E01981FD
:107CDE00088128960895E1E0E093B90F0E945BAD0C
:107CEE000E9472ADDE0115960E94B238A5E3B4E093
:107CFE0080E090E00E946493E0E01981088128966C
:107D0E0008952697A091B60FA63010F00C94923ECF
:107D1E00E1E0269608950E9479AD0E9472ADDE01D3
:107D2E0013960E94B238E0E0E093B90FA4E4B4E0F9
:107D3E0080E090E00E946493E0E026960895BA9366
:107D4E00AA930E947AA90034E0E01E0710F00C946A
:107D5E00B63EF8010E94B3A60F5F1F4FF4CFA8E105
:107D6E00B0E00E9454BBAE81BF81EC93E091B60FA0
:107D7E00AE81BF811196EC93A2E0B0E00E9482AD7D
:107D8E00A4E0B0E00E9489ADA0E0B0E00E949FADFB
:107D9E00A1E0B0E00E94A6AD0031E0E01E0710F0B9
:107DAE000C94E53EF80137960E94D3A70F01E8E048
:107DBE00F0E00E94AFAD0F5F1F4FEECFAAE1B0E033
:107DCE000E94B7ADACE1B0E00E94C1ADE091B80F3A
:107DDE00AE81BF815A96EC93E091B90F0E94C8AD67
:107DEE000031E0E01E0710F00C940A3FAEE1B0E067
:107DFE00F8010E9449AD0E94D1AD0E94D8AD4083DA
:107E0E000F5F1F4FEDCFE0E40E94B3B9289608959F
:107E1E00E091B50F08950E9467A5E091B50FE0308F
:107E2E0011F00C942D3FAD85BE85E0E00E94DFADD4
:107E3E00EFEFEC93AF81B885E0E0EC93AD81BE81BE
:107E4E00EC93E1E00E94B4B92F960895E091B50F3E
:107E5E00E150E093B50F0E94E7ADE03011F40C94C1
:107E6E007A3F0E94E7ADAD85BE850E94F0ADE25629
:107E7E00F04FE081A985BA850E94F0ADE156F04F32
:107E8E004081AB85BC854C93403110F00C94653F1E
:107E9E00AEE1B0E0E42FF0E00E9449AD0E94F7ADF4
:107EAE0010F00C945C3F980109C0A8E0B0E0EE27FA
:107EBE00A40FBE1F0E9454BB2E2F3327AF81B8854F
:107ECE002C93E32FF070AD81BE810E94F0ADE3568E
:107EDE00F04F0E94FEADE256F04F0E94FEADE1560D
:107EEE00F04FA0E0A083E0E00E94B4B92F96089571
:107EFE000E9475A9A091B50FA83010F40C948C3F78
:107F0E00E1E019810881239608950E9406AEE3569A
:107F1E00F04FA1E0A0830E9406AEE256F04F008320
:107F2E000E9406AEE156F04F1083E091B50FEF5F61
:107F3E00E093B50FE0E01981088123960895BA9376
:107F4E00AA93A2970E94ACB94FEF5FEF3AA50E9499
:107F5E000CAEE8A5F9A50E9460A7A32FBB270E942F
:107F6E00961A00E0E02FF0E00E947BA7EC91E07FF4
:107F7E001E2FE02FF0E00E947BA7EC91EF702E2FCA
:107F8E00103711F40C94D03F103811F40C94D03FEC
:107F9E0001C0422F103711F00C94DC3FE2E5F4E003
:107FAE0060E070E00E9416AE0AC0103811F00C941A
:107FBE00E63FE1E6F4E060E070E00E9416AE1039B4
:107FCE0011F40C94EF3F103A11F40C94EF3F07C0EC
:107FDE00522FAFE6B4E080E090E00E9464930F5F12
:107FEE00031710F00C94FC3FBDCF4A93A52F0E94AF
:107FFE007F3FE1E00E94B3B9AB9608950A9300E08B
:10800E000A3010F00C941C40A3E00A9FF001E952D4
:10801E00F04F0E94EBACE852F04F0E94EBACE752EF
:10802E00F04FA0E0A0830F5FEBCFE0E0E093F50F01
:10803E00E093F70FE093F60FE093F90FE093F80F4C
:10804E0009910895A8970E94ADB9E091F60FE0301E
:10805E0011F00C944B400E94C437E03011F40C9494
:10806E0040400E941EAE10F40C943F400E9427AE7A
:10807E0006C0E0E0E093F70FA5E10E94820EE0E07B
:10808E000E94B4B9AD960895A091F60FA13011F0EB
:10809E000C945C40E1E0EA93A8E00E949E38A5E1D2
:1080AE000E94820E0E9427AE89C1A091F60FA230C7
:1080BE0011F00C946F400E941EAE10F40C946E40A2
:1080CE000E942DAE0E9427AEA5E10E94820E76C1BF
:1080DE00A091F60FA33011F00C94A9400E9436AE79
:1080EE00013011F40C948040043011F40C94804053
:1080FE0005C0E0E0E093F70F0E9427AEA5E10E94D5
:10810E00990E3E2F4F2F3536E0E04E0710F40C94AB
:10811E009F400E943BAEA63010F40C949C400E94EF
:10812E0043AEE9ECE093C50F03C0E1E0E093F60F38
:10813E000E94C437E03011F00C94A840E0E0E093C8
:10814E00F60F3CC1A091F60FA43011F00C94B7407D
:10815E00E1E0EA93A9E00E949E380E9427AE2EC16C
:10816E00A091F60FA53011F00C9432410E9436AE5C
:10817E00043011F00C9428410E944CAE153010F0D2
:10818E000C94DC400E943BAEAB3010F40C94D84003
:10819E000E9443AEEAECE093C50FE0E0E093F60FE9
:1081AE0003C0E4E0E093F60F4CC00E9456AD0E946F
:1081BE001439A0E4B0E0ED810E9470BBE2E4F0E07F
:1081CE00FF93EF93EE81EA93A8850E944920AF9129
:1081DE00BF910E9468BBE885AEE3B0E00E9470BB21
:1081EE00AFE3B0E0E9850E9470BBE4E4F0E0FF93FA
:1081FE00EF93EA85EA93AC850E944920AF91BF9137
:10820E000E9468BB20E0203110F00C941E41A6E4C1
:10821E00B0E0E22F0E946AA9E22FE95FF0E00E942F
:10822E00EAA7EC91D0010E9470BB2F5FECCFA6E5C0
:10823E00B0E0E1E00E9470BB0E9427AEE1E0E09367
:10824E00C50F0E94C437E03011F00C943141E0E0CC
:10825E00E093F60FB3C0A091F60FA63011F00C9478
:10826E007041E091F80FE03011F40C944B41E09125
:10827E00F90FE03011F00C944B41A091F50FA330A3
:10828E0010F00C944B4101C003C0E7E0E093F60FF1
:10829E00E091F80FE03011F40C946241E091F90F87
:1082AE00E03011F40C946241A091F50FA33010F060
:1082BE000C94624101C003C0E8E0E093F60F0E9407
:1082CE00C437E03011F00C946F41E0E0E093F60F0C
:1082DE0075C0A091F60FA73011F00C94AB41E09150
:1082EE00F80FE03011F00C947F41E6E0E093F60FCA
:1082FE00E091F90FE03011F40C948841E8E0E0933E
:10830E00F60F0E94C437E03011F00C949141E0E07A
:10831E00E093F60FA091F50FAA3010F40C949A4149
:10832E00E6E0E093F60F0E9436AE043011F00C94A6
:10833E00AA410E944CAE113010F40C94AA410E9436
:10834E0056AD0E9451AE3AC0A091F60FA83011F072
:10835E000C94E541E091F80FE03011F00C94BA4125
:10836E00E6E0E093F60FE091F90FE03011F00C9497
:10837E00C341E7E0E093F60F0E94C437E03011F0FE
:10838E000C94CC41E0E0E093F60FA091F50FAA30EB
:10839E0010F40C94D541E6E0E093F60F0E9436AE51
:1083AE00043011F00C94E5410E944CAE113010F4E3
:1083BE000C94E5410E9456AD0E9451AEE1E00E9440
:1083CE00B4B9AD9608950E94ACB9AD01A8E5B0E080
:1083DE00EF81F8850E9468BBAAE5B0E0EE810E94AD
:1083EE0070BB00E010E00031E0E01E0710F00C94CE
:1083FE001742ACE5B0E0F8010E9458AE0F01F8014B
:10840E00DA010E945DAED0010E9468BB21E030E02F
:10841E00E02FD9010E94F0B99F010F5F1F4FE3CFEC
:10842E00A6E5B0E00E944EAD08950A930A2FA091E2
:10843E00F60FA63010F00C942742E0E00991089553
:10844E00003011F00C9430420E9443AEE0E00991EE
:10845E0008950E942DAEE1E00991089526971A9392
:10846E000A93A091F60FA63010F00C944342E1E06F
:10847E001981088128960895E091F80FE03011F0E7
:10848E000C944E42E2E01981088128960895A8E5E1
:10849E00B0E00E9450BB8F01002E012A11F00C9407
:1084AE006042E0E0E093F90FE3E01981088128963D
:1084BE000895E1E0E093F90F0E945BAD0E9461AE7A
:1084CE00DE0115960E94B238E0E0198108812896E7
:1084DE0008952697A091F60FA63010F00C947A42CC
:1084EE00E1E0269608950E9479AD0E9461AEDE010C
:1084FE0013960E94B238E0E0E093F90F26960895A5
:10850E00BA93AA930E947AA90034E0E01E0710F0F5
:10851E000C949742F8010E94B3A60F5F1F4FF4CF41
:10852E00A6E5B0E00E9454BBAE81BF81EC93E09112
:10853E00F60FAE81BF811196EC93A0E4B0E00E94DD
:10854E0082ADA2E4B0E00E9489ADAEE3B0E00E943D
:10855E009FADAFE3B0E00E94A6AD0031E0E01E0794
:10856E0010F00C94C642F80137960E94D3A70F0163
:10857E00E6E4F0E00E94AFAD0F5F1F4FEECFA8E52F
:10858E00B0E00E94B7ADAAE5B0E00E94C1ADE091A7
:10859E00F80FAE81BF815A96EC93E091F90F0E94CD
:1085AE00C8AD0031E0E01E0710F00C94EB42ACE5D4
:1085BE00B0E0F8010E9449AD0E94D1AD0E94D8AD45
:1085CE0040830F5F1F4FEDCFA4E4B0E00E9450BB7D
:1085DE000E9468AEAE81BF81DC96EC930E946EAEB7
:1085EE00AE81BF81DD96EC93E0E40E94B3B928968C
:1085FE000895E091F50F08950E94EEA6E091F50F13
:10860E00E03011F00C941E43AF85B889E0E0EC9396
:10861E00AD85BE85EFEF0E94DFADE0E0EC93AF815C
:10862E00B885EC93E1E00E94B3B961960895E091AC
:10863E00F50FE150E093F50F0E9473AEE952F04F43
:10864E00E081AF85B889EC930E9473AEE852F04F8B
:10865E00E081AB85BC85EC930E9473AEE752F04F80
:10866E00E081EE83AD85BE85EC93AE81A03110F036
:10867E000C946243ACE5B0E0F0E00E9449AD0E947C
:10868E00F7AD10F00C944D43980115C0A6E4B0E080
:10869E00EE81F0E0AE0FBF1F0E9454BB2E2F33278A
:1086AE00AEE3B0E00E9454BB4E2F5527FA01D9011C
:1086BE000E9466BA9F01A985BA852C93E32FF070AC
:1086CE00AF81B885EC930E9473AEE952F04FA0E0F3
:1086DE00A0830E9473AEE852F04FA0E0A0830E94E8
:1086EE0073AEE752F04FA0E0A083E0E00E94B3B972
:1086FE00619608950E9479AEA091F50FAA3010F4FC
:10870E000C948E43E1E00E94B6B9259608950E941E
:10871E0073AEE952F04F20830E9473AEE852F04FD1
:10872E0000830E9473AEE752F04F1083E091F50F75
:10873E00EF5FE093F50FE0E00E94B6B9259608953D
:10874E00BA93AA93A3970E94ACB910E02FEF30E032
:10875E0040E05BA50E947FAE0E9486AEE9A5FAA519
:10876E00FA93EA930E948AAEA52FBB270E94961A0F
:10877E0000E0E02F0E948FAEEC91EE83E07811F4D2
:10878E000C94D243EE81E0774E2F42954F70EE81DE
:10879E00EF702E2F2DC0EE81E07411F40C94F24385
:1087AE00EE81E07FE03711F00C94DF4313E00FC051
:1087BE00EE81E07FE03511F00C94E74312E007C044
:1087CE00EE81E07FE03411F00C94EE4311E0EE8187
:1087DE00EF702E2F0DC0EE81E07211F40C94F84361
:1087EE0007C0EE81E07111F40C94FE4301C03E818E
:1087FE000F5F051710F00C940E44103011F40C940A
:10880E000D44303011F40C940D4401C001C001C070
:10881E00B0CF1A932A93A32F0E948143E1E00E94C6
:10882E00B3B9AC9608950895E0E008950E9495AE10
:10883E000E947D13A1E00E94F725A0E00E9417265A
:10884E0008950E945CAA0E94A84B0E945CAA0E94F6
:10885E0096440E945CAAA5E00E94ED490E945CAA83
:10886E00A5E00E94014A0E945CAAEDE0EA93E4E0D2
:10887E00EA93A2E0B0E080E090E00E9499AEEDE0D5
:10888E00EA93E9E00E949CAEEEE0EA93E3E00E94F8
:10889E009CAEE2E1EA93E3E0EA93A6E9B0E080E081
:1088AE0090E00E94244AE6E9F0E0E0930910F0938C
:1088BE000A100E945CAAE2E1EA93E7E1EA93AEE1D4
:1088CE00B0E080E090E00E9499AEE2E1EA93E7E248
:1088DE00EA93A8EEB3E080E090E00E9499AEE2E168
:1088EE00EA93E8E2EA93A4E6B0E080E090E00E942A
:1088FE0099AEE8E0EA93AAE00E942E450E945CAA97
:10890E00A0E00E9481450E945CAAA0E00E946945F9
:10891E000E945CAAA4E6B0E00E943C4C08950E941E
:10892E00A2AE0E94ADAE0E94B3AEE1E4EC930E9403
:10893E00B8AEE0E00E94BBAEA2E0B0E00E940C1523
:10894E000881659608950E941D44A1E20E941C14A0
:10895E00A1E00E94332CA8ECB0E00E940A0E0E9407
:10896E005026E03011F40C94C0440E9428440E941A
:10897E0096440895A0E00E94332C089526970A93FA
:10898E000A2F033011F00C94DB44ADE00E941C144E
:10899E00AAE00E941C14AAE00E941C14AAE00E94E5
:1089AE001C14AAE00E941C14EBE1E983E3E4EA83C1
:1089BE00013011F40C94E844033011F40C94E844A3
:1089CE0003C0E0E0EB8306C0023011F00C94F144DA
:1089DE00E1E0EB83E0E0EC830E94C1AE0E94C6AE04
:1089EE0008812796089564970E94B5A90E94CAAE81
:1089FE000E94ADAE0E94EAA7E6E40E94D9AE0E94A4
:108A0E00DEAE2083E02FF0E00E94EAA7E0E0EC93D8
:108A1E000E94F9AB0E94E3AE089564970E94B5A937
:108A2E000E94CAAE0E94ADAE0E94EAA7ECE50E947B
:108A3E00D9AE0E94DEAE2083E02FF0E00E94EAA7BE
:108A4E00E0E0EC930E94F9AB0E94E3AE08956497C8
:108A5E000E94AFB91A2F2F8900E02F3110F40C9419
:108A6E00394520E0163010F40C944245153110F0C3
:108A7E000C94424501C01AE00E94EBAE0E94ADAECE
:108A8E000E94F3AEE0E5EC930E94EBAEEFEF0E9496
:108A9E00F8AEDE0113960E94FDAEDE0113960E9423
:108AAE0004AFF0E00E94F3AE0E9409AFA5E0B0E083
:108ABE000E940C152093FA0F1093FB0F0E94B6B96B
:108ACE00689608950E9410AF153010F40C947045FE
:108ADE0010E00E9416AF0E941EAFE7E50E94F8AEAE
:108AEE000E9423AF0E9429AF1093FC0F19810881B9
:108AFE00669608950E9410AF183010F40C948845B5
:108B0E0010E00E9416AF0E941EAFE8E40E94F8AE7D
:108B1E000E9423AF0E9429AF1093FD0F1981088187
:108B2E00669608950E9410AF0E9416AF0E941EAF67
:108B3E00E9E50E94F8AE0E9423AF0E9429AF109380
:108B4E00FE0F19810881669608950E9410AF1230AB
:108B5E0010F40C94B34510E00E9416AF0E941EAFA5
:108B6E00EAE40E94F8AE0E9423AF0E9429AF109350
:108B7E00FF0F19810881669608950E9410AF12307A
:108B8E0010F40C94CB4510E00E9416AF0E941EAF5D
:108B9E00ECE40E94F8AE0E9423AF0E9429AF10931E
:108BAE00001019810881669608950E9410AF123048
:108BBE0010F40C94E34510E00E9416AF0E941EAF15
:108BCE00E9E40E94F8AE0E9423AF0E9429AF1093F1
:108BDE00011019810881669608950E9410AF1C3607
:108BEE0011F40C940F46133611F40C940F461237F1
:108BFE0011F40C940F461C3411F40C940F461334DC
:108C0E0011F40C940F46123511F40C940F4601C05A
:108C1E0001C01CE60E9416AF0E941EAFE9E60E943C
:108C2E00F8AE0E9423AF0E9429AF10930210198153
:108C3E000881669608950E9410AF0E9416AF0E949A
:108C4E001EAFE3E20E94F8AE0E9423AF0E9429AF4E
:108C5E0019810881669608950E9410AF0E9416AF82
:108C6E000E941EAFEDE60E94F8AE0E9423AF0E9456
:108C7E0029AF1981088166960895AA93EF9769978F
:108C8E000E94ACB924E630E040E0FE01E25AFF4F0C
:108C9E005081FE01B8960E9432AF0E9486AE0E94AD
:108CAE000CAE5F3110F40C945D465EE100E00517EA
:108CBE0010F00C9473460E9437AFEA0FFB1F0E9410
:108CCE003CAFDB01EC93E02F0E9461A90E943CAF08
:108CDE00DB01EC930F5FEBCFDE01AE59BF4FAC91D2
:108CEE00A03011F00C9482460E9444AFA13011F0D6
:108CFE000C94824601C001C012E40E9449AFA0301C
:108D0E0011F00C9491460E9444AFA03011F00C94D7
:108D1E00914601C001C012E60E9449AFA13011F088
:108D2E000C94A0460E9444AFA13011F00C94A046C2
:108D3E0001C001C013E40E9449AFA13011F00C94A0
:108D4E00AF460E9444AFA03011F00C94AF4601C064
:108D5E0001C013E60E9449AFA23011F00C94BE463A
:108D6E000E9444AFA13011F00C94BE4601C001C068
:108D7E0014E40E9449AFA23011F00C94CD460E942B
:108D8E0044AFA03011F00C94CD4601C001C014E6E2
:108D9E000E9449AFA33011F00C94DC460E9444AF00
:108DAE00A13011F00C94DC4601C001C019E40E9400
:108DBE0049AFA33011F00C94EB460E9444AFA030A3
:108DCE0011F00C94EB4601C001C019E60E9449AFA8
:108DDE00A43011F00C94FA460E9444AFA13011F069
:108DEE000C94FA4601C001C015E50E9449AFA430AB
:108DFE0011F00C9409470E9444AFA03011F00C946E
:108E0E00094701C001C015E70E9449AFA53011F016
:108E1E000C9418470E9444AFA13011F00C941847DF
:108E2E0001C001C016E50E9449AFA53011F00C94A7
:108E3E0027470E9444AFA03011F00C94274701C081
:108E4E0001C016E7123411F40C943247123611F4A5
:108E5E000C9432471DC000E0051710F00C944047EB
:108E6E000E944EAF0F010E9437AF0E94BFA70F5F47
:108E7E00F3CFEAE2EE830E9451AFEAE2EC93E52FE4
:108E8E00EE5FF0E00E947BA7E0E0EC935E5FB6C081
:108E9E00133411F40C945847133611F40C945847AC
:108EAE000CC0E52FF0E00E947BA7EFEFEC930E9441
:108EBE0051AFE0E0EC935F5FA1C0143411F40C9459
:108ECE006D47143611F40C946D471DC00E940CAE04
:108EDE000E9455AF0E945CAF5CE000E0051710F0F9
:108EEE000C9489470E9437AF0E9460AF11F40C9426
:108EFE0087470E944EAF0F010E9437AF0E94BFA757
:108F0E000F5FECCF7BC0193411F40C9493471936D4
:108F1E0011F40C9493472CC00E9455AF0E9463AF7E
:108F2E0000E0051710F00C94AC470E9437AF0E947A
:108F3E0060AF11F40C94AA470E944EAF0F010E942D
:108F4E0037AF0E94BFA70F5FECCFE0E0EE835F5F0D
:108F5E0050FF08C0E52FF0E00E947BA7EFEFEC93E7
:108F6E005F5F05C00E9451AFEFEFEC935E5F46C0AE
:108F7E00153511F40C94C847153711F40C94C847E5
:108F8E0016C00E940CAE0E9455AF0E945CAF00E06E
:108F9E00051710F00C94DC470E944EAF0F010E9493
:108FAE0037AF0E94BFA70F5FF3CF5CE027C0163527
:108FBE0011F40C94E747163711F40C94E7471EC0D2
:108FCE000E940CAE0E9455AFA7E0B0E00E94831B3A
:108FDE0057E000E0051710F00C9405480E9437AFDB
:108FEE000E9460AF11F40C9403480E944EAF0F0123
:108FFE000E9437AF0E94BFA70F5FECCF0E9467AFF2
:10900E000E946CAF0E94ADAE0E946CAFE3E60E9470
:10901E00F8AEDE01A65BBF4F0E9404AF0F5FF0E01B
:10902E00DE01A65BBF4F0E94FDAEDE01A65BBF4F09
:10903E000E9472AFDE01A65BBF4FEA0FFB1F40839B
:10904E00E02FF0E00E946CAFE0E0EC93FE01E65BF7
:10905E00FF4FFA93EA93A6E0B0E00E940C150E942F
:10906E0079AFA52FBB270E947EAFEF96A4960895E9
:10907E000E94D9A50839E0E01E0714F00C944E4862
:10908E00ABE0B0E10E946FA60F5F1F4FF3CFE0E0A1
:10909E00E093A310E093A410099119910895BA9347
:1090AE00AA930E94ACB9AE81BF810E94A3199F0101
:1090BE002134E0E03E0714F40C94674820E430E0DD
:1090CE00E885E03011F00C94814800E010E00034A7
:1090DE00E0E01E0714F00C947C48F801E55FFF4EAB
:1090EE000E9483AF0F5F1F4FF2CF2093A3103093D8
:1090FE00A4104AC0A885A13011F00C949E4800E03F
:10910E0010E00034E0E01E0714F00C949648F801CD
:10911E00E55BFF4E0E9483AF0F5F1F4FF2CFF90149
:10912E00E05CFF4FE093A310F093A4102DC0A88530
:10913E00A23011F00C94CB4848E150E04134E0E00D
:10914E005E0710F40C94AD4840E450E000E010E0EF
:10915E000417150710F00C94BC48F801E557FF4EA4
:10916E000E9483AF0F5F1F4FF3CFF901E058FF4FFF
:10917E00E093A310F093A41047E950E0ABE0B0E108
:10918E00A40FB51FE0E0EC930E94B3B929960895A1
:10919E00BA93AA9368970E94ACB900E011E720E059
:1091AE003CE445E050E0EE8DFF8DEE83FF83EE81D3
:1091BE00E887EF81F070EE83FF83EE81E9870E94EE
:1091CE0088AFAE0FBF1F0E94ADAE0E948EAFE3E61A
:1091DE000E94F8AEDE011A960E9404AF0F5FF0E017
:1091EE00DE011A960E94FDAEDE011A960E9472AF43
:1091FE00DE011A96EA0FFB1F40830E9488AFEA0F2A
:10920E00FB1F50830E9488AFEA0FFB1FA985A08326
:10921E000E9488AFEA0FFB1FA885A083E02FF0E025
:10922E000E948EAFE0E0EC930E9493AFA9E0B0E015
:10923E000E947EAFA0960895A091A310B091A410A5
:10924E000E94CF48EBE0F0E1FA93EA93A091A310CD
:10925E00B091A4100E940C1508950E946FA9D80118
:10926E000E94CF480E9498AF0E94B5B926960895E5
:10927E0064970E945DA500E00E94EBAE0E94ADAE29
:10928E000E94F3AEE3E6EC930E94EBAEEDEFEC93AF
:10929E00012E022A11F00C945C49E02F0F5FF0E0D2
:1092AE00DE0113960E9449A704C00E94EBAEE1E3D3
:1092BE00EC930E949DAF0E9409AFA4E0B0E00E9423
:1092CE000C150E94B6B96796089564970E945DA525
:1092DE0000E00E94EBAEECE0EC930E949DAF0E948A
:1092EE0009AFA1E0B0E00E940C150E94B6B96796D6
:1092FE0008951A930A931A2F00E0011710F00C9498
:10930E008D49AAE00E941C140F5FF7CF09911991A5
:10931E0008950E946FA90E9498AFAAE00E941C14A3
:10932E000E94B5B9269608950E94AEB99D010E947D
:10933E00A3198F010E9498AFAAE00E941C140E94EC
:10934E00B5B9249608950E9444BB0E9435BB0E9475
:10935E003F1524960895EF97EF9724970A9300E010
:10936E00023810F00C94C1490E94B8AEE0E0EC93C4
:10937E000F5FF6CF00E0013610F00C94CD490E943D
:10938E00B8AEE02FE05EEC930F5FF5CF0E94C1AE5A
:10939E00A0E6B0E00E940C1500E0003810F00C942E
:1093AE00DF490E94B8AEE02FE058EC930F5FF5CF87
:1093BE000E94C1AEA0E8B0E00E940C15AAE00E9487
:1093CE001C140881EF96EF9625960895AA930A939A
:1093DE00E981EE0FEE0FEE0F0E2FE1E1EA93E4E0DE
:1093EE00EA93A02FBB27882799270E94244A088139
:1093FE0022960895AA932497E0ECE883E1E0E983AE
:10940E000E94E7AC0A93ED81EE0FEE0FEE0F0E2FDA
:10941E000E94A0AF0E94CDB9A983BA838B839C838F
:10942E00E1E1EA93E5E0EA93AB81BC818D819E8117
:10943E000E94244A0881269608950E9444BBAF9745
:10944E00E0E0E883E9830E94E7AC0E94ACB900E05B
:10945E0020E0EDA9FEA96FA978AD0E94A8AFADA935
:10946E00BEA98FA998ADA935EEE3BE07EFE08E0732
:10947E00E0E09E0710F40C94494AE1E00E94B3B973
:10948E00EB9608951AADA12FE4E60E949EBA3E2FE8
:10949E000E94ADAF4E2F0E948AA85E2F305D405DB8
:1094AE00505D19ADA12FE4E60E949EBAEE8B0E948C
:1094BE00ADAFED8B0E948AA8EC8BEE89E05DEE8B52
:1094CE00ED89E05DED8BEC89E05DEC8B0E9403A9EC
:1094DE000E94ACA50E94C4BAEB8B0E9403A90E9405
:1094EE00ACA50E94B3AFE0E1F7E260E070E00E944D
:1094FE00C4BAEA8B0E94BCAFE0E1F7E260E070E034
:10950E000E94C1AFE8EEF3E060E070E00E94C4BAE2
:10951E00E98B0E9403A9E8EEF3E060E070E00E94A0
:10952E00B3AFE4E6F0E060E070E00E94C4BAE88B0E
:10953E000E94BCAFE4E6F0E060E070E00E94C1AFD4
:10954E000E94C6AF0E94C4BAEF870E9403A90E9470
:10955E00CBAFEE87EB89E05DEB8BEA89E05DEA8BC2
:10956E00E989E05DE98BE889E05DE88BEF85E05DF8
:10957E00EF87EE85E05DEE870E94D0AFAE0FBF1F86
:10958E00EEE10E94F8AE0E94D6AFEBE50E94F8AE77
:10959E000E94D6AFE2E30E94F8AE0E94D6AFEAE395
:1095AE00EC93313310F40C94E14A0E94D0AFEA0FE1
:1095BE00FB1F3083413310F00C94EA4A313310F024
:1095CE000C94EA4A05C00E94D0AFEA0FFB1F4083FD
:1095DE000E94D0AFEA0FFB1F50830E94D0AF0E94B3
:1095EE0044A7AE89A13310F40C94034B0E94D0AF64
:1095FE00EA0FFB1FAE89A083AD89A13310F00C9446
:10960E000E4BAE89A13310F00C940E4B06C00E9487
:10961E00D0AFEA0FFB1FAD89A0830E94D0AFEA0F37
:10962E00FB1FAC89A0830E94D0AFAE0FBF1FEAE331
:10963E00EC93AB89A13310F40C942B4B0E94D0AF5A
:10964E00EA0FFB1FAB89A083AA89A13310F00C94FB
:10965E00364BAB89A13310F00C94364B06C00E94EA
:10966E00D0AFEA0FFB1FAA89A083A989A13310F0FE
:10967E000C944C4BAA89A13310F00C944C4BAB8933
:10968E00A13310F00C944C4B06C00E94D0AFEA0FE1
:10969E00FB1FA989A083A889A13310F00C94674BF6
:1096AE00A989A13310F00C94674BAA89A13310F04D
:1096BE000C94674BAB89A13310F00C94674B06C02A
:1096CE000E94D0AFEA0FFB1FA889A083AF85A133FC
:1096DE0010F00C94874BA889A13310F00C94874B93
:1096EE00A989A13310F00C94874BAA89A13310F0ED
:1096FE000C94874BAB89A13310F00C94874B06C0AA
:10970E000E94D0AFEA0FFB1FAF85A0830E94D0AF9F
:10971E00EA0FFB1FAE85A0830E94D0AFAE0FBF1F16
:10972E00EDE5EC93E02FF0E00E94D6AFE0E0EC9395
:10973E00FE0177960E94DBAFE0E00E94B3B9EB9694
:10974E0008950E94A2AEEEE10E94F8AE0E94B3AE62
:10975E00EBE50E94F8AE0E94B3AEE6E30E94F8AECF
:10976E000E94B3AEEAE30E94F8AE0E94E1AF0E94FF
:10977E00E5AFE02F0F5FF0E00E94E1AF0E94ECAF8B
:10978E00EAE30E94F8AE0E94E1AF0E94ECAFEDE575
:10979E000E94BBAEA02FBB270E940C150E9467AF84
:1097AE000E94B3AEEEE10E94F8AE0E94B3AEEBE5BE
:1097BE000E94F8AE0E94B3AEE9E30E94F8AE0E949A
:1097CE00B3AEEAE30E94F8AE0E94E1AF0E94E5AFAD
:1097DE00E02F0F5FF0E00E94E1AF0E94ECAFEAE3F2
:1097EE000E94F8AE0E94E1AF0E94ECAFEDE50E9440
:1097FE00BBAEA02FBB270E940C150881659608955D
:10980E0064970E94ACB92A2F3A8D4B8D5C8D00E087
:10981E0015E0E02F0F5FF0E00E947BA7EBE1EC93E9
:10982E000E94F0AF50830E94F0AF40830E94F0AFD1
:10983E0030830E94F0AF2083403011F00C94294CFD
:10984E0012E00BC0303011F00C942F4C13E005C019
:10985E00203011F00C94344C14E00E9479AFA12FFB
:10986E00BB270E947EAF6D9608951A930A938D01C1
:10987E000530E0E01E0710F40C944C4C0B3FE0E07A
:10988E001E0710F00C944C4C01C00DC0E2E1EA939F
:10989E00E3E0EA93D801882799270E94244A00938F
:1098AE00091010930A100991199108956C970E944E
:1098BE00ACB900E030E010E00E942914E0E0E09343
:1098CE0008100E9467AF0E94F3AF0E94ADAE0E94D7
:1098DE00F3AFEBE6EC93E02FF0E00E94F3AFE0E0A5
:1098EE00EC93FE013E960E94DBAFADE00E94820E2D
:1098FE0000E00E94FE140E2FADE00E94990EAF0103
:10990E00003011F00C94924C4436E0E05E0710F0FB
:10991E000C94924C01C001C0ECCF003011F00C94AD
:10992E009F4CE0E4E09308100E94B3B9A29608950C
:10993E000E94AA140E94FEA8199714F40C94AB4C22
:10994E00A4EFB1E00E940A0EAE81BF81119714F40C
:10995E000C94B84CAE81BF81199714F00C94B84C8E
:10996E0006C01F5F1E3110F00C94BE4C01C001C02A
:10997E00A3CFAE81BF81119714F00C94CF4C0E94EF
:10998E002914E0E8E09308100E94B3B9A296089556
:10999E00FE013E960E9432AF0E94F8AFFE013E9647
:1099AE00FA93EA93A4E1B0E00E94CF1400E00630EF
:1099BE0010F00C94EA4CE02FF0E0DE0118960E94B5
:1099CE00FCAF0F5FF4CFAE81BF81169714F40C94E9
:1099DE00F44CE5E0F0E0EE83FF8300E0EE81FF81E2
:1099EE00A02FB0E0AE17BF0714F00C94314DE02F4E
:1099FE00F0E00E94F3AF2C91E22FE07F1E2F17FFB5
:109A0E0003C016FD01C001C004C0E22FEF73E8874A
:109A1E001FC0103C11F00C94184DE22FEF70E98727
:109A2E0017C0103D11F00C94204DE22FEF70EA8715
:109A3E000FC0103E11F00C94284DE22FEF70EB8703
:109A4E0007C0103F11F00C942F4DE22FEF70EC87F2
:109A5E000F5FC4CF00E0053010F00C94434DA3E02F
:109A6E00B0E1E02F0E946AA9E12FF0E0DE01189626
:109A7E000E94BFA70F5FEFCF388530FF02C03E7F39
:109A8E0001C03160E32F0E94B3B9A29608950E94DF
:109A9E005DA500E00E9401B0A0910310A0830E947A
:109AAE0001B0A0910410A0830E9401B0A0910510F6
:109ABE00A0830E9401B0A0910610A0830E9401B065
:109ACE00A0910710A0830E9401B0A0910810A0835E
:109ADE000E9462A508950E94ACB9AD0100E00E94FB
:109AEE0007B0A091FA0FA0830E9407B0A091FB0FC0
:109AFE00A0830E9407B0A091FD0FA0830E9407B023
:109B0E00A091FC0FA0830E9407B0A091FF0FA0832D
:109B1E000E9407B0A0910110A0830E9407B0A091EF
:109B2E000010A0830E9407B0A091FE0FA083209189
:109B3E00091030910A10122F232F33270E9407B0DD
:109B4E0020830E9407B010830E9407B0A0910210DC
:109B5E00A083E02F0E94B3B926960895A1E00E943B
:109B6E00EE4FE0E0E093A81008950895BA93AA93FB
:109B7E00A0970E94ACB9E0E0EE83AE81A73010F062
:109B8E000C94D34DEE81AEA1BFA1F0E00E94FCAFCC
:109B9E00EE81EF5FEE83F1CFE0E0EE83AE81AA308F
:109BAE0010F00C94E34DEE810E948FAEE0E0EC934A
:109BBE00EE81EF5FEE83F2CF0E940DB0E8E00E94DF
:109BCE0012B0DE0157960E9452112E2F213010F442
:109BDE000C94F44D0E9418B00895EA89E07811F0C3
:109BEE000C940C4EEA89EA8FE068EA8F0E940DB061
:109BFE00E1E00E9412B00E941DB010F40C940A4EC7
:109C0E000E9418B008950E942BABED89E07211F0FE
:109C1E000C94134EED89ED8FED89E07111F40C94D7
:109C2E002A4EED89ED8FDE015D96EC91EF7E0E945E
:109C3E0024B00E941DB010F40C94284E0E9418B04F
:109C4E0008950E942BABED89E87011F00C94414EF3
:109C5E00ED89ED8FDE015D96EC91E8600E9424B0F7
:109C6E000E941DB010F40C943F4E0E9418B008953F
:109C7E000E942BABEC89E07411F40C94584EEC89D5
:109C8E00EA8FEF7BEA8FE2E0F0E00E942BB00E94B9
:109C9E001DB010F40C94564E0E9418B008950E94F8
:109CAE002BABEA89E093A510EB89E093A610EC8923
:109CBE00E093A710ED89E093A810E7703E2F3130A6
:109CCE0010F40C946F4E383010F00C946F4E01C09F
:109CDE0001C03F83ED89E093A810EC89EF730E94D9
:109CEE002FB02E2F0B89A02F0E94FD1F1E2F1C336D
:109CFE0010F00C94854EFE0138961083EA89EF77AA
:109D0E000E942FB01E2F1C3310F00C94914EFE01AA
:109D1E0039961083283110F00C94984EFE013A9625
:109D2E002083EF89EF710E942FB05E2FEE89EF73C3
:109D3E000E942FB0E98BA88D0E94FD1F4E2FFE01B1
:109D4E003B964083FE013C965083E989ED87AB85B7
:109D5E00A43610F40C94B84EE2E00E94B3B9A89663
:109D6E000895AC85AD3010F00C94C24EA03011F4B5
:109D7E000C94C24E05C0E3E00E94B3B9A8960895B4
:109D8E00AD85A03210F00C94D14EA03011F40C948D
:109D9E00D14E05C0E4E00E94B3B9A8960895AA85F5
:109DAE00A83110F40C94E04EE5E00E94B3B9A896E9
:109DBE000895A885AC3310F40C94EA4EE6E00E94A8
:109DCE00B3B9A8960895AF81A83010F40C94F44E50
:109DDE00E7E00E94B3B9A8960895E0E0EE83AE8165
:109DEE00A73010F00C940A4FEE81AEA1BFA10E94D5
:109DFE006AA9EE81F0E0DE0117960E94BFA7EE8100
:109E0E00EF5FEE83ECCFE0E00E94B3B9A896089521
:109E1E0029970E94ACB92A2F3F8548895989583114
:109E2E0011F00C941B4F50E0583110F40C94224F4B
:109E3E000E9433B008954C3311F00C94274F40E03C
:109E4E004C3310F40C942E4F0E9433B008953C33D3
:109E5E0010F40C94334F30E0E091A810E862E093D8
:109E6E00A810EF7EE093A810E32FE068EE83E09158
:109E7E00A610EF83E091A710E887E091A810E9877C
:109E8E00E0E0EA87EB87EC87ED87503011F00C9419
:109E9E00554F403011F00C94554F09C0583110F009
:109EAE000C945E4F4C3310F00C945E4F01C00CC0FE
:109EBE00A32F0E940E20EE83A42F0E940E20EF836C
:109ECE00A52F0E940E20E887213010F40C94744FB9
:109EDE00283010F00C94744F01C007C01091A810D8
:109EEE00187F122BFE0139961083EE81E068EE8307
:109EFE00DE011996EC91E862EC930E940DB0E4E05D
:109F0E000E9412B0DE011B960E9482100E2F0E943C
:109F1E005CAA003011F40C94974F0E9433B0089550
:109F2E00E0E00E94B3B96296089524970E94AEB9FC
:109F3E001A2F28853985203011F40C94AB4F2D3013
:109F4E0010F00C94AB4F03C00E9438B0089510303F
:109F5E0011F40C94B74F103210F00C94B74F03C09D
:109F6E000E9438B00895343110F40C94C34F33333B
:109F7E0010F00C94C34F01C037E1A12F0E940E20A8
:109F8E00EC83A22F0E940E20ED83A32F0E940E20A1
:109F9E00EE83E0E0EF830E943DB0E4E0F0E0FA9360
:109FAE00EA93E3E00E9412B0DE0119960E9482103D
:109FBE000E2F0E943DB0003011F40C94E94F0E9418
:109FCE0038B00895E0E00E94B5B92A960895229718
:109FDE000E94AFB92A2F022FE02FE03011F00C941F
:109FEE00FB4FE0E0EB830DC0E13011F00C9402501A
:109FFE00E0E4EB8306C0E23011F00C940850E4E488
:10A00E00EB83E0E0EC83E7E0F0E00E942BB0DE01B2
:10A01E0018960E9482101E2F103011F40C941C50B2
:10A02E00E1E00E94B6B925960895E0E00E94B6B927
:10A03E002596089522970A93E7E0F0E00E942BB050
:10A04E00DE0116960E9452110E2F003011F00C9464
:10A05E003450E981088123960895EFEF0881239605
:10A06E0008950881239608952C970E94AEB99D01FC
:10A07E00FE0134960E9432AFACE00E94FEABE0E3EC
:10A08E00EA930E9441B00E9445B0DE0119960E94EB
:10A09E0050B010F40C945850E1E00E94B5B960969F
:10A0AE00089510E0183010F00C9466500E9455B0D0
:10A0BE00F0E0DE0114960E94BFA71F5FF3CFE0E031
:10A0CE000E94B5B96096089568970E94ACB99D013B
:10A0DE004E8D5F8D05C0E2E00E94B3B9A096089543
:10A0EE00FE0172960E9432AF0E945CAF5A934A9361
:10A0FE00E0E3EA93A0E10E94FEABE0E3EA930E9464
:10A10E00F8AF0E9445B0DE0157960E9450B010F491
:10A11E000C949650E1E00E94B3B9A0960895E98D93
:10A12E000E945CB0DA011F96EC93EE85DA011E9662
:10A13E00EC93E88D0E945CB0DA011D96EC93EE85EF
:10A14E00DA011C96EC93EF890E945CB0DA011B9643
:10A15E00EC93EE85DA011A96EC93EE890E945CB0D0
:10A16E00DA011996EC93EE85DA011896EC93ED89E7
:10A17E000E945CB0DA011796EC93EE85DA01169622
:10A18E00EC93EC890E945CB0DA011596EC93EE85A7
:10A19E00DA011496EC93EB890E945CB0DA01139607
:10A1AE00EC93EE85DA011296EC93EA890E945CB08C
:10A1BE00DA011196EC93EE85DA01EC93EE89FF2726
:10A1CE00662777270E9467B0EF890E946FB0E88DEF
:10A1DE000E946FB0E98DFF27662777270E9403A99B
:10A1EE000E94D2B90E94A8AFEA89FF276627772777
:10A1FE000E9477B0EB890E9480B0EC890E9480B0FB
:10A20E00ED89FF27662777270E94BCAF0E94D2B93F
:10A21E000E9436A80E9446A83A932A930E9488B0BC
:10A22E000E940DA90E943FBBFE017696FA93EA9317
:10A23E000E9488B013E11A3010F40C9430510E9431
:10A24E0055B0EA50F0E0DE0152960E94BFA71150C1
:10A25E00F2CF10E0143110F00C9442510E945CA623
:10A26E00EC91E03011F00C9440510E945CA6E0E3BA
:10A27E00EC931F5FEFCFE0E00E94B3B9A096089574
:10A28E002E970A93DE0115960E94BD4D0E2F0030BB
:10A29E0011F40C94555108812F960895E885E0939A
:10A2AE00690EEE81E0936A0EEF81E0936B0EE98505
:10A2BE00E093650EEA85E093660EEB85E093670EFC
:10A2CE00ED81E093680EACE6BEE0E091690EF0E041
:10A2DE00ED93FC93A0916C0EB0916D0EECE30E9489
:10A2EE008EBAE0936C0EF0936D0EA0916C0EB09141
:10A2FE006D0EE0916A0EF0E0EA0FFB1FE0936C0E1C
:10A30E00F0936D0EE0916C0EF0916D0E662777272F
:10A31E000E9491B00E9494A90E94B1A5E0916B0E8B
:10A32E000E94A0AF0E94C8B90E9491B0E0936E0E39
:10A33E00F0936F0E6093700E7093710EE0E00881D3
:10A34E002F960895E0E0E093A91008950E9495B02D
:10A35E00F901DA01ED93FC93DA0112960E949AACA0
:10A36E00DA0114960E949AACDA0116960E949AAC03
:10A37E00DA01ED91FD91DA011896ED93FC93E091DF
:10A38E00A910EF5FE093A910DA011A96EC9300E0A2
:10A39E0010E0DA010E942CBB0E171F0710F00C9470
:10A3AE00E151FA013B96E00FF11FAEE2A0830F5F81
:10A3BE001F4FEFCF0E94B3B9289608951A930A93B0
:10A3CE00E3E0EA93A3E0B0E00E94470BA1E00E9415
:10A3DE007925A8E0B0E00E9415BDE1E0E093AB1056
:10A3EE00E0E0E093AA100E949BB000E0053010F070
:10A3FE000C94165210E0123010F00C941452AAE085
:10A40E001A9FF001E055FF4EDF01E02FF0E00E94B1
:10A41E0049AD0E949AAC1F5FEECF0F5FE7CFEAE027
:10A42E00F0E0E093AC10F093AD10A091AC10B091B1
:10A43E00AD10E2E00E948EBAE093AC10F093AD1036
:10A44E00E0E0E093AE10E093AF10099119910895FA
:10A45E000E94A2B011F40C9437520E94A7B0089536
:10A46E000E948525E03011F00C944352A1E00E9429
:10A47E007925A3E00E94820EA3E00E94990E8F011F
:10A48E000630E0E01E0710F40C9487520E94AC0BCD
:10A49E009F0144E0413010F40C946A520E94ACB01B
:10A4AE00DF01E42FF0E00E9458AEBF010E94ACB075
:10A4BE00DF01E42FE150F0E00E945DAEDB01ED9391
:10A4CE00FC934150E7CF0E94ACB020833183E091E2
:10A4DE00AA10EF5FE093AA10A091AA10A23010F478
:10A4EE000C947C52E0E0E093AA100E949BB00E9474
:10A4FE00B4B010F40C948752AEEAB0E10E947FA57E
:10A50E000E94A7B008950E94AFB90E948525E03041
:10A51E0011F00C9494520E94BFB00E94B4B010F48B
:10A52E000C949F52E0EEFEE20E94B6B92396089577
:10A53E0000E010E020E0253010F00C94B052AAEBB1
:10A54E00B0E1E22FF0E00E9449AD0E949FAC2F5F78
:10A55E00F2CF0E94C6B00E94CDB00E94B6B923962B
:10A56E0008950E94ADB90E948525E03011F00C943B
:10A57E00C2520E94BFB00E94B4B010F40C94CD52DF
:10A58E00ECE8F0E00E94B4B92596089500E010E0E2
:10A59E0040E0453010F00C94DE52E42FA0EBB0E119
:10A5AE00F0E00E9449AD0E949FAC4F5FF2CF0E9437
:10A5BE00C6B0D8010E9425869F010E94B4B9259687
:10A5CE0008950E94AEB93A2F323010F40C94F55221
:10A5DE00E0E0F0E00E94B5B92496089500E010E0A6
:10A5EE0020E0253010F00C940A53AAE03A9FF001B7
:10A5FE00E055FF4EDF01E22FF0E00E9449AD0E94D0
:10A60E009FAC2F5FEECF0E94C6B0F8010E94B5B985
:10A61E00249608950E94AEB9A1E00E947925A0E08B
:10A62E000E94DDB0D8010E9425869F010E94B5B917
:10A63E00249608951A930A93A1E00E947925A1E029
:10A64E000E94DDB00E94CDB00991199108951A9320
:10A65E000A9310E00E94358BE03011F40C943C53B9
:10A66E00A6ECB1E10E94128B1E2FA091D311AF5F09
:10A67E00A093D311A53010F40C944853E0E0E0936E
:10A68E00D311E091D311F0E0E253FE4EFF93EF931E
:10A69E000E94BF64AF91BF91EC93EEECF1E1FA939F
:10A6AE00EA93A5E00E947B230E2F0E940D65E030F9
:10A6BE0011F40C947F53E0E0E093D411113011F4B7
:10A6CE000C946E53123011F40C946E530DC00E9404
:10A6DE0006650E94548B003011F40C947B53E1E01C
:10A6EE00E093C411E093C511E1E009911991089529
:10A6FE00113011F00C948753A1E00E94106507C031
:10A70E00123011F00C948E53A0E00E9410650030B0
:10A71E0011F40C949953E02FE853E093CF0F0E945D
:10A72E002B6508C0E1E0E093CF0FE0E0E093C411A9
:10A73E00E093D411E02FE57011F40C94AD53A09179
:10A74E00C411A03011F00C94AD5301C010C0E1E063
:10A75E00E093C4110E94E664113011F40C94BA53C4
:10A76E000E94F06402C00E9406650E94548B01FF95
:10A77E0007C0A091C511A03011F00C94C75301C0B1
:10A78E0013C0E1E0E093C5110E94E664123011F4AB
:10A79E000C94D4530E94F06405C00E940665E1E05B
:10A7AE00E093D4110E94548BE02FE57011F40C94B9
:10A7BE00E553113011F00C94E55301C002C00E9414
:10A7CE00066501FF05C0123011F00C94EF5301C065
:10A7DE0002C00E940665003011F00C940054113036
:10A7EE0011F40C94FF53123011F40C94FF5301C06A
:10A7FE0001C002C00E940665A091D411A13011F0D3
:10A80E000C940C5401FF01C001C020C00E943D6495
:10A81E00E03011F40C941654E1E0E093D5110E944F
:10A82E003D64E03011F00C942354E091D511E030EA
:10A83E0011F40C94235401C008C0E0E0E093D5114C
:10A84E00E091D411EF5FE093D4110BC0A091D4111D
:10A85E00A23011F00C943854E091D411EF5FE093D4
:10A86E00D411013010F40C944054E1E00991199187
:10A87E000895E0E0099119910895AA93EF97219711
:10A88E000E94ACB9DE01AA5BBF4FAC91E4E1EA9F36
:10A89E0090010E94E7B00E94EAB040E050E04431DF
:10A8AE00E0E05E0710F00C946954FA01E20FF31F1A
:10A8BE008F010E94EEB0DE0119960E9446844F5F12
:10A8CE005F4FEDCF0E94B3B9EF9628960895BA93D5
:10A8DE00AA930E94ACB9588500E010E039854885EE
:10A8EE00303110F40C947E540E94F3B0089544312C
:10A8FE0010F40C9485540E94F3B00895E4E1E39FA4
:10A90E008001E42FF0E00E0F1F1F0E94EEB0A9850C
:10A91E00BA850E9446842E2F203011F40C949A543E
:10A92E000E94F3B008950E9455A70895EF97E997F6
:10A93E000E94ACB920E030E0E0E0E0932017E09315
:10A94E0021170E943755AF014130E5E05E0710F444
:10A95E000C94B35440E055E0FE01E659FF4F0E94BF
:10A96E00F8B00E94E7B00E94FBB0E0912017F09182
:10A97E002117EA5EFD4E0081003210F00C94D05487
:10A98E000A3011F40C94D0540D3011F40C94D054B0
:10A99E001CC0F9012F5F3F4FDE011696EA0FFB1F19
:10A9AE0000832336E0E03E0710F40C94E7540E9437
:10A9BE0079AFD9010E9490490E94E7B00E94FBB086
:10A9CE00A0E2B7E10E947FA53CC00B3111F00C94C0
:10A9DE0024550E9479AFD9010E9490490E94E7B098
:10A9EE000E94FBB010E0183010F00C941555E12FBA
:10A9FE00F0E0DE01AC58BF4FEA0FFB1F0F01E12F55
:10AA0E00A0912017B0912117F0E0EA0FFB1FEA5E2C
:10AA1E00FD4EE081D001EC931F5FE5CFDE01AC5817
:10AA2E00BF4F0E946255E0912017F0912117389682
:10AA3E00E0932017F093211704C0A0E2B7E10E9423
:10AA4E007FA5A0912017B09121174A175B0710F42C
:10AA5E000C9432558ACF0E94B3B9EF96EF960895B3
:10AA6E001A930A930FEF14E0A6E1B2E1A00FB11F03
:10AA7E00AC91A13010F40C944E55A6E1B2E1A00FAA
:10AA8E00B11FAC91AF3F10F00C944E5501C005C0F4
:10AA9E00F8013A96099119910895015010400B3022
:10AAAE00E0E01E0710F40C945D55DECFEAE0F0E016
:10AABE00099119910895BA93AA9365970E94ACB91A
:10AACE00AB8DBC8DAC91AB3111F40C947355E1E0B0
:10AADE000E94B3B96D960895AB8DBC8D11960C91F5
:10AAEE00AB8DBC8D12961C91AB8DBC8D13962C919B
:10AAFE00AB8DBC8D14963C91AB8DBC8D17964C9145
:10AB0E00E02FE23311F00C94B355E12FEA3011F03F
:10AB1E000C94A355313011F00C949A55A22FBB27EB
:10AB2E000E94FA4408C0323011F00C94A255A22FA4
:10AB3E00BB270E9414450FC0EB3011F00C94AB559F
:10AB4E00A22F0E94C54407C0EC3011F00C94B255F0
:10AB5E00A22F0E94804983C1E33311F00C94525608
:10AB6E00E12FEA3011F00C94DD5520932217A091BD
:10AB7E002217A73110F00C94C955A03011F40C9483
:10AB8E00C95503C0E8E0E0932217A0912317A63021
:10AB9E0010F40C94D755A53110F00C94D75503C072
:10ABAE00ECE0E09323170E9402B174C0EB3011F079
:10ABBE000C94025620932317A0912217A73110F060
:10ABCE000C94EE55A03011F40C94EE5503C0E8E051
:10ABDE00E0932217A0912317A63010F40C94FC5585
:10ABEE00A53110F00C94FC5503C0ECE0E093231754
:10ABFE000E9402B14FC0EC3011F00C9412562E830D
:10AC0E00AE81A53010F40C940E56E1E0EE83AE81C9
:10AC1E000E9469453FC0ED3011F00C9422562E83F0
:10AC2E00AE81A83010F40C941E56E1E0EE83AE8196
:10AC3E000E9481452FC0EE3011F00C9432562E83B7
:10AC4E00AE81A23010F40C942E56E0E0EE83AE816D
:10AC5E000E94AC451FC0EF3011F00C9442562E836B
:10AC6E00AE81A23010F40C943E56E0E0EE83AE813D
:10AC7E000E94DC450FC0E03111F00C9451562E832A
:10AC8E00AE81A23010F40C944E56E0E0EE83AE810D
:10AC9E000E94C445E4C0E43311F00C949556E12FA4
:10ACAE00EA3011F00C9483560E947FAE0E94F8AFEA
:10ACBE0050E0583010F00C946A560E9409B10E9470
:10ACCE0011B15F5FF6CF50E0583010F00C947B5608
:10ACDE00E52FE85FF0E0DE011796EA0FFB1F0F018C
:10ACEE000E941AB15F5FF0CF2A933A930E948AAE08
:10ACFE00A42F0E94444611C0EB3011F00C948A56DA
:10AD0E000E9423490AC0EC3011F00C949456A32FE4
:10AD1E000E943346A22F0E942246A1C0E53311F0B5
:10AD2E000C943657E12FEA3011F00C9436570E94EE
:10AD3E007FAE0E94F8AF213011F00C94B75650E060
:10AD4E00583010F00C94B656E52F0E948FAEE52FBA
:10AD5E00F0E0EA52FE4EE081EC935F5FF1CF79C0F6
:10AD6E00223011F00C94C95650E0583010F00C946B
:10AD7E00C8560E9409B1AEEDB1E10E9423B15F5FEA
:10AD8E00F4CF67C0233011F00C94DB5650E05830EE
:10AD9E0010F00C94DA560E9409B1A6EEB1E10E94B1
:10ADAE0023B15F5FF4CF55C0243011F00C94ED56F3
:10ADBE0050E0583010F00C94EC560E9409B1AEEEF3
:10ADCE00B1E10E9423B15F5FF4CF43C0253011F093
:10ADDE000C94FF5650E0583010F00C94FE560E9422
:10ADEE0009B1A6EFB1E10E9423B15F5FF4CF31C08C
:10ADFE00263011F00C94115750E0583010F00C948E
:10AE0E0010570E9409B1AEEFB1E10E9423B15F5F0E
:10AE1E00F4CF1FC0273011F00C94215750E058305A
:10AE2E0010F00C9420570E9409B10E9411B15F5F7F
:10AE3E00F6CF0FC0283011F00C94305750E0583038
:10AE4E0010F00C9430570E9409B10E941AB15F5F46
:10AE5E00F6CF0E942AB1A8E0B0E00E9490490E946D
:10AE6E00B3B96D960895EAE7F4E060E070E00E94F1
:10AE7E003FBBA6EDB1E10E94B11BE3E8F4E060E058
:10AE8E0070E00E943FBBAEEDB1E10E94B11BECE859
:10AE9E00F4E060E070E00E943FBBA6EEB1E10E94DC
:10AEAE00B11BE5E9F4E060E070E00E943FBBAEEE5E
:10AEBE00B1E10E94B11BEEE9F4E060E070E00E94A7
:10AECE003FBBA6EFB1E10E94B11BE7EAF4E060E000
:10AEDE0070E00E943FBBAEEFB1E10E94B11BE0EB10
:10AEEE00F4E060E070E00E943FBBA6E0B2E10E9499
:10AEFE00B11BE9EBF4E060E070E00E943FBBAEE016
:10AF0E00B2E10E94B11B08950A930E941A440E9456
:10AF1E00AA44A4EFB1E00E940A0E0E945D4C0E2FCF
:10AF2E000E945026E03011F00C949E5700620030C3
:10AF3E0011F00C94A657E1E0E093C00F1DC0E02F76
:10AF4E00E07E11F40C94AF57E8ECE093C00F14C000
:10AF5E00E02FEC7111F40C94B857E9ECE093C00FAC
:10AF6E000BC001FF04C0EAECE093C00F05C000FF68
:10AF7E0003C0E4E6E093C00FE02F09910895EF9728
:10AF8E00EF97A2970E942FB1A2ECB4E080E090E080
:10AF9E000E94AA49A3EDB4E080E090E00E94AA4985
:10AFAE00A4EEB4E080E090E00E94AA49A1E00E94E5
:10AFBE0080490E9427ABA2E00E946945A3E00E944F
:10AFCE008145A5EFB4E080E090E00E94AA490E947E
:10AFDE002FB1A1E00E9422460E9427ABA2E00E9460
:10AFEE006945A2E00E948145ABEFB4E080E090E0BD
:10AFFE000E94AA490E942FB1EFEFF4E060E070E0EA
:10B00E000E946CAA0E94991BFE010E9438B1A1E019
:10B01E000E9480490E943FB1A1E7B5E080E090E038
:10B02E000E94AA49EEE7F5E060E070E00E946CAA8B
:10B03E000E9445B10E944CB1A4E10E9444460E9478
:10B04E0027ABA1E00E9480490E9451B1A0E00E946E
:10B05E006945A0E00E948145AAEAB5E080E090E053
:10B06E000E94AA490E943FB1A3ECB5E080E090E0B7
:10B07E000E94AA49A2E00E948145AFECB5E080E0B3
:10B08E0090E00E94AA490E943FB1A1E00E94AC4507
:10B09E00A3EEB5E080E090E00E94AA49A0E00E94F5
:10B0AE00AC45A1E00E94C445A0EFB5E080E090E081
:10B0BE000E94AA49A0E00E94C445A1E00E94DC457E
:10B0CE00A0E0B6E080E090E00E94AA49A0E00E94D5
:10B0DE00DC450E9451B10E9427ABA3E00E9480493B
:10B0EE00A1E00E94C544A8EEB3E00E940A0EEF96BE
:10B0FE00EF96A2960895AA930E94ACB940E050E054
:10B10E00AE81A03110F40C949158E2E00E94B3B9D4
:10B11E0029960895AE81E4E1EA9F9001EF81F885CA
:10B12E00FA93EA93E6EDF1E1FA93EA93A0E4B0E044
:10B13E000E94961A00E010E00431E0E01E0710F0C5
:10B14E000C94BA583A932A93E6EAEA93A6E1B2E14E
:10B15E00A40FB51F0E9440832F5F3F4F405C5F4F8F
:10B16E000F5F1F4FE9CF0E949D54E0E00E94B3B9DC
:10B17E00299608950E9457B10E945FB110F00C9469
:10B18E00CB580E946AB102C00E946FB100E010E07D
:10B19E000030E2E01E0710F00C94DC58DE0113962E
:10B1AE000E946FA60F5F1F4FF3CF0E9476B10E94D1
:10B1BE0069840E94B6B92396DE5F0895AA932397F9
:10B1CE000E9483B1E985EE83F801E07CAF01405C1B
:10B1DE005F4FFA01E01BF10BEF83F887EE810E94BF
:10B1EE008AB110F00C94FE588A010E946AB10E9436
:10B1FE00EEB0E985EA93AE85BF850E9490B12C969C
:10B20E000895AA932B97E8E0E8830E9483B1F80192
:10B21E00E07CAF01405C5F4FDA01A01BB10BEE8109
:10B22E00F0E0AE17BF0710F00C9420598A010E946F
:10B23E006AB1EBE1EF83EC89E887EB89E987EA896C
:10B24E00EA87E989EB87E0E2EC87ED87EE870E94DB
:10B25E00EEB0E985EA93DE011B960E9490B16596E9
:10B26E0008950E9457B10E945FB110F00C9442599C
:10B27E000E946AB102C00E946FB100E010E000307F
:10B28E00E2E01E0710F00C945359DE0113960E9453
:10B29E006FA60F5F1F4FF3CF0E9476B10E94A2B12F
:10B2AE000E9416AE0E9448930E94A9B10E94AEB1B0
:10B2BE000E94B6B92396DE5F08950E94ACB93A2F6C
:10B2CE004E815F81E32FE0530E2F023010F40C9469
:10B2DE00715900E04A93A32F0E94B4231E2F5236B9
:10B2EE0011F00C947E59A02F0E94AC4542C05537E8
:10B2FE0011F00C948659A02F0E94C4453AC05C36BA
:10B30E0011F00C948E59A02F0E94DC4532C051369C
:10B31E0011F00C949659A42F0E94F4452AC054366D
:10B32E0011F00C94A359133310F40C949F5912E39B
:10B33E00A12F0E9499451DC0563611F00C94AC59A0
:10B34E001A93ACE00E942E4514C0533711F00C94A2
:10B35E00C059A12FEAE00E949EBA2E2FA22F0E9462
:10B36E008145A12FEAE00E94EDBA2E2FA22F0E9456
:10B37E0069450E94B3B9289608950E94DEA5E22F72
:10B38E00E0530E2F3A93A22F0E94B4231E2FE42FC8
:10B39E00E33611F00C94D759A1E00E94C5445BC06E
:10B3AE00E03711F00C94DF59A2E00E94C54453C05F
:10B3BE00E53611F00C94E759A3E00E94C5444BC04A
:10B3CE00E23411F00C94F059A8EEB3E00E946C49EF
:10B3DE0042C0EE3611F00C94025A003011F40C9467
:10B3EE00FD590A3010F00C94FD5901C001E0A02F58
:10B3FE000E94804930C0EC3611F00C940E5A000FAA
:10B40E00000F000FA02FBB270E94FA4424C0E23683
:10B41E0011F00C941A5A000F000F000FA02FBB272B
:10B42E000E94144518C0ED3611F00C94225AA12F2B
:10B43E000E94ED4910C0E23711F00C942A5AA12F48
:10B44E000E94014A08C0E33711F00C94325AA12F22
:10B45E00BB270E943C4C0E94B4B927960895A29730
:10B46E000E94ACB95A2F0E940CAEA9A5A43411F0BB
:10B47E000C949C5AE52FE03311F00C944D5AE6EDE6
:10B48E00F1E10E9460A70E94C0B14CC0E13311F0FF
:10B49E000C94585AEEEDF1E10E9460A70E94C0B1E3
:10B4AE0041C0E23311F00C94635AE6EEF1E10E94D2
:10B4BE0060A70E94C0B136C0E33311F00C946E5AEF
:10B4CE00EEEEF1E10E9460A70E94C0B12BC0E43302
:10B4DE0011F00C94795AE6EFF1E10E9460A70E94F8
:10B4EE00C0B120C0E53311F00C94845AEEEFF1E1B7
:10B4FE000E9460A70E94C0B115C0E63311F00C94F3
:10B50E008F5AE6E0F2E10E9460A70E94C0B10AC025
:10B51E00E73311F00C94995AEEE0F2E10E9460A725
:10B52E000E94C0B10E94C4B10895E9A5E33611F09E
:10B53E000C94A65A0E94CDB10E94D2B19CC0ED3699
:10B54E0011F00C94AF5A0E94DBB10E94D2B193C09D
:10B55E00EC3611F00C94BC5AE8E8F0E00E9460A7BB
:10B56E00A0E2B0E00E94BD1A86C0E73611F00C943E
:10B57E00C55A0E94E0B10E94D2B17DC0EA3711F0E7
:10B58E000C94CE5A0E94E5B10E94D2B174C0E1363D
:10B59E0011F00C94D75A0E94EAB10E94D2B16BC03E
:10B5AE00E43711F00C94F45AA8A5AC3611F00C94B3
:10B5BE00E25A41E001C040E0E091690EEA93E09169
:10B5CE006A0EEA93E0916B0EEA93E0E0EA934A93F7
:10B5DE00DE011B960E94181E4EC0E43611F00C942C
:10B5EE00115B20E030E0A8A5A53711F00C94015BAB
:10B5FE0022E031E0E091670E0E94EFB1E0E2EA93C3
:10B60E00E091650EEA932A933A93DE011C960E940E
:10B61E00C41E31C0E73711F00C94425BA091680E46
:10B62E00A13010F40C94225BA091680EA83010F09B
:10B63E000C94225B0BC0E3E3F6E060E070E00E9446
:10B64E003FBBDE011A960E94991B15C041E055368C
:10B65E0011F00C94335B42E0E091680EEA934A934A
:10B66E00DE0118960E946E24A8A5A33711F00C9443
:10B67E00425BE0E0E8870E94C4B10895EF97EF9730
:10B68E00A2970E94AEB91A2FFE01EC55FF4F2081F2
:10B69E00FE01EB55FF4F3081FE0134960E9432AF12
:10B6AE00A0EAB0E00E94831BE32FE23611F00C9467
:10B6BE00755BEFE3F6E060E070E00E943FBBDE01F9
:10B6CE0018960E9445B10E9479AFA4E10E944446AB
:10B6DE000E9427ABA1E00E9480492AC0EC3611F0EF
:10B6EE000C948A5BE12FE0530E2F0A3010F40C9469
:10B6FE00815B01E0A02F0E9422460E9427ABA1E0B1
:10B70E000E94804915C0E13711F00C949F5BE4E56F
:10B71E00F6E060E070E00E943FBBDE0118960E94EA
:10B72E00991BFE0134960E9438B1A1E00E94804917
:10B73E000E94B5B9EF96EF96A89608951A930A93BC
:10B74E008D01F801E181E33711F00C94B35B0E9497
:10B75E00F4B10E9464591AC0E63611F00C94BC5B29
:10B76E000E94F4B10E94C45911C0E63711F00C9436
:10B77E00C55B0E94F4B10E94365A08C0E73611F03C
:10B78E000C94CD5B0E94F4B10E94455B0991199116
:10B79E000895AA932897D2500E94ACB9A0E00E94B7
:10B7AE008B250E940CAAFE01E25FFD4F008111273E
:10B7BE00D801E9E00E94F0B98F010030EEE31E07D8
:10B7CE0010F00C94ED5B0E946AB102C00E946FB142
:10B7DE0000E010E00030E2E01E0710F00C94FE5B7B
:10B7EE00DE0116960E946FA60F5F1F4FF3CFE091FA
:10B7FE002417F09125170E94FDB1E0E0F2E0FA93D4
:10B80E00EA93DE011C960E94A2B10E943FBBDE01AC
:10B81E00AE5EBD4FAC910E9404B20E9448930E944E
:10B82E0079AF0E94AEB10E948B574E2F423010F46A
:10B83E000C94265C0E94B3B92F96DE5F0895A3E0A8
:10B84E000E94804920E030E040E0F9012F5F3F4F39
:10B85E000E947BA75C915B3111F00C94385C41E047
:10B86E0009C0503011F00C943E5C42E003C0A52F8D
:10B87E000E941C142034E0E03E0710F00C944C5C47
:10B88E00403011F00C944C5C01C001C0DECF0E9420
:10B89E005CAA413011F00C946A5C21503040F901E1
:10B8AE00DE0116960E9409B2FE01E85FFD4FFA9383
:10B8BE00EA930E94C0B1DE01AA5FBD4F0E94A55B54
:10B8CE00285F3F4F05C0423011F00C946F5C00C0F2
:10B8DE002030E2E03E0710F00C94765CB5CF0E946B
:10B8EE005CAAE0E00E94B3B92F96DE5F08950A933A
:10B8FE0000E00E946228E03011F40C94875C026034
:10B90E000E949028E03011F40C948E5C04600E942A
:10B91E00C028E03011F40C94955C08600E94EC286D
:10B92E00E03011F40C949C5C00610E941A29E03006
:10B93E0011F40C94A35C0062E02F099108950A9310
:10B94E0000E00E94B52BE03011F40C94AF5C016066
:10B95E000E94D129E03011F40C94B65C04600E9470
:10B96E003A29E03011F40C94BD5C08600E945A290B
:10B97E00E03011F40C94C45C00610E94B029E030F8
:10B98E0011F40C94CB5C0062E02F099108950E9493
:10B99E00ACB91A2F2E813F8148855985183010F089
:10B9AE000C94DE5CE1E00E94B3B92A9608950E94E1
:10B9BE000EB200E00E946127E03011F40C94E85CB6
:10B9CE0001600E940D26E03011F40C94EF5C0260D1
:10B9DE000E942D26E03011F40C94F65C04600E9457
:10B9EE009826E03011F40C94FD5C08600E94132838
:10B9FE00E03011F40C94045D0061E02FDA01EC9359
:10BA0E000E94A65CDA011196EC9300E00E94092CCC
:10BA1E00E03011F40C94145D01600E94D52BE030DF
:10BA2E0011F40C941B5D02600E94E425E03011F4C9
:10BA3E000C94225D04600E94BE27E03011F40C9439
:10BA4E00295D08600E94A827E03011F40C94305D47
:10BA5E0000610E94D427E03011F40C94375D00622F
:10BA6E000E94F427E03011F40C943E5D00640E94B5
:10BA7E00492CE03011F40C94455D0068FA01028304
:10BA8E000E94FB29DA011396EC930E94472ADA01F1
:10BA9E001496EC93D901E8E0EC930E94B3B92A9680
:10BAAE0008952A970E94ACB91A2F288939894A8994
:10BABE005B8900E0183010F00C946A5DE1E00E94A2
:10BACE00B3B9649608950E940EB20E9479AF0E9497
:10BADE00C6A900E00E94652BE03011F40C94785D4D
:10BAEE0001600E947F2BE03011F40C947F5D0260A8
:10BAFE000E94C32CE03011F40C94865D04600E9409
:10BB0E002F2BE03011F40C948D5D08600E944B2BAE
:10BB1E00E03011F40C94945D0061E02FDA01EC93A7
:10BB2E0000E00E94CD2AE03011F40C949F5D01607C
:10BB3E000E94B12AE03011F40C94A65D02600E94BE
:10BB4E00F52AE03011F40C94AD5D04600E941D2BBB
:10BB5E00E03011F40C94B45D08600E949F2AE0302E
:10BB6E0011F40C94BB5D00610E94952BE03011F432
:10BB7E000C94C25D0064FA0101830E947E5CDA01BE
:10BB8E001296EC9300E00E94EE25E03011F40C9436
:10BB9E00D15D01600E941627E03011F40C94D85D3F
:10BBAE0002600E945026E03011F40C94DF5D0460B8
:10BBBE000E949227E03011F40C94E65D08600E941A
:10BBCE00FE27E03011F40C94ED5D00610E94F22628
:10BBDE00E03011F40C94F45D00620E946429E030B0
:10BBEE0011F40C94FB5D0064FA01038300E00E94E3
:10BBFE007D27E03011F40C94055E01600E940D2744
:10BC0E00E03011F40C940C5E02600E942527E030A7
:10BC1E0011F40C94135E04600E941328E03011F4AA
:10BC2E000C941A5E08600E94962CE03011F40C946D
:10BC3E00215E00610E949F2CE03011F40C94285E6E
:10BC4E0000620E94AB2CE03011F40C942F5E006465
:10BC5E000E94B42CE03011F40C94365E0068FA01A8
:10BC6E0004830E94EA2CDA011596EC935A934A93B8
:10BC7E000E9416B20E94C0B1D901E8E0EC93E0E058
:10BC8E000E94B3B9649608956697FE010E9432AF82
:10BC9E00A6E1B0E00E94831BE2E7F6E060E070E010
:10BCAE000E946CAA0E941BB266960895A8970A93EA
:10BCBE000E94C1AE0E9428B2E8A7E3E8F6E060E079
:10BCCE0070E00E9430B2DE0111960E94A3190E2F71
:10BCDE000E94B8AEE0E2EC93E0E9F6E060E070E0DE
:10BCEE000E943FBB0E94F9ABA4E1B0E00E945A1B38
:10BCFE00DE0111960E94A319EA93DE0112960E94AC
:10BD0E00FD74A0E00E94EE740881A9960895A8978C
:10BD1E000E9460AAEDE9F6E060E070E00E946CAA75
:10BD2E000E941BB2A89608956E970E94ADB90A2F75
:10BD3E001BA12CA13DA14EA10E3110F00C94AC5EB6
:10BD4E00E1E00E94B4B9A79608954A933A93E0E0D1
:10BD5E00EA93A02FBB270E94831B0E94F9AB0E947F
:10BD6E00C6A9E091BB0FA32FB42FEC93E091BC0FAB
:10BD7E00A32FB42F1196EC93E091BD0FA32FB42FE8
:10BD8E001296EC93E091BE0FA32FB42F1396EC9363
:10BD9E00E091BF0FA32FB42F1496EC93E091C00F38
:10BDAE00A32FB42F1596EC93E091C10FA32FB42FB0
:10BDBE001696EC93E091C20FA32FB42F1796EC9327
:10BDCE00E091C30FA32FB42F1896EC93E091C40FFC
:10BDDE00A32FB42F1996EC93E091C50FA32FB42F78
:10BDEE001A96EC93E091C60FA32FB42F1B96EC93EB
:10BDFE00E091C70FA32FB42F1C96EC93E091C80FC0
:10BE0E00A32FB42F1D96EC93E091C90FA32FB42F3F
:10BE1E001E96EC93E091CA0FA32FB42F1F96EC93AE
:10BE2E00E091CB0FA32FB42F5096EC93E091CC0F53
:10BE3E00A32FB42F5196EC93E091CD0FA32FB42FD7
:10BE4E005296EC93E091CE0FA32FB42F5396EC9312
:10BE5E00E091CF0FA32FB42F5496EC93E091D00F17
:10BE6E00A32FB42F5596EC93E091D10FA32FB42F9F
:10BE7E005696EC93E091D20FA32FB42F5796EC93D6
:10BE8E00E091D30FA32FB42F5896EC93E091D40FDB
:10BE9E00A32FB42F5996EC93E091D50FA32FB42F67
:10BEAE005A96EC93E091D60FA32FB42F5B96EC939A
:10BEBE00E32FF42F7C96A0E0A083E32FF42F7D9642
:10BECE00A083E32FF42F7E96A0834A933A930E9489
:10BEDE002AB1AEE1B0E00E94961AA12FB22FEEE188
:10BEEE00EC93E0E00E94B4B9A7960895E6971A93F2
:10BEFE000A93E091690EEE83E0916A0EEF83E09172
:10BF0E006B0EE887E091650EE987E091660EEA8791
:10BF1E00E091670EEB87E091680EEC87E0E2ED872B
:10BF2E0000916C0E10916D0E1A930A93A0E00E9470
:10BF3E003523EE870E946EAEEF87E0E2E88BE98B49
:10BF4E00E0916E0EF0916F0E6091700E7091710E09
:10BF5E000E9436B2EA8B0E943FB2A1E00E945123AA
:10BF6E00EB8B0E943FB2A2E00E945123EC8B0E9409
:10BF7E003FB2A3E00E945123ED8BA091650E0E946B
:10BF8E006D22EE8BA091650E0E947A22EF8BA0910E
:10BF9E00650E0E949522E88FE091680EEA93A091BB
:10BFAE00690E0E94C422E98FE091680E0E9446B28B
:10BFBE000E94D5220E9468AEEA8F0E946EAEEB8F71
:10BFCE00E091670EEA93A091690E0E94E3220E940F
:10BFDE0068AEEC8F0E946EAEED8FE091670E0E9400
:10BFEE0046B20E94F1220E9468AEEE8F0E946EAEA3
:10BFFE00EF8F0E944DB2A091670E0E9436220E94D2
:10C00E0068AEE8A30E946EAEE9A30E944DB2E09125
:10C01E00670EEA93A091690E0E94FE220E9468AEFE
:10C02E00EAA30E946EAEEBA3E0E0ECA3EDA30E94A8
:10C03E004DB2E091670E0E9446B20E9412230E94FA
:10C04E0036B2EEA30E943FB2A1E00E945123EFA3AD
:10C05E000E943FB2A2E00E945123E8A70E943FB285
:10C06E00A3E00E945123E9A70E942150EAA7E0E035
:10C07E00EBA7ECA7EDA7EA83EB83EC83ED830E949D
:10C08E003FB2A0E00E945123EEA70E943FB2A1E072
:10C09E000E945123EFA70E943FB2A2E00E945123BB
:10C0AE00E8AB0E943FB2A3E00E945123E9ABECE261
:10C0BE00EA93DE0117960E94FD74A0E00E94EE74D2
:10C0CE00E0E019810881E8960895E0E0E0932617F4
:10C0DE00E0932717E0932817EAE0E0932917E093FF
:10C0EE002A170E9450B2E0E0E0933B17E0933A1714
:10C0FE00E0933D1708950E9450B2A0E00E94DB2904
:10C10E00A0E00E941C2AA0E00E94B2270E9456B214
:10C11E00A0E00E949F2B0E9453AB0E947F2A08959D
:10C12E0021970E9471AAA0912617A13011F00C94AC
:10C13E00A060A0912617A23011F00C94A660A091D9
:10C14E002717A13011F00C94AC60A0912717A230E4
:10C15E0011F00C94B260A0913917A33011F00C9429
:10C16E00C3600E949227E03011F40C94C0600E94CC
:10C17E0060B2EE81E260EE83A0913917A23011F425
:10C18E000C94CE60A33011F40C94CE6020C020919C
:10C19E0038173327AAE0A29FF001A39FF00D9F014D
:10C1AE002436E0E03E0710F00C94DF6024E630E029
:10C1BE00A3E10E94990E8F010217130710F40C943D
:10C1CE00EB60A0E00E94B227EE81E260EE830E9457
:10C1DE0066B25E2F513011F40C94FA60523011F4A5
:10C1EE000C94FA6077C0A4E10E94990E8F010E9410
:10C1FE00FE274E2FA0913A17A23011F00C940E612B
:10C20E000536E0E01E0710F40C940E6101C002C06A
:10C21E000E9456B20333E0E01E0710F40C94226124
:10C22E000436E0E01E0710F00C942261403011F04D
:10C23E000C9422610CC0093CE0E01E0710F40C9433
:10C24E002D61403011F40C942D6101C009C0A091F4
:10C25E003A17A23011F00C943761E9ECE093C60F57
:10C26E000333E0E01E0710F40C9448610436E0E05E
:10C27E001E0710F00C944861403011F40C94486184
:10C28E0001C003C0E1E0E0933B17093CE0E01E076C
:10C29E0010F40C9463610A3FE0E01E0710F00C945A
:10C2AE006361403011F00C946361E0913B17E03014
:10C2BE0011F40C94636101C006C0E1E0E093C60F77
:10C2CE00E0E0E0933B17403011F40C947161EE8185
:10C2DE00E260EE83AAE10E946BB210F40C947B61D3
:10C2EE00A0E00E94CD2C03C0EE81E260EE830E949E
:10C2FE0072B25E2F513010F40C94D961A0913C179C
:10C30E00A53010F40C948C614DC0A0913C17A03058
:10C31E0011F40C949761A23011F40C94976107C03C
:10C32E000E946429E03011F00C949E6101C002C09D
:10C33E000E9477B2A0913C17A13011F40C94AC611D
:10C34E00A33011F40C94AC6107C00E946429E03054
:10C35E0011F40C94B36101C002C00E9477B2ABE13C
:10C36E000E94990E8F01A0913C17A43011F00C94ED
:10C37E00C861A0E00E946A290E9477B2E1E0E093D2
:10C38E00C90F0D32E1E01E0710F40C94D661A0E047
:10C39E000E946A290E9477B2E8ECE093C90FEE8101
:10C3AE00E260EE83A0912817A23011F00C94FE618A
:10C3BE00A7E10E94990E8F01E0912B170E947DB28A
:10C3CE0010F00C94F161A0E00E949F2BA7E10E9457
:10C3DE00820E0DC0E0912A170E947DB210F00C94CF
:10C3EE00FE61A1E00E949F2BEE81E460EE83A0919E
:10C3FE002C17A23011F00C941F62A8E10E94990E26
:10C40E008F01E0912F170E947DB210F00C941662EE
:10C41E00A0E00E94BB29A8E10E94820E09C0E09113
:10C42E002E170E947DB210F00C941F620E9482B2F1
:10C43E00A0913317A23011F00C944062A9E10E9432
:10C44E00990E8F01E09136170E947DB210F00C9478
:10C45E003762A0E00E94BB29A9E10E94820E09C0AA
:10C46E00E09135170E947DB210F00C9440620E944C
:10C47E0082B2E0914417E03011F40C945962AAE0B4
:10C48E000E94E40E8F010230E0E01E0710F40C94BF
:10C49E005662A0E00E94D525E0E0E0934417EE81BD
:10C4AE00E860EE83A091D60FA23011F00C946E626C
:10C4BE00A9E00E9489B210F40C946B62A0E00E9475
:10C4CE00DF2BE1E0E093D60FEE81E061EE83E091A9
:10C4DE00D60FE03011F00C947762A0E00E94DF2BB3
:10C4EE00A0913D17A23011F00C948B62ADE00E942A
:10C4FE00E40E8F010B30E0E01E0710F40C948A62FC
:10C50E00E0E0E0933D171CC0A0913D17A13011F063
:10C51E000C94A762ADE00E94E40E8F010430E0E0BF
:10C52E001E0710F40C94A462A0E00E94F129E2E030
:10C53E00E0933D17ADE00E94C80EEE81E160EE8300
:10C54E00EE810E94B3B9279608950A930A2F00939D
:10C55E002617A1E00E947F2AA0912617A13011F084
:10C56E000C94BB620E9490B2A0912617A23011F0DB
:10C57E000C94C3620E9490B2E0912617E03011F045
:10C58E000C94CC62A0E00E94DB29099108950A93D5
:10C59E000A2F00932717A0912717A13010F40C949F
:10C5AE00DB62E1E0E0932717A1E00E947F2AA091D1
:10C5BE002717A13011F00C94F1620E94F52AE03099
:10C5CE0011F00C94F162A2E10E94820EA091271745
:10C5DE000E941C2AA0912717A23011F00C94F7622A
:10C5EE00E0912717E03011F00C940063A0E00E9458
:10C5FE001C2A099108950E9479AE209328171130B4
:10C60E0010F40C940C6310932917013010F40C9451
:10C61E00126300932A17E0912917A0912A17EA0FA7
:10C62E00E0932B17213011F00C942163A1E00E94AE
:10C63E009F2B03C0A0E00E949F2B0E94B6B92596A7
:10C64E0008950E9479AE20932C17113010F40C949B
:10C65E00326310932D17013010F40C94386300934D
:10C66E002E17E0912E17A0912D17EA0FE0932F179A
:10C67E00213011F00C944763A1E00E94BB2903C046
:10C68E00A0E00E94BB290E94B6B9259608950E948B
:10C69E0079AE20933017113010F40C945863109328
:10C6AE003117013010F40C945E6300933217213071
:10C6BE0011F00C946663A1E00E94242903C0A0E04F
:10C6CE000E9424290E94B6B9259608950E9479AE3B
:10C6DE0020933317113010F40C94776310933417A2
:10C6EE00013010F40C947D6300933517E0913417EC
:10C6FE00A0913517EA0FE0933617213011F00C9404
:10C70E008C63A1E00E94442903C0A0E00E9444294A
:10C71E000E94B6B9259608950A930A2F00933717EB
:10C72E00013011F00C949F63A1E00E949A2903C07E
:10C73E00A0E00E949A29099108950A930A2F0030C9
:10C74E0011F40C94B163A1E00E94B227E1E0E093F2
:10C75E00391706C0A0E00E94B227E1E0E093391736
:10C76E00099108950E9460B2E2E0E09339170895AE
:10C77E00E3E0E093391708950A930A2F00933817D0
:10C78E00099108951A930A931A2F0E9466B20E2FDA
:10C79E00013011F40C94D863023011F40C94D86368
:10C7AE001CC0113011F00C94E2630E9497B2E1E0CC
:10C7BE00E0933A170FC0123011F00C94EC630E9404
:10C7CE009DB2E1E0E0933A1705C00E94A3B2E0E00B
:10C7DE00E0933A17A4E10E94820E099119910895EF
:10C7EE000A930E9466B20E2F013011F40C94046469
:10C7FE00023011F40C94046408C0A1E00E94DA2700
:10C80E00A0E00E94C4270E94A9B2099108950A933C
:10C81E000E9466B20E2F013011F40C941B6402308C
:10C82E0011F40C941B6404C00E949DB20E94A9B224
:10C83E0009910895A1E00E94CD2CAAE10E94820EDA
:10C84E0008950A930E9472B20E2F013010F40C94C8
:10C85E003B640E94E62CA1E00E946A29ABE10E9493
:10C86E00820EE0E0E0933C17099108950A930E942E
:10C87E0066B20E2F013010F40C945C640E949F2A55
:10C88E00E03011F40C945064A1E00E947F2A0E94C3
:10C89E00E6AB0E947F2BE03011F40C945964E1E07A
:10C8AE0009910895E0E009910895E1E00991089554
:10C8BE000A930E94B2B20E2F013010F40C947E64D3
:10C8CE000E949F2AE03011F40C947264A1E00E9441
:10C8DE007F2A0E94E6AB0E944B2BE03011F40C94A1
:10C8EE007B64E1E009910895E0E009910895E1E0AB
:10C8FE00099108950A930E949F2AE03011F40C9436
:10C90E008A640E94B7B20E94BF2A0E2F013011F026
:10C91E000C949464E1E009910895E0E00991089582
:10C92E000A930E949F2AE03011F40C94A0640E9496
:10C93E00B7B20E94C32C0E2F003011F00C94AA64D3
:10C94E00E0E009910895E1E0099108950E949F2A7F
:10C95E00E03011F40C94B5640E94B7B20E943D2BE6
:10C96E00E03011F40C94BD64E1E00895E0E0089528
:10C97E001A930A9310E00E949F2AE03011F40C944F
:10C98E00CA640E94B7B20E94BF2A0E2F013011F066
:10C99E000C94D26411600E94C32C0E2F013011F042
:10C9AE000C94DA6412600E943D2B0E2F013011F0B0
:10C9BE000C94E2641460E12F099119910895E1E05D
:10C9CE00E0934417A1E00E94D525AAE00E94C80E6C
:10C9DE0008950A93E1E0E093D60F0E94BEB20E2FA7
:10C9EE00013010F40C940465E2E0E093D60FA9E058
:10C9FE000E94C80EA1E00E94DF2B09910895A0E0CD
:10CA0E000E94DF2BE0E0E093D60F0895E091D60F61
:10CA1E0008950A930A2FE0913D17E03011F00C941F
:10CA2E002965013010F40C942065A1E00E94F129D3
:10CA3E0003C0A2E00E94F129E1E0E0933D17ADE0D2
:10CA4E000E94C80E09910895A0E00E94F129E0E02D
:10CA5E00E0933D170895EFE4F7E1E093DC17F093D0
:10CA6E00DD170E94C3B20895E0E00895BA93AA9329
:10CA7E00EF97AD970E94ACB9FE01EC58FF4F0190B5
:10CA8E00F081E02DDE01A059BF4FED93FC93FE0126
:10CA9E00EE58FF4F0190F081E02DDE01A259BF4FFD
:10CAAE00ED93FC930E9466B25E2FDE01A059BF4F3C
:10CABE00AC910E942F75FE01E059FF4F0190F0815D
:10CACE00E02DEA30A0E0FA0711F00C9471650E9497
:10CADE004B5EE4C2E436A0E0FA0711F00C948365D5
:10CAEE000E94C9B22E2FE1E0EA93ADB7BEB72F93E5
:10CAFE000E94FD742F91D2C2E936A0E0FA0711F020
:10CB0E000C9499650E94CEB2EA8FE8E0EB8F0E94FA
:10CB1E00D3B2EC8FE2E0ED8FE0E0EE8FE4E00E9426
:10CB2E00D8B2BCC2EB30A0E0FA0711F00C94A265AB
:10CB3E000E945D5EB3C2EC30A0E0FA0711F00C94D7
:10CB4E00AB650E948E5EAAC2E536A0E0FA0711F030
:10CB5E000C94BF650E94DDB2EDB7FEB7FA93EA936F
:10CB6E002F93A2E40E949B5E2F910E94E2B296C286
:10CB7E00E636A0E0FA0711F00C94D3650E94DDB200
:10CB8E00EDB7FEB7FA93EA932F93A2E40E94585D95
:10CB9E002F910E94E2B282C2E736A0E0FA0711F0AE
:10CBAE000C94E7650E94DDB2EDB7FEB7FA93EA93F7
:10CBBE002F93A2E40E94CE5C2F910E94E2B26EC22D
:10CBCE00E836A0E0FA0711F00C940466DE01A45AD0
:10CBDE00BF4F0E94BD4D3E2FE0E0DE01AD59BF4F6D
:10CBEE00EC93303011F00C940366E8E0EA93DE012A
:10CBFE00A35ABF4F0E94FD7451C2E331A0E0FA0761
:10CC0E0011F00C940D660E947D5F48C2EA36A0E0DA
:10CC1E00FA0711F00C9439660E94B8520E9468AE61
:10CC2E00EA8F0E946EAEEB8F0E948A520E9468AE0F
:10CC3E00EC8F0E946EAEED8FA0E00E94E8520E9433
:10CC4E0068AEEE8F0E946EAEEF8FA1E00E94E852AA
:10CC5E000E9468AEE8A30E946EAEE9A3E8E00E94CF
:10CC6E00D8B21CC2EE30A0E0FA0711F00C947C662C
:10CC7E00A8EAB0E00E9454BBEA8F0E9466B2EB8F26
:10CC8E00AAEAB0E00E9454BBEC8FABEAB0E00E947F
:10CC9E0054BBED8FACEAB0E00E9454BBEE8FADEA10
:10CCAE00B0E00E9454BBEF8FAEEAB0E00E9454BBDE
:10CCBE00E8A30E9472B2E9A3A0EBB0E00E9454BBBD
:10CCCE00EAA30E94B2B2EBA3A2EBB0E00E9454BB67
:10CCDE00ECA30E94BEB2EDA3A4EBB0E00E9454BB45
:10CCEE00EEA3EDE00E94D8B2D9C1E131A0E0FA077F
:10CCFE0011F00C94D0660E94CDB10E94E7B2EA8F7B
:10CD0E000E94CDB10E94ECB2EB8F0E94DBB10E946B
:10CD1E00E7B2EC8F0E94DBB10E94ECB2ED8F0E9465
:10CD2E00E0B10E94E7B2EE8F0E94E0B10E94ECB239
:10CD3E00EF8F0E94E5B10E94E7B2E8A30E94E5B131
:10CD4E000E94ECB2E9A30E94EAB10E94E7B2EAA304
:10CD5E000E94EAB10E94ECB2EBA340E0403210F028
:10CD6E000C94CC66E42FE65FF0E0DE015A96EA0FF3
:10CD7E00FB1F0F01A8E8B0E0EE27A40FBE1F0E9414
:10CD8E0054BBD001EC934F5FE9CFEAE20E94D8B2D8
:10CD9E0085C1E231A0E0FA0711F00C94EB66DE01DA
:10CDAE0016960E943B503E2F303011F00C94E666E2
:10CDBE00E8E0EA93DE0117960E94FD7404C0E2E0FB
:10CDCE000E94F1B208956AC1EF36A0E0FA0711F0A1
:10CDDE000C94F8660E942150EA8FE1E00E94D8B2CE
:10CDEE005DC1E431A0E0FA0711F00C940C670E94CB
:10CDFE00F6B2FA93EA930E94FDB2DE015E960E94AD
:10CE0E00BB0CE0E40E94D8B249C1E531A0E0FA07BC
:10CE1E0011F00C942A670E94F6B20E94FDB10E9496
:10CE2E00FDB2DE0190960E9458833E2F303011F0F5
:10CE3E000C942567E0E40E94D8B204C0E2E00E94A0
:10CE4E00F1B208952BC1EB36A0E0FA0711F00C9465
:10CE5E0043670E9402B30E9405B30E94C437EA8F53
:10CE6E000E94B42CEB8F0E942527EC8FE1E0EC8F13
:10CE7E00E3E00E94D8B212C1E631A0E0FA0711F049
:10CE8E000C9468670E9402B30E9405B3E0914D179F
:10CE9E00EA8FE0914E17EB8FA0914D170E94FB3851
:10CEAE00EC8FA0914D170E940A39ED8FE0914D172E
:10CEBE00EA93DE015F960E941439E8E20E94D8B22E
:10CECE00EDC0E731A0E0FA0711F00C9488675330FB
:10CEDE0011F00C947767DE015A960E9487420DC0BE
:10CEEE00513011F40C948067523011F40C94806719
:10CEFE0004C0DE015A960E94A63EE0E40E94D8B21B
:10CF0E00CDC0EC36A0E0FA0711F00C94C8670E9471
:10CF1E0002B30E9405B3533011F00C94A9670E941E
:10CF2E0000430E9409B30E9410B3E42FEE5FF0E0BD
:10CF3E000E944DA80E9416B30E941EB30E94034386
:10CF4E004B5F1BC0513011F40C94B267523011F488
:10CF5E000C94B26712C00E940F3F0E9409B30E9448
:10CF6E0010B3E42FEE5FF0E00E944DA80E9416B3BE
:10CF7E000E941EB30E94123F4B5FE8E00E94D8B29F
:10CF8E008DC0ED36A0E0FA0711F00C94D3670E9425
:10CF9E0002B30E9405B382C0E831A0E0FA0711F097
:10CFAE000C94E367203011F00C94DE6704C0E4E0CB
:10CFBE000E94F1B2089572C0E931A0E0FA0711F0B3
:10CFCE000C9405680E9402B30E9405B3E4EBF6E0F0
:10CFDE0060E070E00E943FBBFE017E96FA93EA93FA
:10CFEE000E9426B3E0E0DE01A55ABF4FEC93DE01AE
:10CFFE005A960E94A3190E94D8B250C0EE36A0E0F5
:10D00E00FA0711F00C9416680E9402B30E9405B341
:10D01E000E942AB32F5FE8E00E94D8B23FC0EA31E7
:10D02E00A0E0FA0711F00C9428680E9402B30E9447
:10D03E0005B3DE015A960E94724D2E2F0E94E2B267
:10D04E002DC0EB31A0E0FA0711F00C9451680E944C
:10D05E0002B30E9405B30E94E7B00E94F8AF0E948F
:10D06E002AB3DE0116960E94724D2E2F0E9479AFC2
:10D07E000E940DB0FE017E96FA93EA93EAE0F0E08C
:10D08E00FA93EA93AAE0B0E00E94301BE6E10E9418
:10D09E00D8B204C0E1E00E94F1B20895E0E00E942F
:10D0AE00F1B20895EEEDF7E1E0936B18F0936C1882
:10D0BE000E94C3B20895E0E00895BA93AA932F9701
:10D0CE00D1500E94ACB9FE01E65EFE4F0190F08198
:10D0DE00E02DDE01AD5EBE4FED93FC93FE01E85EEA
:10D0EE00FE4F0190F081E02DDE01AF5EBE4FED935D
:10D0FE00FC93FE01E95EFE4F5081FE01EF52FF4FA1
:10D10E000E9432AF0E94EAB00E94FDB2DE01A75E1D
:10D11E00BE4FAC91BB270E94E7215E2F20E0251762
:10D12E0010F00C94AE68E22F0E9433B3EA0FFB1F8F
:10D13E00BF01DE01AB5EBE4F0D90BC91A02DEE2760
:10D14E00A20FBE1FEC91DB01EC932F5FE8CF0E9484
:10D15E0066B2EAA7DE01AD5EBE4F0D90BC91A02D6A
:10D16E00A130E0E1BE0710F40C94C068E0E0E8875F
:10D17E00E987FE01ED5EFE4F0190F081E02DEA3071
:10D18E00A0E0FA0711F00C94E468E0EDF6E060E040
:10D19E0070E00E943FBBDE01AB52BF4F0E94931F57
:10D1AE004E2F403011F40C94DF680E94AC0C04C07A
:10D1BE00E2E00E9438B30895AAC5E436A0E0FA076B
:10D1CE0011F00C94EF680E943DB30E9402639FC55C
:10D1DE00E536A0E0FA0711F00C94F66898C5E6362D
:10D1EE00A0E0FA0711F00C9401690E943DB30E9471
:10D1FE0028638DC5E736A0E0FA0711F00C940C6990
:10D20E000E943DB30E944E6382C5E836A0E0FA0745
:10D21E0011F00C9417690E943DB30E946D6377C59F
:10D22E00E936A0E0FA0711F00C9422690E944CB383
:10D23E000E9493636CC5EA36A0E0FA0711F00C94D5
:10D24E00296965C5EB36A0E0FA0711F00C94346934
:10D25E000E944CB30E94DF2B5AC5EC36A0E0FA07B1
:10D26E0011F00C943F690E944CB30E94BF2B4FC526
:10D27E00ED36A0E0FA0711F00C944A690E944CB307
:10D28E000E94C92544C5EE36A0E0FA0711F00C94B1
:10D29E0055690E944CB30E94072839C5E231A0E0BF
:10D2AE00FA0711F00C9470690E9451B30E943E2847
:10D2BE000E9456B30E946C280E945BB30E949A286B
:10D2CE000E9460B30E94C8280E9465B30E94F6288F
:10D2DE001EC5E331A0E0FA0711F00C948B690E9491
:10D2EE0051B30E9456280E9456B30E9484280E9471
:10D2FE005BB30E94B2280E9460B30E94E0280E9495
:10D30E0065B30E940E2903C5EF36A0E0FA0711F0AF
:10D31E000C9496690E944CB30E947F2AF8C4E431A3
:10D32E00A0E0FA0711F00C94CC690E946AB3DE01FA
:10D33E00A552BF4FAC910E940F4F4E2F0E947AB351
:10D34E000E9460B30E9480B38F010A93FE01E952DE
:10D35E00FF4FE081EA93DE01A752BF4FAC910E94CE
:10D36E009C4F3E2F403011F00C94C269303011F0BA
:10D37E000C94C26901C004C0E0E00E9438B3089565
:10D38E00E1E00E9438B30895C2C4E531A0E0FA0787
:10D39E0011F00C94DE690E946AB3DE01A952BF4FF0
:10D3AE00AC910E940F4F0E9486B30895B0C4E6312F
:10D3BE00A0E0FA0711F00C94F7690E9488B30E945E
:10D3CE0080B38F010A93FE01EC52FF4FE081EA9386
:10D3DE000E9465B30E949C4F0E9486B3089597C425
:10D3EE00E037A0E0FA0711F00C940D6A0E948EB39C
:10D3FE0041E0323010F00C94086AA32F0E94EE4FD9
:10D40E004E2FE42F0E9438B3089581C4E137A0E077
:10D41E00FA0711F00C94146A7AC4E237A0E0FA0706
:10D42E0011F00C941B6A73C4E337A0E0FA0711F0F5
:10D43E000C94266A0E944CB30E94AC6268C4E43716
:10D44E00A0E0FA0711F00C94316A0E944CB30E94CE
:10D45E00CE625DC4E537A0E0FA0711F00C943A6A8B
:10D46E000E94216454C4E637A0E0FA0711F00C9430
:10D47E00456A0E944CB30E946A2949C4E737A0E06E
:10D48E00FA0711F00C944E6A0E94286440C4E731EA
:10D49E00A0E0FA0711F00C94096B0E948EB33230A3
:10D4AE0010F40C945B6A31E0E32FA8EAB0E00E941E
:10D4BE0070BBFE01EE52FF4F3081343010F40C94ED
:10D4CE00696A31E0A9EAB0E0E32F0E9470BBFE0169
:10D4DE00ED52FF4F3081323010F40C94776A31E008
:10D4EE00AAEAB0E0E32F0E9470BBFE01EC52FF4FA0
:10D4FE003081323010F40C94856A30E0ABEAB0E043
:10D50E00E32F0E9470BBFE01EB52FF4F3081313092
:10D51E0010F40C94936A30E0ACEAB0E0E32F0E9472
:10D52E0070BBFE01EA52FF4F3081313010F40C9483
:10D53E00A16A30E0ADEAB0E0E32F0E9470BBFE01BD
:10D54E00E952FF4F3081313010F40C94AF6A30E065
:10D55E00AEEAB0E0E32F0E9470BBFE01E852FF4F2F
:10D56E003081313010F40C94BD6A30E0AFEAB0E097
:10D57E00E32F0E9470BBFE01E752FF4F3081313026
:10D58E0010F40C94CB6A30E0A0EBB0E0E32F0E94D5
:10D59E0070BBFE01E652FF4F3081313010F40C9417
:10D5AE00D96A30E0A1EBB0E0E32F0E9470BBFE0120
:10D5BE00E552FF4F3081313010F40C94E76A30E0C1
:10D5CE00A2EBB0E0E32F0E9470BBFE01E452FF4FCE
:10D5DE003081313010F40C94F56A30E0A3EBB0E0FA
:10D5EE00E32F0E9470BBFE01E352FF4F30813130BA
:10D5FE0010F40C94036B30E0A4EBB0E0E32F0E9428
:10D60E0070BB85C3EB30A0E0FA0711F00C94676B8A
:10D61E000E9488B30E9449208F01ACE7B0E00E94BF
:10D62E0068BBFE01EC52FF4FE081EA930E945BB3B0
:10D63E000E9449208F01AEE7B0E00E9468BBFE0158
:10D64E00EA52FF4FE081EA930E9465B30E9449209F
:10D65E008F01A0E8B0E00E9468BBFE01E852FF4FC8
:10D66E00E081EA93DE01A852BF4FAC910E9449209F
:10D67E008F01A2E8B0E00E9468BBFE01E652FF4FA8
:10D68E00E081EA93DE01A652BF4FAC910E94492081
:10D69E008F01A4E8B0E00E9468BB20E0203210F0B9
:10D6AE000C94666BA8E8B0E0E22F0E946AA9E22F04
:10D6BE00E65F0E9433B30E9431AD2F5FEFCF27C3D9
:10D6CE00E837A0E0FA0711F00C94796B0E944CB386
:10D6DE00A13010F40C94766B0E94EC3702C00E94BD
:10D6EE00DA3715C3E937A0E0FA0711F00C94826B14
:10D6FE000E94B9370CC3EA37A0E0FA0711F00C9478
:10D70E008D6B0E944CB30E940C3801C3EB37A0E026
:10D71E00FA0711F00C949F6B0E9493B30E9498B37A
:10D72E000E9493B3EA930E9456B30E949E38EFC2B2
:10D73E00EC30A0E0FA0711F00C94B16B0E9493B399
:10D74E000E9498B30E946AB3DE01A952BF4F0E9495
:10D75E00B238DDC2E831A0E0FA0711F00C94126C79
:10D76E000E9488B30E9449208F01E3E0F0E0E88731
:10D77E00F987E0E0EE83EF83AE81BF81509710F022
:10D78E000C94F16BEE81FF81DE011A960E9458AE69
:10D79E00FF93EF93E885F9853196DE01AF52BF4FC7
:10D7AE00AE0FBF1FEC91EA93E985FA85DE01AE520A
:10D7BE00BF4FAE0FBF1FAC910E944920AF91BF91DA
:10D7CE00ED93FC93E885F9853296E887F9870E94F8
:10D7DE0038A6D2CFAAA5A33011F00C94FF6B1A93E2
:10D7EE000A930E947AB3DE011D960E94EA4112C08E
:10D7FE00AAA5A13011F40C94096CA23011F40C946A
:10D80E00096C08C01A930A930E947AB3DE011D9622
:10D81E000E94A33D7CC2EC37A0E0FA0711F00C94F5
:10D82E00316CAAA5A33011F00C94226C0E944CB35B
:10D83E000E941C420EC0AAA5A13011F40C942C6CAF
:10D84E00A23011F40C942C6C04C00E944CB30E94B4
:10D85E001A3E5DC2ED37A0E0FA0711F00C944C6C45
:10D86E00AAA5A33011F00C943F6C0E9435420CC057
:10D87E00AAA5A13011F40C94496CA23011F40C94A9
:10D88E00496C02C00E943E3E42C2EE37A0E0FA074B
:10D89E0011F00C94676CAAA5A33011F00C945A6C7D
:10D8AE000E9470420CC0AAA5A13011F40C94646CB5
:10D8BE00A23011F40C94646C02C00E94883E27C200
:10D8CE00EF37A0E0FA0711F00C946E6C20C2E0382E
:10D8DE00A0E0FA0711F00C94756C19C2E138A0E0C3
:10D8EE00FA0711F00C94806C0E944CB30E94A46352
:10D8FE000EC2E238A0E0FA0711F00C948D6C0E9473
:10D90E004CB30E94C3630E94B96301C2E338A0E026
:10D91E00FA0711F00C949A6C0E9451B30E94C363E3
:10D92E000E94BF63F4C1E438A0E0FA0711F00C9432
:10D93E00B86C0E9493B3E17011F40C94AA6CA1E040
:10D94E000E94C9630DC00E9493B3E27011F40C944F
:10D95E00B46CA2E00E94C96303C0A0E00E94C96338
:10D96E00D6C1E538A0E0FA0711F00C94C16C0E9404
:10D97E00F763CDC1E638A0E0FA0711F00C94CA6C3B
:10D98E000E940E64C4C1E738A0E0FA0711F00C94AF
:10D99E00DC6C0E948EB3A32F0E947A2CA1E00E9411
:10D9AE00F725A1E00E941726B2C1E838A0E0FA07D9
:10D9BE0011F00C94E76C0E944CB30E946A26A7C12A
:10D9CE00E938A0E0FA0711F00C94F46C0E944CB305
:10D9DE000E94A22C0E94A4B39AC1EA38A0E0FA07D2
:10D9EE0011F00C94FF6C0E944CB30E94CD268FC197
:10D9FE00EB38A0E0FA0711F00C94166D0E944CB3B0
:10DA0E00A13011F00C940E6D0E94AA4402C00E9427
:10DA1E00C144E0E0E0936D180E943F4878C1E931BF
:10DA2E00A0E0FA0711F00C94426DFE01E852FF4F90
:10DA3E00E0810E94AAB3FE01E952FF4FE0810E94ED
:10DA4E00AAB3FE01EA52FF4FE0810E94AAB3FE0183
:10DA5E00EB52FF4FE081FF2766277727EDA7FEA742
:10DA6E006FA778AB0E94BDB3AFA5B8A989A99AA933
:10DA7E000E94244A4CC1EA31A0E0FA0711F00C943E
:10DA8E00516D0E946AB3DE01A952BF4FAC910E9444
:10DA9E00074C3DC1EB31A0E0FA0711F00C946C6D10
:10DAAE000E9488B30E944920DF010E943C4C0E94D4
:10DABE0056B30E9499450E945BB30E94F4450E94A2
:10DACE0060B3BB270E943F4922C1EC38A0E0FA07A1
:10DADE0011F00C948A6D0E9451B3A13011F00C9488
:10DAEE007E6D0E944CB3BB270E94FA440BC00E946D
:10DAFE0051B3A23011F00C94896D0E944CB3BB2728
:10DB0E000E94144504C1ED38A0E0FA0711F00C9400
:10DB1E00A06D0E9493B3EA930E9456B30E942E45C5
:10DB2E000E9456B30E9469450E945BB30E948145D4
:10DB3E00EEC0EE38A0E0FA0711F00C94B36D0E941F
:10DB4E004CB30E94AC450E9451B30E94DC450E942A
:10DB5E0056B30E94C445DBC0EF38A0E0FA0711F0BF
:10DB6E000C94BE6D0E944CB30E94C544D0C0ED30E3
:10DB7E00A0E0FA0711F00C94CE6DFE01EF52FF4FAC
:10DB8E00FA93EA93A52FBB270E940C15C0C0E0396B
:10DB9E00A0E0FA0711F00C94D96D0E944CB30E94CC
:10DBAE008049B5C0E139A0E0FA0711F00C94E26D9E
:10DBBE000E94B249ACC0EE30A0E0FA0711F00C940E
:10DBCE000A6EFE01EB52FF4F308120E0231710F05A
:10DBDE000C94006EE22FF0E0DE01D196EA0FFB1FEF
:10DBEE000F01E22FEB5F0E9433B30E94BFA72F5F9E
:10DBFE00EDCF0E94BDB3FE01F396FA93EA93A32FE5
:10DC0E000E94444684C0EF30A0E0FA0711F00C9455
:10DC1E00246EA0916D18A33010F00C94236EE09139
:10DC2E006D18EA93DE01AE52BF4F0E945648E09146
:10DC3E006D18EF5FE0936D186AC0E239A0E0FA0745
:10DC4E0011F00C942D6E0E94234961C0E339A0E0BF
:10DC5E00FA0711F00C943C6E0E9451B30E943346A9
:10DC6E000E944CB30E94224652C0E031A0E0FA0757
:10DC7E0011F00C945C6EFE01EF5EFE4FE081ECA79E
:10DC8E00FE01EF5EFE4F01911081012F11270BA7B0
:10DC9E00EBA5EA93EDA5EA93DE01AD52BF4F0E94CC
:10DCAE006E540E9486B3089532C0E131A0E0FA07A7
:10DCBE0011F00C94716EFE01EF52FF4FFA93EA933E
:10DCCE00DE01AD5EBE4FAC910E9482580E9486B3BB
:10DCDE0008951DC0E439A0E0FA0711F00C947C6E93
:10DCEE000E944CB30E94445412C0E231A6E3FA07DC
:10DCFE0011F00C94836E0BC0EC31A0E0FA0711F01A
:10DD0E000C948A6E04C0E1E00E9438B30895FE01BF
:10DD1E00EF5EFE4F0190F081E02DDE01AF5EBE4F53
:10DD2E00ED93FC93E0E00E9438B308951A930A93A2
:10DD3E008D01E2E0EC93099119910895EA97E0E0E4
:10DD4E00EFAB20E030E040E050E0FE01F596EBABAB
:10DD5E00FCABABA9BCA90E949D6EABA9BCA90C9152
:10DD6E0011279924E0E0F2E03E2E4F2EE4E3F2E19B
:10DD7E007E2E8F2EE72DF82DA32DB42DED93FC9333
:10DD8E00E2E0F0E03E0E4F1EE72DF82DEF5FFE4F66
:10DD9E007E2E8F2EEEEFF1E23E164F0610F00C9413
:10DDAE00D96EE8CFE0E0F2E03E2E4F2EE4E3F2E152
:10DDBE007E2E8F2EA32DB42D5D906C90751486043F
:10DDCE0011F40C94EC6EE1E09E2EE2E0F0E03E0EDB
:10DDDE004F1EE72DF82DEF5FFE4F7E2E8F2EEEEFAE
:10DDEE00F1E23E164F0610F00C94FE6EE3CFE0E02B
:10DDFE00F2E03E2E4F2EA32DB42DE0E0F0E0ED9399
:10DE0E00FC93E2E0F0E03E0E4F1EEEEFF1E23E1626
:10DE1E004F0610F00C94146FEECF0E945E78E4B7AC
:10DE2E00E093D40F992011F00C94216FE1E0E09370
:10DE3E00BB0F03C0E8ECE093BB0FE0E0E5BFE5BF2E
:10DE4E00E0E8E0936100E0E0E0936100E3BF0E9450
:10DE5E00D60B0E94930C7894E1E0E0934517A6E868
:10DE6E00B0E00E9450BB9F01EAE3FCE5E217F30726
:10DE7E0011F40C94F96FA6E8B0E00E9468BBACE711
:10DE8E00B0E0E9E1F1E00E9468BBAEE7B0E0E8EE99
:10DE9E00F3E00E9468BBA0E8B0E0E1E0F0E00E9491
:10DEAE0068BBA2E8B0E00E9468BBA4E8B0E0E8EE70
:10DEBE00F3E00E9468BBECEDF6E060E070E00E94DB
:10DECE003FBBDE0115960E94991BE0E0EA83FE013E
:10DEDE003196FA93EA93E8E8F0E0FA93EA93A0E237
:10DEEE00B0E00E94E61AA6EBB0E0E1E00E9470BB43
:10DEFE00A7EBB0E0E5E00E9470BBA8EBB0E0E0E07D
:10DF0E000E9470BBA9EBB0E0E3E00E9470BBAAEBED
:10DF1E00B0E0E0E00E9470BBA8EAB0E0E1E00E9451
:10DF2E0070BBA9EAB0E00E9470BBAAEAB0E00E9402
:10DF3E0070BBABEAB0E0E0E00E9470BBACEAB0E0D0
:10DF4E00E1E00E9470BBADEAB0E0E0E00E9470BB81
:10DF5E00AEEAB0E0E1E00E9470BBAFEAB0E0E0E014
:10DF6E000E9470BBA0EBB0E0E1E00E9470BBA1EBA1
:10DF7E00B0E0E0E00E9470BBA2EBB0E00E9470BB8C
:10DF8E00A3EBB0E00E9470BBA4EBB0E0E1E00E9416
:10DF9E0070BBACEBB0E0EFEFFFEF0E9468BBAEEBF7
:10DFAE00B0E0E0E00E9470BBA2EDB0E0E4EFF2E082
:10DFBE000E9468BBA0EDB0E0EAE7F1E00E9468BB0A
:10DFCE00AEECB0E0EDEBF0E00E9468BBACECB0E084
:10DFDE00ECE4F0E00E9468BBAAECB0E0E6E2F0E010
:10DFEE000E9468BB0E9431250E94300EA1E00E9463
:10DFFE006525A1E00E94532C0E94CB7DEEABAEA90D
:10E00E00A13010F40C940F70E953E093BF0F03C0CE
:10E01E00E1E0E093BF0F0E94832DEFABE03011F4EF
:10E02E000C942670E2E0E09345170E94A62DA92DD0
:10E03E000E94FB2DEEABAEA90E94C02FFCCFE3E0F9
:10E04E00E09345170E9438360E94EC37A9EAB0E0FB
:10E05E000E9454BBE883A881A33011F00C943A704F
:10E06E000E9405400CC0A881A13011F40C9444709C
:10E07E00A23011F40C94447002C00E946C3B0E94BA
:10E08E006C600E941A440E947F740E94A1880E94B4
:10E09E00E5510E94390F0E94B54D0E94D77FE4E0F2
:10E0AE00E09345170E9478780E94D9790E948B7868
:10E0BE00E5E0E09345170E94E1730E94A9510E948A
:10E0CE003A570E9460A3A4E00E94C80EA3E00E94EB
:10E0DE00C80EE1E0E0934117E0E0E0933E17E093D5
:10E0EE003F17E0934017E1E0E0934217E0E0E09342
:10E0FE004417E0934317E0934C17ACE00E94820E56
:10E10E00E2E0EA93E5E0EA93E3E0EA93E0E0EA9303
:10E11E00A0E00E947D13E1E0E0939418E0E0E0932C
:10E12E0095187894A1E00E94820EA8E00E94C80E75
:10E13E000E94700EE03011F00C94A8700E94300E08
:10E14E007894E0E0E0934617E0934717E093481782
:10E15E00E0934917A3E00E94E40E8F01ABEAB0E012
:10E16E000E9454BBEFABE03011F40C94C770E0E0AA
:10E17E00E0933F17E0914617E260E093461703C025
:10E18E00E1E0E0933F170A30E0E01E0710F00C9438
:10E19E00D870E0E0E0933F17E0914617E460E0931B
:10E1AE004617A4980E944125EFABE03011F40C9471
:10E1BE00E870E0E0E0933F17E0914617E860E093E7
:10E1CE0046170E949760EFABAFA9A13010F40C94E4
:10E1DE00F670E0E0E0933F17EFA9E0934917A091A6
:10E1EE0095180E942F52EFABE03011F40C9407718A
:10E1FE00E0E0E0933F17E0914617E062E0934617A8
:10E20E000E94AB74EFABE03011F40C941671E0E0A9
:10E21E00E0933F17E0914617E064E09346170E94A3
:10E22E006268EFABE03011F40C942571E0E0E093FE
:10E23E003F17E0914617E068E09346170E943B6552
:10E24E00EFABE03011F40C943471E0E0E0933F1743
:10E25E00A7E4B7E1EC91E160EC930E941B44EFABB5
:10E26E00E03011F40C944371E0E0E0933F17A7E423
:10E27E00B7E1EC91E260EC930E94E788EFABE030FF
:10E28E0011F40C945671E0E0E0933F17A7E4B7E168
:10E29E00EC91E460EC93E1E0E0934C1703C0E0E016
:10E2AE00E0934C17A09195180E949778EFABE03051
:10E2BE0011F40C946A71E0E0E0933F17A7E4B7E124
:10E2CE00EC91E860EC930E94AB36EFABE03011F4CA
:10E2DE000C947971E0E0E0933F17A7E4B7E1EC917D
:10E2EE00E061EC93A9EAB0E00E9454BBE883A881F8
:10E2FE00A33011F00C9493710E942940EFABE030E3
:10E30E0011F40C949271E0E0E0933F17A7E4B7E1AB
:10E31E00EC91E062EC9319C0A881A13011F40C9439
:10E32E009D71A23011F40C949D710FC00E949E3B02
:10E33E00EFABE03011F40C94AC71E0E0E0933F17DA
:10E34E00A7E4B7E1EC91E064EC930E94BC4DA09180
:10E35E0095180E94EA7FEFABE03011F40C94BF7178
:10E36E00E0E0E0933F17A7E4B7E1EC91E068EC93AF
:10E37E000E944F7DA0914C170E949E94EFABE0300F
:10E38E0011F40C94D271E0E0E0933F17A8E4B7E1EA
:10E39E00EC91E068EC930E94AA25EFABE07111F4CA
:10E3AE000C94E371E0E0E0933F17A8E4B7E1EC9141
:10E3BE00E160EC930E94C888EFA9E07211F40C940E
:10E3CE00F871E0E0E0933F17A8E4B7E1EC91E2606A
:10E3DE00EC930E948378E23010F00C94F8710E9456
:10E3EE00C888EFA9E07411F40C940572E0E0E09394
:10E3FE003F17A8E4B7E1EC91E460EC93EFA9E07865
:10E40E0011F40C941272E0E0E0933F17A8E4B7E128
:10E41E00EC91E860EC930E942E53EFABE03011F4D8
:10E42E000C942172E0E0E0933F17A8E4B7E1EC9181
:10E43E00E061EC930E9483A3EFABE03011F40C94F7
:10E44E003072E0E0E0933F17AAE4B7E1EC91E160AF
:10E45E00EC930E94BF64EFABAFA9A13010F40C9403
:10E46E003C72E853E093CF0F03C0E1E0E093CF0F8F
:10E47E00EFA9E17011F40C944C72E0E0E0933F17B9
:10E48E00A8E4B7E1EC91E061EC93EFA9E27011F42E
:10E49E000C945972E0E0E0933F17A8E4B7E1EC91D9
:10E4AE00E062EC93EFA9E47011F40C946672E0E074
:10E4BE00E0933F17A8E4B7E1EC91E064EC93E091B0
:10E4CE003F17E03011F00C946F72A4E00E94C80E5A
:10E4DE00A0914017A43011F00C947A72E1E0F0E0B4
:10E4EE00E8AFF9AF0FC0A0914017A13011F00C9416
:10E4FE008572EEE1F0E0E8AFF9AF04C0E3E0F0E0E2
:10E50E00E8AFF9AFA4E00E94E40E8F01E8ADF9ADDB
:10E51E000E171F0710F40C949B72A0E00E94D525D5
:10E52E000E944B7300E010E00E9447510E94AF7FA3
:10E53E00A1E00E94532CACE00E94990E8F0105368B
:10E54E00E0E01E0710F40C94AF72ACE00E94820E55
:10E55E00EFCD9901AA01EA96FFCFE0E0E3BF0E945A
:10E56E00000C0E94B173E1E0E0934217E093401774
:10E57E00AEEDB6E080E090E00E94C6B30E94A188A6
:10E58E000895E0E0E3BF0E942E0C0E94B173E1E01B
:10E59E00E0934217E2E0E0934017ABEEB6E080E086
:10E5AE0090E00E94C6B30895E0E0E3BF0E945C0CC9
:10E5BE000E94B173E2E0E0934217E3E0E09340176C
:10E5CE00A9EFB6E080E090E00E94649308950A936C
:10E5DE00E0E0E3BF0E948A0CE3E0E0934217E4E040
:10E5EE00E09340170E949973E0919618EF5FE093C5
:10E5FE009618E0919718EF5FE0939718A0919618F0
:10E60E00A93310F40C941D73A6E0B7E080E090E0FF
:10E61E000E946493E7E0E0934017A1E00E946F250B
:10E62E00E0E0E09396180E94E6640CC0A091961864
:10E63E00A83310F40C942973A1E00E946F25E6E034
:10E64E00E09340170E94BF640E2F013010F40C941B
:10E65E003D730E942993AEE1B7E080E090E00E9406
:10E66E00C6B3E5E0E09340170E94F0640991089567
:10E67E0008950E9480110895089508950E94CAB3C6
:10E68E0008950E94CAB30895F894A4E2B7E080E01A
:10E69E0090E00E946493A1E00E948B25A0E00E946E
:10E6AE006525A0E00E946F25E0E0E0934017E0931F
:10E6BE0041170E9482600E94DA370E94880F0E94E2
:10E6CE007B0D0E947C120E9418140E9405160E9457
:10E6DE006817E0E9E0BF0E94790B0E947E0D0E9450
:10E6EE004325A0E00E94132CA0E00E94532CE0E8EA
:10E6FE00E0936100E8E0E0936100A2E00E94DB0B92
:10E70E00A2E00E94090CA2E00E94370CA2E00E9437
:10E71E00650CE0E0EBB9EAB978940E9421A50E945D
:10E72E0025A508950E94D7B30E94E173A4E00E942C
:10E73E00C80EE0E0E0934117E09343170E94300EBD
:10E74E0078940E942993AFE2B7E080E090E00E94B7
:10E75E00649308950E94D7B3A1E00E9465250E949C
:10E76E00E1730E94D77F0E9438360E94EC37A1E0F9
:10E77E000E94820EA4E00E94C80EA1E00E94532CBB
:10E78E000E94E5510E94300D0E94390FE1E0E093A6
:10E79E004117E0E0E09343170E947E0D0E94300E79
:10E7AE0078940E942993AAE3B7E080E090E00E945B
:10E7BE00649308950E94ADB90E94C9B20E2F023023
:10E7CE0010F40C94EF73A6EBB0E0E1E00E9470BB86
:10E7DE000E94CEB21E2F113010F40C94FB73193020
:10E7EE0010F00C94FB7306C0A7EBB0E0E2E00E94C1
:10E7FE0070BB12E00E94D3B22E2F2F3411F40C9462
:10E80E0011742E3411F40C941174253411F40C94EB
:10E81E00117401C006C0A8EBB0E0EEE40E9470BB1C
:10E82E002EE40E94CEB2E73011F40C942374A7EBC1
:10E83E00B0E0E7E00E9470BB0E94D3B2EE3411F458
:10E84E000C942E74A8EBB0E0EEE40E9470BBE12FA6
:10E85E00E23011F00C94357440E025C0E33011F035
:10E86E000C943B7441E01FC0E43011F00C944174E1
:10E87E0042E019C0E53011F00C94477443E013C028
:10E88E00E63011F00C944D7444E00DC0E73011F0F9
:10E89E000C94537445E007C0E83011F00C94597491
:10E8AE0046E001C040E0E22FE53411F00C946174B3
:10E8BE0031E00DC0EF3411F00C94677432E007C0F4
:10E8CE00EE3411F00C946D7430E001C030E00E9413
:10E8DE0095AE0E94F511A1E00E94F7250E943265C7
:10E8EE000E9459680E945CAA0E94B4B925960895A8
:10E8FE000A930E94E173E1E0E093EF180E948D12FB
:10E90E0000E0043510F00C949474E02FF0E0E8561B
:10E91E00F74EA0E0A0830F5FF4CFE0E0E093EC1899
:10E92E00E093ED18E093EE180E94652BE093F0183B
:10E93E000E947F2BE093F118E0E0E0938C19A6E0A3
:10E94E000E94C80E099108950E94AFB900E00E947E
:10E95E003E750E2FA2E0B0E00E940A0E013011F0BB
:10E96E000C94D274E1E0E093ED180E94BE751E2F58
:10E97E00A12F0E94C677103011F00C94C9740E941A
:10E98E00CE7601C020E00E94FA76E0E0E093ED182A
:10E99E000E94C2AA08950E94F4770E2F003011F43F
:10E9AE000C94DC740E94C2AA08950E94E1AB0895F3
:10E9BE000A930A2F000F000F000F087100934319DE
:10E9CE00E0914219E260E0934219099108950A9389
:10E9DE000A2F0295007F000F007600934319E091F5
:10E9EE004219E460E0934219099108950E94CEA75E
:10E9FE0040934B19E091FA18F091FB18E0934719E8
:10EA0E00F0934819E091FC18F091FD18E093491924
:10EA1E00F0934A19E42FF0E0FA93EA93A0E4B0E001
:10EA2E000E94E7211E2F00E0011710F00C942B75A9
:10EA3E00ACE4B9E1E02F0E946AA9D9010E94B0A905
:10EA4E00D001EC930F5FF0CF0E94B4B926960895D3
:10EA5E000A930A2F043610F00C943975E1E0E09316
:10EA6E008C1903C0E0E0E0938C19099108950E947F
:10EA7E00AFB90E9417138F01112312F00C944A752F
:10EA8E000E94E3B308950635E0E01E0714F40C94DB
:10EA9E0053750E94E3B3089500240016010614F086
:10EAAE000C94A17520E0243510F00C946675E22FBD
:10EABE00F0E0E856F74EA0E0A0832F5FF4CFE8E930
:10EACE00F8E1FA93EA93A4E5B0E00E941A130093DA
:10EADE00EC18E091EC18A0918D19EA1711F40C9432
:10EAEE007F75ACE10E94820EE091EC18E0938D19D7
:10EAFE00A091EC18AA3010F40C948C75A091981873
:10EB0E00AF3311F00C948C7501C003C00E94EAB3B0
:10EB1E000895A091EC18A63410F40C949D75A09154
:10EB2E009818AD3311F00C949D7501C003C00E946E
:10EB3E00EAB30895ACE10E94990E8F010530E0E032
:10EB4E001E0714F40C94B275A0918D19A13010F417
:10EB5E000C94B27501C008C00E948D12E0E0E093E3
:10EB6E008D190E94C7AA08950E94E1AB08952297BD
:10EB7E000E947AA9E0E0E093F218E0E0F0E0E09382
:10EB8E00F318F093F418E093F518F093F618E09359
:10EB9E00F718F093F818EFEFE093F918E0E0F0E0D3
:10EBAE00E093FA18F093FB18E093FC18F093FD181D
:10EBBE00EFEF0E94F1B3E0E0E093011940E050E086
:10EBCE004034E0E05E0710F00C94F675E2E0F9E1F7
:10EBDE00E40FF51FA0E0A0834F5F5F4FF1CFA09130
:10EBEE009818AD3311F40C940176AF3311F40C94E4
:10EBFE00017601C005C0E1E00E94B3B928960895E0
:10EC0E00A0919818AD3311F00C941476A091EC18D5
:10EC1E00A63410F00C9414760EC0A0919818AF3351
:10EC2E0011F00C942176A091EC18AA3010F00C94EF
:10EC3E00217601C005C0E2E00E94B3B9289608957E
:10EC4E00E0E0EF83A0919818AD3311F00C9432767A
:10EC5E00E0E4EF8308C0A0919818AF3311F00C9444
:10EC6E003A76E4E0EF83EF81EA5FEE83E150F0E085
:10EC7E00E856F74EE081EA93EF81E250F0E0E85675
:10EC8E00F74EA0810E9449209F01EE81E250EE8353
:10EC9E0040E050E0EE810E94C5AC10F00C9462761C
:10ECAE00A8E9B8E1A40FB51FEC91F0E00E0F1F1FFD
:10ECBE004F5F5F4FEFCF2017310711F40C946E7634
:10ECCE0040E050E0E4E00E94B3B928960895A09188
:10ECDE009818AD3311F00C947776E2E0E093F218C9
:10ECEE00A0919818AF3311F40C948076E1E0E09384
:10ECFE00F218E1E0F0E0E093F318F093F418A5EFCA
:10ED0E00B8E1E0919918F0E0ED93FC93A7EFB8E12C
:10ED1E00E0919B18F0E0ED93FC93E0E0E093F9189E
:10ED2E00AAEFB8E1E0919A18F0E0ED93FC93E09130
:10ED3E00F718F091F818E093FC18F093FD18E0E046
:10ED4E000E94F1B3EF81E0930119A0910119A13452
:10ED5E0010F40C94B576E0E4E093011940E050E035
:10ED6E00E09101190E94C5AC10F00C94CB76E2E054
:10ED7E00F9E1E40FF51FDF01FA01E456F74EE081E9
:10ED8E00EC934F5F5F4FECCF0E94A4AC08950A93B3
:10ED9E0000E0E091F518F091F618FA93EA93E091FD
:10EDAE00F718F091F818FA93EA93E0910119EA93A3
:10EDBE00A2E0B9E10E9464680E2FA02F0E94DF74BA
:10EDCE0000E0E091FA18F091FB18FA93EA93A09103
:10EDDE00FC18B091FD180E943D650E2FA02F0E94C9
:10EDEE00EE7409910895EF9765970E94ADB9E09181
:10EDFE004219E03011F00C940A77E0E00E94B4B9A9
:10EE0E00EF966A960895E0E0EF83E887AF81B885C4
:10EE1E00A035E0E0BE0710F00C941C770E94FAB308
:10EE2E00E0E0EC930E94FEB3F1CFE0918C19E0305C
:10EE3E0011F00C942677EFE5E98708E003C0EDE5C5
:10EE4E00E98700E4A0914B190A1710F00C94317762
:10EE5E0000934B19E0914319EA87E0E0EF83E887CE
:10EE6E00E0914B190E948AB110F00C945077EF810B
:10EE7E00F8853296ED83FE830E9404B40F01ECE414
:10EE8E00F9E10E9403A7EC91D001EC930E94FEB32E
:10EE9E00E7CFED81FE813196ED83FE83EF83F88718
:10EEAE00E02FEE5F0E948AB110F00C9465770E94FD
:10EEBE00FAB3E0E0EC930E94FEB3F2CFE02FF0E065
:10EECE0032961E2F2F2F30E040E0E0E0EF83E887F0
:10EEDE00AF81B885A117B20710F00C947F770E940E
:10EEEE00FAB3EC91F0E03E0F4F1F0E94FEB3F0CF4D
:10EEFE00E12FF22F0E9404B43083342F4427E12FE8
:10EF0E00F22F31960E9404B430831E5F2F4FA985D5
:10EF1E00AD3511F00C949977AA85A03211F00C94AE
:10EF2E00997701C004C0E1E0F0E0EF83F887E4E4F4
:10EF3E00F0E0E117F20711F40C94AD77ECE0F0E09D
:10EF4E00E117F20711F40C94AD7707C00E948AAE58
:10EF5E00A12FB22F0E94671303C0E0E0EF83E88772
:10EF6E000E94E6ABE0E0E0934219EF81F885EF8373
:10EF7E00F887E1E00E94B4B9EF966A9608951A9365
:10EF8E000A931A2F10934319E3E6E0934419E09382
:10EF9E004519E0E0E0934B1900E0003410F00C94BA
:10EFAE00E077ACE4B9E1EE27A00FBE1FEC930F5F44
:10EFBE00F4CFE0914319E03011F00C94EC77E0912E
:10EFCE004219E160E093421905C0E0914219E161F6
:10EFDE00E0934219099119910895A091EC18AE3061
:10EFEE0010F40C945C78A0919818A23011F00C9447
:10EFFE004F78A0919918A13511F00C944F78A091EB
:10F00E009A18A33411F00C944F78A0919B18A23249
:10F01E0011F00C944F78A0919C18A53511F00C941A
:10F02E004F78A0919D18AB3511F00C944F78A091AC
:10F03E009E18AD3211F00C944F78A0919F18A43306
:10F04E0011F00C944F78A091A018A23411F00C94EA
:10F05E004F78A091A118AD3411F00C944F78A09177
:10F06E00A218A83511F00C944F78A091A318A23DC8
:10F07E0011F00C944F78A091A418A33D11F00C94AC
:10F08E004F78A091A518A33011F00C944F7801C0C1
:10F09E000CC0A4E4B7E080E090E00E9464930E946C
:10F0AE0027AB0E94AC0CE1E00895E0E008950E94C9
:10F0BE00ACB90DE110E04AEB5FE020E030E0DA01A0
:10F0CE00E0E0EC934F5F5F4FF90131969F01E0173F
:10F0DE00F10710F00C947478F2CF0E94B3B9269613
:10F0EE000895E0E0E0938E19E0938F190E94299322
:10F0FE00E3E6E09390190895E0918F190895E2E008
:10F10E00E0938F19E0E008950E9409B4A0E00E94F8
:10F11E006B27A0E00E949C27A0E00E9486270895FE
:10F12E00AA9325970E94ACB9EB85E03011F40C94AC
:10F13E00A3780E940DB40895E0918E19E03011F07D
:10F14E000C94AC780E9412B415C0E13011F00C94FE
:10F15E00B3780E9418B40EC0E23011F00C94B87857
:10F16E0009C0E33011F00C94BD7804C0E43011F006
:10F17E000C94C178A0918E19AF5FA0938E19A53013
:10F18E0010F40C94CD78E0E0E0938E190E94358B4C
:10F19E00E03011F40C941079A1E9B9E10E94128BC0
:10F1AE005E2FE0918F19E03011F40C94E778513016
:10F1BE0010F40C94E7785A3010F00C94E77801C0F4
:10F1CE0015C0E0E0E0938F19A0E00E94A4630E94B6
:10F1DE00A3B20E9429930E9409B4ACE5B7E080E087
:10F1EE0090E00E9464930E94548B13C0533011F030
:10F1FE000C940779E1E0E0938F190E94548B09C0BB
:10F20E00543011F00C941079E2E0E0938F190E94C3
:10F21E00548BA0918F19A13011F00C941E790E947D
:10F22E0029930E94C657E0E0E0938F19B8C0A091D1
:10F23E008F19A23011F00C944C790E942993ABE6F1
:10F24E00B7E080E090E00E946493A8E8B7E080E029
:10F25E0090E00E946493AFEAB7E080E090E00E94F5
:10F26E006493AEE00E94C80EE0918F19EF5FE093B9
:10F27E008F190E94EC370E94D33DA1E00E941A3EE6
:10F28E000E94BF630E949DB28AC0A0918F19A330C5
:10F29E0011F00C94C079AEE00E94E40E9F0125316E
:10F2AE00E0E03E0710F40C946179E0918F19EF5F66
:10F2BE00E0938F190E94173E4E2F483011F00C9498
:10F2CE006A790E943E3EE0919019E41711F40C9475
:10F2DE009279409390190E942993483011F00C9422
:10F2EE007E79A4ECB7E080E090E00E946493493010
:10F2FE0011F00C948879A6EDB7E080E090E00E94C2
:10F30E0064934A3011F00C949279AFEDB7E080E03F
:10F31E0090E00E9464930E9493AFFE013B960E9480
:10F32E003DA9FE013D96FA93EA93DE011E960E94D8
:10F33E00123F4E2F403011F00C94BF790E811127E1
:10F34E00AFEFA09FF001A19FF00D8F01EF81F0E0D4
:10F35E000E0F1F1FE5EFF7E060E070E00E943FBB6D
:10F36E00D8010E943DAD0E944893AEE00E94C80EA7
:10F37E0016C0A0918F19A43011F00C94D679A0E08C
:10F38E000E94A4630E94A3B20E9409B4A0E0B8E058
:10F39E0080E090E00E946493E0E0E0938F190E9479
:10F3AE000DB40895E6970E94ADB900E00E941EB418
:10F3BE000E9448930E941EB4AEE0B8E080E090E058
:10F3CE000E946493A091BB0FA13011F00C94F679BA
:10F3DE00A7E2B8E080E090E00E94649306C0AEE23F
:10F3EE00B8E080E090E00E9464931091BF0F11305E
:10F3FE0011F00C94097AAEE3B8E080E090E00E9440
:10F40E00649306C0EAE4F8E060E070E00E9422B483
:10F41E000E94047D1E2F113010F40C941E7A01E010
:10F42E00EAE5F8E060E070E00E9422B406C0A5E6CE
:10F43E00B8E080E090E00E9464930E94387D1E2F19
:10F44E00103011F40C94337A01E0ECE6F8E060E051
:10F45E0070E00E9422B406C0A7E7B8E080E090E01A
:10F46E000E9464930E9481642E2F203011F40C941C
:10F47E00467AAEE7B8E080E090E00E9464930E9486
:10F48E0097643E2F303011F40C94537AA1E9B8E012
:10F49E0080E090E00E9464930E94AD644E2F403055
:10F4AE0011F40C94607AA4EAB8E080E090E00E9437
:10F4BE006493203011F00C946D7A303011F00C946E
:10F4CE006D7A403011F00C946D7A01C006C0A9EB34
:10F4DE00B8E080E090E00E9464930E941153EF83A5
:10F4EE00F887AF81B8850E949D7D1E2F103011F4D4
:10F4FE000C94897A01E0E2ECF8E060E070E00E94A2
:10F50E0022B406C0A5EDB8E080E090E00E946493BE
:10F51E000E942153EF83F887AF81B8850E946C7DDE
:10F52E001E2F103011F40C94A47A01E0E4EEF8E0F2
:10F53E0060E070E00E9422B406C0A3EFB8E080E065
:10F54E0090E00E9464930E949B7C1E2F103011F459
:10F55E000C94B97A01E0EEEFF8E060E070E00E9402
:10F56E0022B406C0ABE0B9E080E090E00E94649364
:10F57E000E94C47C1E2F103011F40C94CE7A01E040
:10F58E00E4E1F9E060E070E00E9422B406C0A1E27E
:10F59E00B9E080E090E00E9464930E945E7C1E2F92
:10F5AE00103011F40C94E37A01E0EAE2F9E060E045
:10F5BE0070E00E9422B406C0ADE3B9E080E090E0B6
:10F5CE000E9464930E948B571E2F123010F40C94DD
:10F5DE00137B01E0ECE4F9E060E070E00E9422B4FD
:10F5EE0011FF02C00E9426B415FF02C00E942CB467
:10F5FE0017FD03C016FD01C003C00E9432B40BC03C
:10F60E0012FD03C014FD01C002C00E9438B413FFE6
:10F61E0002C00E943EB406C00E9444B410FF02C055
:10F62E000E944AB40E943D641E2F103011F40C94B7
:10F63E002B7BE8ECE093CA0F01E0AAEBB9E080E087
:10F64E0090E00E94649309C0E1E0E093CA0FA7EC3A
:10F65E00B9E080E090E00E9464930E945F641E2FE8
:10F66E00103011F40C94457BE8ECE093CB0FA4ED35
:10F67E00B9E080E090E00E94649309C0E1E0E0937D
:10F68E00CB0FA0EEB9E080E090E00E9464930E9460
:10F69E00EC370E940A3E1E2F113010F40C94627B40
:10F6AE00E8ECE093C40F01E0ACEEB9E080E090E04E
:10F6BE000E94649309C0E1E0E093C40FA6EFB9E0A5
:10F6CE0080E090E00E946493E1E0E093D30FE0E0ED
:10F6DE00E093C70F0E94C888ADE10E94820EADE193
:10F6EE000E94990EED83FE831091C70F0E94E7884A
:10F6FE00AD81BE81A039E1E0BE0710F00C948C7B89
:10F70E00103011F00C948C7B01C001C0E8CF0E9428
:10F71E002993113011F00C949B7BADEFB9E080E092
:10F72E0090E00E94649307C001E0EAE0FAE060E036
:10F73E0070E00E9422B4ABE1BAE080E090E00E945B
:10F74E006493A0E00E94C3811E2F0E94267FA09189
:10F75E00C40FA83C10F40C94B87BE8ECE093C50FF2
:10F76E0039C0E0E0E093C50F0E94D33DA1E00E94B6
:10F77E001A3E0E943E3EADE10E94820EADE10E9415
:10F78E00990EED83FE831091C50F0E94AB360E9439
:10F79E009E3BAD81BE81A83EE3E0BE0710F00C9407
:10F7AE00DD7B103011F00C94DD7B01C001C0E6CF83
:10F7BE00113011F00C94EA7BA7E3BAE080E090E000
:10F7CE000E94649307C001E0E7E4FAE060E070E0B5
:10F7DE000E9422B4003011F40C94FF7BA7E5BAE02E
:10F7EE0080E090E00E946493A1E00E946F2509C022
:10F7FE00A6E6BAE080E090E00E946493A1E00E9449
:10F80E006525E1E0E093D50F0E9448930E948AAEF1
:10F81E000E9428B2E8ABE0E7FAE060E070E00E94F8
:10F82E0050B40E94991BE6E8FAE060E070E00E9496
:10F83E0050B40E949C930E948AAE0E9428B2E8ABFC
:10F84E00E2E9FAE060E070E00E9450B40E94991B79
:10F85E00EFE9FAE060E070E00E9450B40E949C93E1
:10F86E000E948AAE0E9428B2E8ABEBEAFAE060E0B2
:10F87E0070E00E9450B40E94991BE8EBFAE060E041
:10F88E0070E00E9450B40E949C930E944893E1E065
:10F89E00E093C80FE0E0E093CE0F0E942993A7E01B
:10F8AE000E94C80EE02F0E94B4B9EB9608951A93E9
:10F8BE000A9300E0E0E0E093C60F0E9466B21E2FAE
:10F8CE00113010F40C948C7C0E94FE27E03011F461
:10F8DE000C94727C01E0A1E00E94C4270E9455B4F2
:10F8EE0011F00C947B7C02E00E9497B20E9455B4FA
:10F8FE0011F00C94837C03E0A0E00E94DA270E94B2
:10F90E0055B411F40C948C7C04E0013010F40C947A
:10F91E00947CE8ECE093C60F03C0E1E0E093C60FE1
:10F92E00E02F0991199108950A93EFEFFFE0FA93F2
:10F93E00EA93A9E70E945DB4093711F40C94AD7CEB
:10F94E00E8ECE093BC0FE1E009910895EFEFFFE0E2
:10F95E00FA93EA93A6E80E945DB4063811F40C946B
:10F96E00BE7CE8ECE093BC0FE1E009910895E1E084
:10F97E00E093BC0FE0E0099108950A93A0E00E9485
:10F98E008B250E940CAAEEEFFFEF0E94FDB1A2E1C3
:10F99E000E94CA830E2F0E942BAB0E9465B40231C7
:10F9AE0011F40C94E07CE8ECE093BD0FE1E00991DA
:10F9BE000895EEEFFFEF0E94FDB1A7E30E94CA8308
:10F9CE000E2F0E942BAB0E9465B4073311F40C94DA
:10F9DE00F67CE8ECE093BD0FE1E009910895E1E0DB
:10F9EE00E093BD0FE0E0099108950E943DB00895A7
:10F9FE00AEE1B0E00E940A0E089562970A93DE010E
:10FA0E0011960E94BD4D0E2F023010F40C941D7DE8
:10FA1E000E945CAA0E9487AAAFE10E949C4F0E949E
:10FA2E005CAADE0111960E94BD4D0E2F003011F022
:10FA3E000C94257DE1E0E093BE0F0FC0013011F074
:10FA4E000C942D7DE8ECE093BE0F07C0023011F050
:10FA5E000C94347DE9ECE093BE0FE02F08816396A1
:10FA6E000895A8970A93FE017796FA93EA93DE011A
:10FA7E0013960E946B500E2F003011F40C94487D9B
:10FA8E0004C0E02F0881A99608950881A9960895CB
:10FA9E000E94AEB920E0A1E00E9479250E94FF7C71
:10FAAE000E9412B43E2F313010F40C945F7D21E091
:10FABE000E9418B43E2F313010F40C94677D21E073
:10FACE00E22F0E94B5B9249608950E9470B40832B0
:10FADE00E3E21E0710F40C947B7D0939EAE31E075E
:10FAEE0010F00C947B7D05C021E0E8ECE093CC0F88
:10FAFE0018C00033EAE21E0710F00C948B7DE9EC7F
:10FB0E00E093CC0F22E00DC0003CEBE21E0710F09C
:10FB1E000C94957DE4E6E093CC0F03C0E1E0E09316
:10FB2E00CC0FE22F0E94B6B9259608950E9470B4AC
:10FB3E000832E0E01E0710F40C94AC7D0530E1E0D5
:10FB4E001E0710F00C94AC7D05C021E0E8ECE093AC
:10FB5E00CD0F15C00135E0E01E0710F40C94BE7DEC
:10FB6E000C3DE0E01E0710F00C94BE7D05C022E0B7
:10FB7E00E9ECE093CD0F03C0E1E0E093CD0FE22F6F
:10FB8E000E94B6B9259608951A930A9300E00E9432
:10FB9E000727E03011F40C94D97DA0E00E94FB26DB
:10FBAE000E94FF7CA1E00E94FB260E94FC7C0E942A
:10FBBE000D27E03011F00C94E57D01E0013010F4DA
:10FBCE000C94ED7DE02F0991199108950E94292C36
:10FBDE00E03011F40C94F87DA0E00E94132C0E94EA
:10FBEE00FF7CA0E00E94132C0E94FC7CA1E00E94EE
:10FBFE00132C0E94FC7C0E94B42CE03011F00C946B
:10FC0E00097E02E0013010F40C94117EE02F099170
:10FC1E0019910895A0E00E9478B411F40C94187E06
:10FC2E0003E0A1E00E9478B411F00C941F7E03E073
:10FC3E00A0E00E9485B411F40C94267E03E0A1E0AE
:10FC4E000E9485B411F40C942D7E03E0013010F463
:10FC5E000C94357EE02F099119910895A0E00E9431
:10FC6E0092B411F00C943C7E04E0A1E00E94132C9F
:10FC7E00A1E00E9486270E94FC7CA1E00E9492B423
:10FC8E0011F40C944B7E04E0013010F40C94537E6E
:10FC9E00E02F0991199108950E947727E03011F411
:10FCAE000C945E7EA0E00E946B270E94FF7CA0E079
:10FCBE000E949AB411F40C94657E05E0A1E00E94B6
:10FCCE009AB411F00C946C7E05E0013010F40C9493
:10FCDE00747EE02F0991199108950E94A827E030B3
:10FCEE0011F40C947F7EA0E00E949C270E94FF7C62
:10FCFE00A0E00E94A2B411F40C94867E06E0A1E06E
:10FD0E000E94132CA1E00E94A2B411F00C94907EDC
:10FD1E0006E0013010F40C94987EE02F09911991B1
:10FD2E0008950E94952AE03011F40C94A37EA0E071
:10FD3E000E947F2A0E94FF7CA0E00E947F2A0E94E0
:10FD4E00FC7C013010F40C94B07EE02F09911991D7
:10FD5E0008950E94862CE03011F40C94BB7EA0E036
:10FD6E000E947A2C0E94FF7CA0E00E947A2C0E94B6
:10FD7E00FC7CA1E00E947A2C0E94FC7C0E94962CB6
:10FD8E00E03011F00C94CC7E09E0013010F40C94AC
:10FD9E00D47EE02F0991199108950E94492CE030EC
:10FDAE0011F40C94DF7EA0E00E94332C0E94FF7CA5
:10FDBE00A0E00E94332C0E94FC7CA1E00E94332C18
:10FDCE000E94FC7C0E94AB2CE03011F00C94F07E73
:10FDDE000AE0013010F40C94F87EE02F099119918D
:10FDEE000895A1E00E94532C0E94FC7C0E94692C75
:10FDFE00E03011F00C94047F0BE0013010F40C9401
:10FE0E000C7FE02F099119910895A0E00E94ABB4E8
:10FE1E0011F40C94137F0CE0A1E00E94ABB411F02E
:10FE2E000C941A7F0CE0013010F40C94227FE02F1A
:10FE3E00099119910895E02F099119910895A091B2
:10FE4E00C10FA13011F00C94457FA4ECBAE080E014
:10FE5E0090E00E946493A091C30FA13011F00C9416
:10FE6E003E7FADECBAE080E090E00E946493E8ED56
:10FE7E00FAE060E070E00E94B4B428C0A0EEBAE0F0
:10FE8E0080E090E00E946493E091C10FE83C11F095
:10FE9E000C94587FA7E7B9E080E090E00E9464934D
:10FEAE0015C0E93C11F00C94637FADEEBAE080E032
:10FEBE0090E00E9464930AC0E43611F00C946D7FBA
:10FECE00A8EFBAE080E090E00E94649308950A9350
:10FEDE00A6E0BBE080E090E00E9464930E948B5706
:10FEEE000E2F023010F40C94A17FECE4F9E060E0E8
:10FEFE0070E00E943FBBA02F0E9404B201FF02C01F
:10FF0E000E9426B405FF02C00E942CB407FD03C058
:10FF1E0006FD01C003C00E9432B40BC002FD03C037
:10FF2E0004FD01C002C00E9438B403FF02C00E944B
:10FF3E003EB40CC00E9444B400FF02C00E944AB4FA
:10FF4E000E94A84B0E9427AB0E94C65709910895A4
:10FF5E001A930A93A1E00E946BB210F40C94BE7F28
:10FF6E00A0E00E946525A1E00E94820E09C00B351B
:10FF7E00E0E01E0710F40C94C77FA1E00E946525F7
:10FF8E00099119910895A1E00E941726A1E00E94FF
:10FF9E00F7250E9495AE0E947D130E9429140895A4
:10FFAE000E94E97F0E94CA7FA1E00E947A2C0E94E3
:10FFBE000CAAE0E0E0939919E0939A19EFEFE09321
:10FFCE009B19089508950E94A2B011F40C94F27F2B
:10FFDE000E94A7B00895E0919919A0919B19EA1774
:10FFEE0011F40C94FF7FE0939B19E1E0E0939A19D2
:02FFFE00E09190
:020000021000EC
:0E0000009919E03011F00C941D80E0919A19CE
:10000E00E03011F40C9410800E94B9B440E00E94CC
:10001E00CA7F0E94BFB410F00C941A80403011F0C9
:10002E000C941A8002C00E94C7B485C0A091991981
:10003E00A13011F00C944280E0919A19E03011F445
:10004E000C942E800E94B9B40E94278140E00E9439
:10005E00ED808F01D8010E9442814E2F0E94BFB4C5
:10006E0010F00C943F80403011F00C943F8002C091
:10007E000E94C7B460C0A0919919A23011F00C94DF
:10008E006680E0919A19E03011F40C9452800E942F
:10009E00B9B40E9430810E94ED808F01D8010E9478
:1000AE007F814E2F0E94BFB410F00C9463804030BD
:1000BE0011F00C94638002C00E94C7B43CC0A091A2
:1000CE009919A33011F00C948280E0919A19E030C6
:1000DE0011F40C9475800E94B9B440E00E94D0B423
:1000EE0010F00C947F80403011F00C947F8002C091
:1000FE000E94C7B420C0A0919919A43011F00C949D
:10010E00A280E0919A19E03011F40C9491800E9433
:10011E00B9B440E00E94D0B410F00C949B804030F3
:10012E0011F00C949B8006C0E0E0E0939919E1E099
:10013E00E0939A1900C00E94A7B00895A0970E945C
:10014E00ADB900E010E020E00E945CAA0E94FE140F
:10015E00E03011F40C94D9800E94AA141E2F2F2F78
:10016E00A12FB22F0E94D8B411F40C94C180E12FAC
:10017E00F22F02C0E0E2F0E03E2F4F2F00240116D6
:10018E00020614F00C94D7800E94F9ABA32FB42F63
:10019E000E94CF140E94F9ABA32FB42F0E948A861F
:1001AE000E9429140F5F043610F00C94E580002491
:1001BE000116020611F00C94E58001C001C0C4CFF7
:1001CE00E12FF22F0E94B4B9A5960895EF972197CB
:1001DE000E94AEB900E010E00E94FE14E03011F46F
:1001EE000C9421810E94AA148F01D801E0E4F0E062
:1001FE000E945ABAF0E0E03011F40C940881F80134
:10020E0002C0E0E4F0E09F0100240016010614F0A5
:10021E000C941F81FE013496FA93EA93D9010E9441
:10022E00CF14FE013496FA93EA93D9010E948A867E
:10023E000E942914F8010E94B5B9EF9625960895EB
:10024E000E942914AAE1BBE080E090E00E94DFB496
:10025E0008950E942914A1E2BBE080E090E00E9484
:10026E00DFB408950E942914AAE2BBE080E090E07A
:10027E000E94DFB4089526970E945DA500E01B3012
:10028E00E0E02E0710F40C947A81E4E3FBE060E0EA
:10029E0070E00E943FBB2A931A930E94E4B411F4BB
:1002AE000C947A810E94A9B1A3E00E940088AD81CE
:1002BE00AC3211F00C947181EB81E053AAE0EA9F0D
:1002CE00F001AC81AE0FE0E30E944CBBEA1BE09361
:1002DE00C20F04C0EB81E053E093C20FE1E00E9435
:1002EE00B6B929960895E0E00E94B6B92996089508
:1002FE0026970E945DA500E01B30E0E02E0710F46B
:10030E000C94BE81EBE3FBE060E070E00E943FBB2B
:10031E002A931A93A0E00E94CD860E2F003011F47E
:10032E000C94BE810E94A9B1A3E00E940088AB810B
:10033E00A03311F00C94B381AC81AC3211F00C945B
:10034E00B381AD81A13311F40C94B281A53311F4B4
:10035E000C94B28101C001C007C0E1E0E093C30F6D
:10036E000E94B6B929960895E4E6E093C30FE0E043
:10037E000E94B6B929960895A2970E94ACB95A2F39
:10038E000E94D77FA4E6B0E00E940A0E00E0E0E0F3
:10039E00E093C10FA4E6B0E00E940A0E0E94EAB4F8
:1003AE000E9463AF0E942914A3E4BBE080E090E0BA
:1003BE000E94DFB410E0A8E0B0E00E940A0E0E9496
:1003CE00FE14E03011F40C9426820E94AA143E2FE3
:1003DE004F2FA32FB42F0E94D8B411F40C94FA818E
:1003EE00E32FF42F02C0E0E2F0E0EE83FF8300245F
:1003FE000316040614F00C9424820E9416B2A885EB
:10040E00B9850E94CF140E9416B2A885B9850E94A4
:10041E008A86E6E4FBE060E070E00E94EDB411F441
:10042E000C941C82E1E0E093C10F0E94F9B411F428
:10043E000C942482E1E0E093C10F0E9429141F5F07
:10044E00143610F00C943282A091C10FA03011F02E
:10045E000C94328201C001C0AECF0F5F0A3010F093
:10046E000C944082A091C10FA03011F00C944082E8
:10047E0001C001C08FCFE091C10FE03011F00C949C
:10048E004E82E8ECE093C10F0E9418B008955030F0
:10049E0011F00C94A5820E94EAB40E9463AF0E94F0
:1004AE002914ADE4BBE080E090E00E94DFB40E942E
:1004BE00FEB40E9463AF0E942914A2E5BBE080E067
:1004CE0090E00E94DFB40E94FEB40E9463AF0E94CF
:1004DE002914ACE5BBE080E090E00E94DFB40E94FE
:1004EE0003B51B9710F40C948B82E0E6FBE060E002
:1004FE0070E00E94EDB411F00C948B82E9ECE09365
:10050E00C10F0E9418B008950E94EAB40E9463AF12
:10051E000E942914A9E6BBE080E090E00E94DFB4BF
:10052E000E9403B5159710F40C94A5820E94F9B49D
:10053E0011F00C94A582E4E6E093C10F0E94EAB498
:10054E000E9463AF00E0503011F40C94AF8203E6CA
:10055E00ACE2B1E00E940A0E0E9427810E9403B510
:10056E000E9442810F5F043110F00C94CC82A09156
:10057E00C20FAC3010F40C94CB82A091C20FA032FB
:10058E0010F00C94CB8201C001C001C0E1CF0E94DB
:10059E00EAB40E9463AF0E9430810E9403B50E94AC
:1005AE007F810E94EAB40E9463AF0E9439810E944B
:1005BE0003B51B9710F40C94ED82E0E2FBE060E0D3
:1005CE0070E00E94EDB411F00C94ED82E0E00E9418
:1005DE00B3B9A896089522970E94ADB91A2F2F810C
:1005EE00388549854A933A93E1E0EA932A931A9320
:1005FE00DE011A960E9450B010F40C940B83E0E0CA
:10060E000E94B4B92A9608950D81E02F0E94B4B9C4
:10061E002A96089528970E94ADB91A2F2D853E85EA
:10062E004F854A933A93E4E0EA932A931A93DE01B4
:10063E001E960E9450B010F40C9429830E94BFA9FC
:10064E0060960895EC85FF27662777270E9407B5E9
:10065E00EB850E9410B5EA850E9410B5E9850E94CF
:10066E00C9A50E9418B50E94D6A50E94B4B960967D
:10067E0008950E94CEA700E010E0AE81BF81E6E0B3
:10068E000E94F0B98F011A930A93E0E4EA934A9319
:10069E00E1E0EA93D9010E9452110E94B4B9289662
:1006AE000895BA93AA93EF9727970E94ACB9FE01CB
:1006BE00E05BFF4F5081FE01EE5AFF4F11912081FA
:1006CE00FE01E25BFF4F0190F081E02DE887F98794
:1006DE00E0E0EE83EF832A931A93E0E4EA930E941C
:1006EE0076AAEA935A93DE011F960E9450B010F438
:1006FE000C948783E1E00E94B3B9EF966596089556
:10070E00A885B985A134E0E0BE0710F40C94A3834C
:10071E0030E040E03034E0E04E0710F00C949C8363
:10072E000E941EB53F5F4F4FF5CFE885F985E05427
:10073E00F040E887F98711C030E040E0E885F985A0
:10074E003E174F0710F00C94B1830E941EB53F5F09
:10075E004F4FF4CFE0E0E887E987EE81FF81E05C60
:10076E00FF4FEE83FF83105C2F4FA885B9850E9443
:10077E0085BB10F00C94C483AECFE0E00E94B3B9F9
:10078E00EF966596089522970E94ACB91A2F288588
:10079E0039854A855B85A5E0B0E00E94E80D1E8391
:1007AE005A934A93E1E0EA933A932A93DE011B9619
:1007BE000E9482100E2F013010F40C94EB83E1E0B6
:1007CE000E94B3B92C9608950E940DB408950E940C
:1007DE0044BB28970E94ADB939894A891B892C8957
:1007EE00ED85FE856F8578890E94BFA5ED81E9872D
:1007FE000E9433B5EA870E9433B5EB870E9433B56A
:10080E00EC872A931A93E4E0EA934A933A93DE0133
:10081E001E960E9482100E2F013010F40C941C8430
:10082E00E1E00E94B4B965960895E0E00E94B4B983
:10083E00659608950E94ACB99D014E815F81042F8B
:10084E00013410F40C942C8400E4E885F985FA93B5
:10085E00EA930A935A93E1E0EA93D9010E94821037
:10086E001E2F0E942BAB103011F40C9441840E9469
:10087E0055A70895E02F0E94B3B92A9608950E94B5
:10088E00ACB93A2F4B2F5E8110E020E00E94D6A922
:10089E00AF81B885E6E00E94F0B91E2F2F2F2A9364
:1008AE001A93E0E4EA935A93E1E0EA93A32FB42F6C
:1008BE000E9482100E2F0E942BABE02F0E94B3B924
:1008CE0029960895BA93AA93EF972F970E94ACB9E1
:1008DE00FE01E65AFF4F01911081FE01E65AFF4FCD
:1008EE000190F081E02D662777270E9436A80E949E
:1008FE003CB5662777270E94BCAF0E94C8B90E94FC
:10090E00A8AF0E943CB50E9443B540E050E00E9463
:10091E0049B5A034E0E0BE0710F00C94EF8420E05F
:10092E0030E00E9450B52E173F0710F00C94A484AF
:10093E000E9457B52F5F3F4FF4CFFE01EE5AFF4F87
:10094E00E081E770EF87E03011F40C94B284AF854C
:10095E00E8E0EA1B01C0E0E0EE8720E030E0EE8543
:10096E00D901F0E0AE17BF0710F00C94C9840E94B5
:10097E0050B5E20FF31FDE0150960E94FCAF2F5FC1
:10098E003F4FEDCFEE850E9449B5F0E0EA0FFB1F19
:10099E000E9443B51A930A930E9476AA0E9468B5E4
:1009AE000E9468B50E946EB5AF85A13010F40C940C
:1009BE00E5840E948BA5EF966D9608950E9450B522
:1009CE00E40FF51F9F010E94B3B9EF966D9608953F
:1009DE0020E030E02034E0E03E0710F00C94FC8480
:1009EE000E9457B52F5F3F4FF5CF1A930A93E0E45D
:1009FE000E9468B50E9468B50E946EB5AF85A130A1
:100A0E0010F40C940F850E948BA5EF966D960895A9
:100A1E000E9450B5E054F0400E9443B50E9450B57C
:100A2E00309711F00C942185FA010E94B3B9EF961C
:100A3E006D960895005C1F4FEE81FF816885798564
:100A4E00E05CFF4F6F4F7F4F0E9436A8405C5F4FB8
:100A5E000E940DA90E94BCAF0E9494BB10F00C9492
:100A6E00398555CF0E948BA5EF966D9608950A9302
:100A7E000A2FE4E1E09FF00109910895BA93AA9339
:100A8E00AC978CE2002470E0E4E7FBE060E00E94AB
:100A9E00BAB90E94ADB909A91AA9ED81FE81E01774
:100AAE00F10710F40C946085E0E00E94B4B9E3966F
:100ABE00089541E0E42FF0E0DE0115960E9449AD65
:100ACE002D913C910217130710F00C947485E42FAE
:100ADE00E1500E94B4B9E39608954F5F453110F08E
:100AEE000C947A85E7CFE4E10E94B4B9E3960895B9
:100AFE00BA93AA93EF9721978CE2002470E0E0EA74
:100B0E00FBE060E00E94BAB90E94ACB9FE01EA5B5C
:100B1E00FF4F01911081EEA5FFA50E9476B50E172D
:100B2E001F0710F40C94A285E0E9F1E00E94B3B91E
:100B3E00EF96299608954E815F814017510710F464
:100B4E000C94AE850E948BA5EF9629960895D80138
:100B5E000E944585EBAFF0E0DE0116960E9449AD8E
:100B6E004D915C91EBADEF5FF0E0DE0116960E94C9
:100B7E005DAE0E9476B5E41BF50BEEAFFFAFABADED
:100B8E000E943E85DE01AE5BBF4FED93FC93EBAD55
:100B9E00EF5FEAAFAAAD0E943E85DE01A05CBF4FBB
:100BAE00ED93FC93DE01AE5BBF4F0D90BC91A02D7B
:100BBE00EA1BFB0BECAFFDAFEEADFFAD309711F0C6
:100BCE000C94ED85E4E1F0E0EEAFFFAFECADFDADE2
:100BDE000E947CB5DF01CB01EEADFFAD0E947CB56E
:100BEE000E94D1BCEEABFFAB68AF79AFF801E41B4E
:100BFE00F50B0E947CB5EAABFBAB6CAB7DABEEA903
:100C0E00FFA968AD79ADAAA9BBA98CA99DA90E941F
:100C1E0083BCEAABFBAB6CAB7DAB0E94C6BB9F014A
:100C2E00FE01EE5BFF4F0190F081E02D2E0F3F1F76
:100C3E00F9010E94B3B9EF9629960895BA93AA9333
:100C4E0066970E94ACB9E0E0F0E46CE975E40E94AE
:100C5E00A8AF44EE5CE0E0E0F0E46CE17AE40E94E0
:100C6E0036A80E94BCAFE0E0F0E060E874E40E94B9
:100C7E00D1BC0E9436A80E94BCAFE0E0F0E06AE76B
:100C8E0074E40E94D1BC0E9436A8EC8DFD8D0E94AA
:100C9E007CB50E9481B5EE81FF81688579850E94C1
:100CAE0086B5EE8BFF8B688F798FAE89BF89888D65
:100CBE00998D0E940DA90E9432BCEE87FF87688B2A
:100CCE00798BAE89BF89888D998D0E94D1BC0E9487
:100CDE0081B5FA010E947CB50E9486B50E9481B54D
:100CEE00EA89FB896C897D890E94C6BBEA8FFB8FDE
:100CFE00AA8DBB8D0E947F858F0130969F010E9429
:100D0E00B3B96E9608950E9495B02E3FE1E03E076E
:100D1E0010F40C9494862EEF31E000E010E00E3FBC
:100D2E00E1E01E0710F00C94A386ACE9B9E10E9435
:100D3E006FA60F5F1F4FF3CF20939A1B30939B1B11
:100D4E005A934A93ECE9F9E1FA93EA93A0919A1B2C
:100D5E00B0919B1B0E94961A0E948DB5E456F64EDA
:100D6E00A0E0A083E0E0E0939E1BE0939F1BE09346
:100D7E009C1BE0939D1BE093A01BE093A11BE093B3
:100D8E00A21BE093A31B0E94A4AC0895AA932697DE
:100D9E00D1500E94ACB9FE01E35FFE4F0190F0818D
:100DAE00E02DEA87FB87FE01E45FFE4F10810E9473
:100DBE0092B510F00C94E786E0E00E949BB5089582
:100DCE000E94A0B50E94A7B50E94B0B50E94B7B50B
:100DDE0010F00C940687FA01DE011C96EA0FFB1F39
:100DEE00FF93EF93FA010E94A7B50E94F4A66BBF82
:100DFE00E691AF91BF91EC934F5F5F4FE7CF0E94AB
:100E0E00BCB501E040E050E0FA010E94D3A70E9479
:100E1E00C8B511F40C94148700E04F5F5F4F0E9429
:100E2E00B7B510F00C942087013011F00C94208788
:100E3E0001C001C0E9CF0E9438A6AE81BF812A173A
:100E4E003B0710F40C943087003011F00C9430876F
:100E5E0001C001C0D6CF0E94D2B511F40C943A87CE
:100E6E000E94E7B502C00E94F4B5003011F40C9454
:100E7E004587103011F40C94458701C005C00E94BF
:100E8E00FDB50E949BB50895003011F40C94538764
:100E9E00E1E00E949BB50895E0E00E949BB50895A5
:100EAE000E949BB50895AA932697D1500E94ACB983
:100EBE00FE01E25FFE4F0190F081E02DEA87FB8795
:100ECE00FE01E35FFE4F10810E9492B510F00C946C
:100EDE007487E0E00E9407B608950E94A0B50E94B4
:100EEE000CB60E94B0B50E94B7B510F00C94938763
:100EFE00FA01DE011C96EA0FFB1FFF93EF93FA0136
:100F0E000E940CB60E94F4A66BBFE691AF91BF9102
:100F1E00EC934F5F5F4FE7CF0E94BCB501E040E01E
:100F2E0050E0FA010E94D3A70E94C8B511F40C94A8
:100F3E00A18700E04F5F5F4F0E94B7B510F00C9491
:100F4E00AD87013011F00C94AD8701C001C0E9CF1F
:100F5E000E9438A6EE81FF81E456F64EA081FE0176
:100F6E00E45FFE4FE081EA1711F00C94CA8710304F
:100F7E0011F40C94C687EE81FF810E9415B6E1E054
:100F8E000E9407B60895AE81BF812A173B0710F461
:100F9E000C94D687003011F00C94D68701C001C096
:100FAE00BDCF0E94D2B511F40C94E0870E94E7B534
:100FBE0002C00E94F4B5003011F40C94EB8710308F
:100FCE0011F40C94EB8701C005C00E94FDB50E9480
:100FDE0007B60895003011F40C94F987E1E00E94F1
:100FEE0007B60895E0E00E9407B608950E9407B67E
:100FFE0008950E94ACB95A2F40E0E52F0E941AB610
:10100E000E9422B62017310710F00C941C88E42F92
:10101E004F5FAE81BF810E946AA90E9428B6EC91F3
:10102E00D001EC932F5F3F4FEDCFAE81BF810E9479
:10103E002DB60E94B3B928960895E091A21BF091A7
:10104E00A31B0E9415B608950A930A2FE02FA091B4
:10105E009E1BB0919F1BF0E0EA0FFB1F0E9415B67E
:10106E00E02F0E941AB6E093A21BF093A31B0991E6
:10107E000895AA9321970E9471AA40E0EF810E94E1
:10108E001AB60E9422B62017310710F00C94688809
:10109E000E9428B65C91523211F00C945F88A8859C
:1010AE00B9850E942DB6EE810E94B3B92A96089595
:1010BE00E42F4F5FA885B9850E9436B62F5F3F4F4C
:1010CE00E2CF2093A21B3093A31B0E9455A7089535
:1010DE00AA9321970E9471AA40E0E8850E941AB651
:1010EE000E9422B62017310710F00C9498880E94A7
:1010FE0028B65C91EF81E51711F00C948F88A985C5
:10110E00BA850E942DB6EE810E94B3B92B96089532
:10111E00E42F4F5FA985BA850E9436B62F5F3F4FE9
:10112E00E1CF2093A21B3093A31BE0E00E94B3B942
:10113E002B9608950A93E0E0E093D61BE093D71B1D
:10114E000E94E8AA0E9422AB11F00C94B188A0E193
:10115E000E94820EA1E00E94FB260E9495AE0E9484
:10116E003EB60E9444B60E9452B60E9441B0E1EFD4
:10117E00FBE10E9432AF0E9441B00E9459B6099124
:10118E0008950E94E8AA0E9495AE0E943EB60E9463
:10119E0044B60E9452B60E9441B0E1EFFBE10E94BC
:1011AE0032AF0E9441B00E9459B60895A0E00E944D
:1011BE00FB26E3E6E093D61BA0E10E94820E089583
:1011CE006D970E94ACB9E091D61BE03011F00C94F3
:1011DE00F588E0E00E94B3B9A3960895A091D61BBE
:1011EE00A33611F00C940589E0E00E9472AC0E94C7
:1011FE000263E0E00E94B3B9A3960895A091D61BB6
:10120E00A13011F00C941E89A0E10E94990E8F015D
:10121E00093CE0E01E0710F40C941A89E0E0E0931C
:10122E00C70F0E9465B6E0E0E093D71BF1C1A09115
:10123E00D61BA23011F00C942A89E0EF0E946BB6F7
:10124E000E9465B6E5C1A091D61BA33011F00C9497
:10125E006D89EDB7FEB7FA93EA935F930E9475B668
:10126E005F914E2F403011F00C945489513010F490
:10127E000C944889E1E00E947DB6EAEC0E9483B6A8
:10128E000895E1E0E093C70FAFE00E94820EACE05C
:10129E000E94C80E0E9465B60BC0423010F40C942A
:1012AE005F89E2E00E947DB6E9EC0E9483B6089564
:1012BE00AFE00E946BB210F40C946C89E3E00E94D4
:1012CE007DB6E8EC0E9483B60895A2C1A091D61B0C
:1012DE00A43011F00C94BA890E94F2264E2F4030A1
:1012EE0011F40C948A890E941616E1E00E946BB6E6
:1012FE00ACE00E94C80EE2E0EA93EA93A2E00E94FC
:10130E0002630E9465B6E1E00E9472AC0E94026325
:10131E00ACE00E94E40E8F010630E0E01E0710F4F0
:10132E000C94A089A091D60FA03011F00C94A08936
:10133E000EC00F31E0E01E0710F40C94AD89A091A1
:10134E00D60FA13010F40C94AD8901C00BC0E0E0B3
:10135E000E9472AC0E940263E0E00E947DB60E9481
:10136E008AB6089555C1A091D61BA53011F00C94E4
:10137E00FC89EDB7FEB7FA93EA935F930E9475B6B8
:10138E005F914E2F403011F00C94E589513010F4DE
:10139E000C94D789E4E00E947DB60E948AB6089527
:1013AE00AFE00E94820EE8A1EA93DE0117960E943A
:1013BE007F920E944E8F0E9465B60AC0423010F492
:1013CE000C94EF89E5E00E947DB60E948AB60895DE
:1013DE00AFE00E946BB210F40C94FB89E6E00E9421
:1013EE007DB60E948AB6089513C1A091D61BA63071
:1013FE0011F00C942A8A0E94508D4E2F413010F419
:10140E000C940F8AE7E00E947DB60E948AB608957A
:10141E00AFE00E94820E0E9465B6E0E00E9472ACC0
:10142E000E940263AFE00E94990E8F01053FE1E03A
:10143E001E0710F40C94298AE8E00E947DB60E94E3
:10144E008AB60895E5C0A091D61BA73011F00C9472
:10145E00498AA9EDBBE10E945F8EA9EEBBE10E9415
:10146E00748EA1EFBBE10E94898E0E949F8EE09345
:10147E00F91BF093FA1B6093FB1B7093FC1B0E94ED
:10148E0065B6C6C0A091D61BA83011F00C94E38AA5
:10149E00E0E0E093FD1B0E94E7B00E948FB6ECE106
:1014AE00FCE060E070E00E943FBB0E9493AF0E94A0
:1014BE0026B3E9EDFBE10E9460A7A0E1B0E00E9437
:1014CE007D192E2F0E94E7B00E948FB6EDE2FCE050
:1014DE0060E070E00E943FBB0E9493AF0E9426B373
:1014EE00E9EEFBE10E9460A7A8E0B0E00E947D1942
:1014FE003E2F203011F40C94898A303011F40C9464
:10150E00898A01C047C0A091EE1BA43411F00C943F
:10151E00978AA091EF1BA53511F00C94978A01C004
:10152E0004C0E1E0E093FD1B35C0A091EE1BA43496
:10153E0011F00C94A98AA091EF1BA63511F00C9412
:10154E00A98A01C004C0E2E0E093FD1B23C0A09174
:10155E00EE1BA43511F00C94BB8AA091EF1BA035A5
:10156E0011F00C94BB8A01C004C0E3E0E093FD1BB4
:10157E0011C0A091EE1BA43511F00C94CD8AA09150
:10158E00EF1BA33411F00C94CD8A01C003C0E4E02C
:10159E00E093FD1BA091FD1BA13010F40C94DC8A8E
:1015AE00A43610F00C94DC8A01C003C0ABE00E949C
:1015BE00C80E0E9465B62CC0A091D61BA93011F0A2
:1015CE000C94068BA091F91BB091FA1B8091FB1B1A
:1015DE009091FC1B0E942D912E2F203011F40C9413
:1015EE00FF8AA091FD1BA13010F40C94FF8A01C05C
:1015FE0003C0E4E6E093FD1B0E9465B609C0A0910E
:10160E00D61BAA3011F00C940F8BE3E6E093D61B99
:10161E000E948AB608951A930A938D01A091FD1B1C
:10162E00A13010F40C94208BA43610F00C94208B67
:10163E0001C009C0E1EFFBE1FA93EA931A930A9312
:10164E000E94C0B106C01A930A93E0E0EA930E948A
:10165E0041B0E091FD1B0991199108951A930A93D7
:10166E00ABE00E9489B210F40C94408BE0E0E09362
:10167E00FD1BA091FD1BA13010F40C944B8BA436D6
:10168E0010F00C944B8B01C004C0E1E0099119914C
:10169E000895E0E0099119910895E0E0E093FD1BB3
:1016AE0008950E94ACB91A2F2E813F814885598525
:1016BE000C85043010F00C948C8BA7E00A9FF0017F
:1016CE00EC55F44EAB85A083A7E00A9FF001EB55D5
:1016DE00F44EAA85A083A7E00A9FF001EA55F44EC6
:1016EE0050830A9FF001E955F44E40830A9FF001A2
:1016FE00E855F44E30830A9FF001E755F44E2083EF
:10170E000A9FF001E655F44E10830E94B3B92D9650
:10171E0008950E94AEB99D010C91043010F00C9406
:10172E00C58BA7E00A9FF001EC55F44EA081AB3BB0
:10173E0011F00C94A78BF9013196ABEBA08304C08A
:10174E00F9013196AAEAA08310E0163010F00C943D
:10175E00C48BE12FF0E03296E20FF31FBF01A7E03A
:10176E000A9FF001EB55F44EDF01EE27A10FBE1FCD
:10177E00EC91DB01EC931F5FE8CF12C0F9013196BB
:10178E00AAEAA08310E0163010F00C94D78BE12F4C
:10179E00F0E03296E20FF31FAFEFA0831F5FF3CF9F
:1017AE000E94B5B924960895A4970E94ACB95A2FF9
:1017BE0020E0E0E0E0939118E0917E18E03011F027
:1017CE000C94EE8BE1E00E94B3B9AA96089558A34B
:1017DE00A8A1A83210F40C94F98BE2E00E94B3B9E0
:1017EE00AA960895A0917F18A13011F00C94058C43
:1017FE00A8A1A03110F40C94058C01C005C0E2E044
:10180E000E94B3B9AA960895DE0190960E94908B1D
:10181E00E0E0E8A740E0E2E0EA93E8E00E9493B659
:10182E00EDB7FEB7FA93EA930F93EDB7FEB7FA93BF
:10183E00EA931F930E949AB61F910F913E2F0E941A
:10184E000CAA313011F00C94328C2F5F243610F02C
:10185E000C94328C01C001C0E3CF4F5F453010F0C5
:10186E000C943E8C303011F40C943E8C01C001C0AF
:10187E00D2CFE091D51B2E1710F40C944B8CE4E0D4
:10188E000E94B3B9AA960895303011F40C94548C7A
:10189E00E5E00E94B3B9AA9608950093911802301C
:1018AE0011F40C945F8CE6E00E94B3B9AA960895E9
:1018BE00E8A1E09392180E949EB60895BA93AA9357
:1018CE006C970E94A3B64CA148A3E0E0E9A350E0B8
:1018DE00E3E0EA93E1E00E9493B6EDB7FEB7FA9328
:1018EE00EA930F93EDB7FEB7FA93EA931F930E9414
:1018FE009AB61F910F913E2F0E940CAA313011F013
:10190E000C948F8C2F5F243610F00C948F8C01C0AA
:10191E0001C0E3CF5F5F553010F00C949B8C3030DC
:10192E0011F40C949B8C01C001C0D2CFE091D51B59
:10193E002E1710F40C94A88CE3E00E94B3B9A59670
:10194E000895303011F40C94B18CE4E00E94B3B9D8
:10195E00A596089500939318003011F40C94BC8C46
:10196E00E5E00E94B3B9A5960895103111F40C94D8
:10197E00C58CE6E00E94B3B9A596089520E020310B
:10198E0010F00C94D88CE22FAAA1BBA10E946AA9D8
:10199E00E22FF0E00E947BA7EC91D001EC932F5F39
:1019AE00EECFE0E00E94B3B9A5960895BA93AA933C
:1019BE00AC970E94A3B64CA948A320E0203110F0AA
:1019CE000C94FB8CE22FEF5FF0E0DE019096EA0FB5
:1019DE00FB1F0F01AAA9BBA9EE27A20FBE1FEC91F8
:1019EE00D001EC932F5FEACFE0E0E9AB50E0E4E00A
:1019FE00EA93E1E10E9493B6EDB7FEB7FA93EA934C
:101A0E000F93EDB7FEB7FA93EA931F930E949AB61F
:101A1E001F910F913E2F0E940CAA313011F00C94A1
:101A2E001E8D2F5F243610F00C941E8D01C001C048
:101A3E00E3CF5F5F553010F00C942A8D303011F4E7
:101A4E000C942A8D01C001C0D2CFE091D51B2E1768
:101A5E0010F40C94378DE3E00E94B3B9E596089527
:101A6E00303011F40C94408DE4E00E94B3B9E59649
:101A7E00089500939318003011F40C944B8DE5E00B
:101A8E000E94B3B9E5960895E0E00E94B3B9E596D9
:101A9E0008950A93E0917E18E03011F00C945A8D5F
:101AAE00E1E0099108950E94A18D0E2F0E94E68F0C
:101ABE00013010F40C94668DE2E0099108950E94B5
:101ACE00E08D0E2F013010F40C94708DE3E009912F
:101ADE0008950E94248E0E2F013010F40C947A8DEE
:101AEE00E4E0099108950E94028F0E2F013010F448
:101AFE000C94848DE5E0099108950E94408E0E2F7E
:101B0E00013010F40C948E8DE7E009910895E0E019
:101B1E00099108950E94C9A60217130710F00C949C
:101B2E009D8D0E9492A70F5F1F4FF6CF0E94B3B9F3
:101B3E0028960895A29780E1002470E0ECECFBE07B
:101B4E0060E00E94BAB90E94AFB9E4ECF0E1FA93FA
:101B5E00EA93A0E0B1E00E94918D00E0003110F018
:101B6E000C94DB8D0E949DAF2C912A93DE0154962E
:101B7E000E940E901E2F103011F40C94CB8DE1E0CC
:101B8E000E94B6B9A59608950E94AAB6E02FF0E07D
:101B9E000E942FBAEC53FF4EFA93EA93A0E1B0E005
:101BAE000E94961A0F5FDACFE0E00E94B6B9A596B2
:101BBE00089562971A930A930E94AFB610F40C948C
:101BCE00ED8DE1E019810881649608951E85EE85FC
:101BDE00ED5FEE87E0E0EA930E94A9B1A1E00E94DA
:101BEE007B900E2F043011F00C94028EE0E01981E0
